:020000040000FA
:1000000068050020F5150000852D0000891400000A
:10001000891400008914000089140000891400006C
:10002000891400008914000089140000E10F000009
:100030008914000089140000890F00001B2D0000A6
:10004000B5150000B5150000B5150000B515000088
:10005000B5150000B5150000B5150000B515000078
:10006000B5150000B5150000B5150000B515000068
:10007000B5150000B5150000B5150000B515000058
:10008000B5150000B5150000B5150000B515000048
:10009000B5150000B5150000B5150000B515000038
:1000A000B5150000B5150000B5150000B515000028
:1000B000B5150000B5150000B5150000B515000018
:1000C000B5150000B5150000B5150000B515000008
:1000D000B5150000B5150000B5150000B5150000F8
:1000E000B5150000B5150000B5150000B5150000E8
:1000F000B5150000B5150000B5150000B5150000D8
:10010000B5150000B5150000B5150000B5150000C7
:10011000B5150000B5150000B5150000B5150000B7
:10012000B5150000B5150000B5150000B5150000A7
:10013000B5150000B5150000B5150000B515000097
:10014000B51500007BB972B90029BEBF00204FF081
:10015000004106E008BF00281CBF6FF000414FF0CF
:10016000FF3000F0AFB9ADF1080C6DE904CE002905
:1001700009DB002B1ADB00F035F8DDF804E0DDE9DF
:10018000022304B07047404261EB4101002B1BDBAE
:1001900000F028F8DDF804E0DDE9022304B0404275
:1001A00061EB4101524263EB43037047524263EB00
:1001B000430300F017F8DDF804E0DDE9022304B0A2
:1001C000404261EB41017047524263EB430300F050
:1001D00009F8DDF804E0DDE9022304B0524263EBE4
:1001E000430370472DE9F0478C46089D04468A4634
:1001F000002B4AD18A42174662D9B2FA82F64EB132
:10020000C6F1200E01FA06F3B740B44020FA0EFE04
:100210004EEA030A4FEA1748230C1FFA87F9BAFB84
:10022000F8FE08FB1EAA0EFB09F243EA0A439A42B3
:100230000BD9FB180EF1FF312CBF012000209A4290
:1002400002D9002800F02A818E469A1AA3B2B2FB86
:10025000F8F008FB102200FB09F943EA0244A1452B
:1002600007D93C1900F1FF3302D2A14500F21081F9
:100270001846A4EB090440EA0E4000211DB1F440E9
:100280000023C5E90043BDE8F0878B4208D9002D63
:1002900000F0F2800021C5E9000C0846BDE8F087B7
:1002A000B3FA83F100294ED16345C0F0E880824261
:1002B00040F2E5800846002DE5D0C5E9004AE2E7B6
:1002C00002B9FFDEB2FA82F6002E40F099808B1A56
:1002D0004FEA124E1FFA82F801214FEA144CB3FB89
:1002E000FEF20EFB123008FB02F94CEA004CE1452D
:1002F00008D917EB0C0C02F1FF3302D2E14500F2F2
:10030000CA801A46ACEB090CA3B2BCFBFEF00EFB94
:1003100010CC08FB00F843EA0C44A0450ED93C1968
:1003200000F1FF332CBF4FF0010C4FF0000CA04543
:1003300003D9BCF1000F00F0A8801846A4EB080414
:1003400040EA02409AE7C1F120048B4002FA01FE24
:100350000CFA01F6E24020FA04F72CFA04FC00FA49
:1003600001F813433E431F0C320C1FFA83F9BCFB08
:10037000F7F007FB10CC00FB09FA42EA0C4CE2450F
:1003800008D913EB0C0C00F1FF3202D2E24500F267
:1003900089801046ACEB0A0CB6B2BCFBF7FA07FB3F
:1003A0001ACC0AFB09F946EA0C42914506D99A187B
:1003B0000AF1FF3601D291457AD8B2464AEA0040A6
:1003C000A2EB0902A0FB0E67BA42B446B94602D3BB
:1003D00007D1B04505D2B6EB0E0C67EB030301382D
:1003E0009946002D6BD0B8EB0C0362EB090202FAC0
:1003F00004F4CB40CA4000211C43C5E9004242E757
:10040000B740C6F1200201FA06F3B44021FA02FC1B
:100410004FEA174E20FA02F21FFA87F8BCFBFEF1F2
:100420001A430EFB11CC01FB08F0130C43EA0C4CF1
:10043000604507D917EB0C0C01F1FF3301D2604581
:1004400033D81946ACEB000C92B2BCFBFEF00EFBAD
:1004500010CC00FB08F342EA0C4C634507D917EBBC
:100460000C0C00F1FF3201D2634525D81046ACEBED
:10047000030340EA014130E72946284603E7841A8E
:100480006CEB030301209A4615E702383C4455E71C
:1004900002383C44EDE6023ABC4433E7AEF1020ECA
:1004A0003B44D2E602389C4474E70239BC44C9E7B5
:1004B000AAF1020A1A4481E70238BC44D7E7294668
:1004C000E1E600BF704700BF2DE9E04F2746A04698
:1004D000A146A246A346A4462DED108B4FF0000581
:1004E00045EC185B45EC195A45EC1A5A45EC1B5A79
:1004F00045EC1C5A45EC1D5A45EC1E5A45EC1F5A5A
:10050000F1EE105A4FF66076C0F6FF763540E1EE18
:10051000105A84F3008825462646A447BDEC108B6C
:10052000BDE8E08F82680C4B9A60036883F388888B
:10053000436883F38988027B02F00101EFF394831F
:1005400023F00303920748BF43F0020309B143F0CD
:10055000010383F39488704700ED02E0084AD368F2
:1005600048B123F400531B041B0C43F0BF6343F456
:100570000033D36070479BB243F40053F5E700BFEC
:1005800000ED00E0084AD36840B19BB243F48043D9
:1005900043F0BF6343F40033D360704723F48043D8
:1005A0001B041B0CF4E700BF00ED00E0084AD36811
:1005B00040B19BB243F0080343F0BF6343F4003300
:1005C000D360704723F008031B041B0CF4E700BF43
:1005D00000ED00E0084B1A6818B142F001021A6001
:1005E000704722F001021A601A6811B142F002024B
:1005F000F5E722F00202F2E7D0ED00E00B680133EC
:100600000B60014B1B681847A80E00202DE9F04F26
:1006100085B00E9C9B46012CB8BF0124012B0CBF5A
:100620003023202315468046894601260A270022CA
:10063000DFF870A0019402930AF101040AB9AA45F7
:100640001ED2B5FBF4F049463030C04701220136D6
:10065000B5FBF4F10A23013F012F04FB1155BAFB4E
:10066000F3FAE9D1494605F13000C047BBF1030F69
:1006700003D1019B9C1B002C0FDC05B0BDE8F08F63
:10068000019BBB42E4DBBBF1020FE1D84946029873
:1006900003920136C047039ADAE749462020C04753
:1006A000013CE8E7FFC99A3B014B1860704700BF67
:1006B000A80E0020002313B502AC44F8043D024606
:1006C0000B460348214602F07CF902B010BD00BF82
:1006D000FD05000010B54FF02003EFF3118483F304
:1006E0001188BFF36F8F00F013F80122064BC3F897
:1006F00040254FF0FF32054B9A62DA6284F311888D
:10070000BFF36F8F002010BD0090035000ED00E09C
:10071000524A136843F0020313600022D30003F52A
:100720007F03D3F80013013108D0D3F8001301324E
:10073000D3F80433B2F5807F0B60EFD1484AD36918
:1007400013F001033BD0474B1946D3F80024012A8C
:10075000FBD1C3F80425D1F80034012BFBD1404B69
:10076000DA69D20708D5DA693E4922F00102DA6176
:10077000D1F80024012AFBD11A6A01320AD11A6A7F
:1007800022F0FF0242F020021A62364AD2F8003408
:10079000012BFBD10022334BC3F80425D3F80024EE
:1007A000012AFBD1BFF34F8F2F49304BCA6802F4A7
:1007B000E0621343CB60BFF34F8F00BFFDE7126AC7
:1007C0000132C0D02A4A116809290AD12949096889
:1007D000013901299EBF4FF05021C1F81431C1F8F1
:1007E00018311368092B09D1224B1B68012B01BF5B
:1007F000214A1360A2F63822C2F878351C4B1A68D9
:10080000092A0BD11B4A1268022A07D100211A4A71
:1008100011600121A2F63822C2F878151B68092B55
:1008200006D1144B1B68022B02BF0C22134B1A601B
:100830000D4BD3F88C2042F44062C3F88C20D3F8DF
:10084000882042F47002C3F88820BFF34F8FBFF3B3
:100850006F8F0B4B0B4A1A60704700BFD0ED00E062
:100860000080FF000090035000ED00E00400FA0556
:100870003001FF003401FF00384A0050E4AE03505D
:10088000AC0E00200090D0030A2838B50446074D6E
:1008900004D128680D2143685B6898472868E1B255
:1008A00043685B689847204638BD00BF08000020B9
:1008B00010B5044C204601F09FF82046BDE81040DA
:1008C000FFF7F2BE8908000008B5044801F084FB78
:1008D000034B1860FFF7ECFF002008BDB3360000A3
:1008E0000800002010B54FF02003EFF3118283F3CE
:1008F0001188BFF36F8F154C237833B982F31188B9
:10090000BFF36F8F6FF0440010BD013BDBB223706B
:1009100033B182F31188BFF36F8F6FF00F00F3E7ED
:100920000B4B0121187838B1217082F31188BFF385
:100930006F8F6FF00A00E7E7197082F31188BFF339
:100940006F8F044A11601870DEE700BF5E0100205F
:100950005D0100200450005010B54FF02002EFF36D
:10096000118382F31188BFF36F8F144C207898B1F4
:1009700083F31188BFF36F8F4FF05022D2F81C34ED
:10098000D2F8182403F0030343F48033934314BFD5
:100990006FF04300002010BD0122227083F3118804
:1009A000BFF36F8F4FF05023C3F80401C3F818153D
:1009B0000221C3F804139A60DEE700BF5C01002047
:1009C000F8B54FF02002EFF3118382F31188BFF3E3
:1009D0006F8F294A1078441C147080B183F31188FA
:1009E000BFF36F8F4FF05023D3F80C3403F0011393
:1009F000B3F1011F0CBF00206FF0430009E01F4D51
:100A00002F783FB1107083F31188BFF36F8F6FF0B1
:100A10000A00F8BD01262E7083F31188BFF36F8F93
:100A20004FF0502421B3052000F0CCFCC4F8007135
:100A3000D4F80433C4F804632660D4F800219AB1D2
:100A40000022DB0758BF0123C4F800214FF0200229
:100A500058BFC4F808330A4B0520C3F8802100F0C2
:100A6000A1FC00232B70BDE720BF40BF20BFE4E7FF
:100A7000C4F800112660F4E75E0100205D0100204B
:100A800000E100E00022114B10B4C3F840214FF008
:100A90002002EFF3118482F31188BFF36F8FD3F834
:100AA000040540F247130A4A1168401A20F07F40BB
:100AB000B0FBF3F003FB0013136084F31188BFF362
:100AC0006F8F5DF8044B01F079BE00BF00500150FC
:100AD0000C00002038B51B4801F07EFA70B3436863
:100AE00002211B689847002440F24713164D4FF42B
:100AF0000012C5F80845C5F840354FF48033C5F8F5
:100B00004433C5F80433114B01211C60104B1520F0
:100B1000C3F88021224600F069FC152000F042FC59
:100B2000012320460B4A13602B60D5F8043503F2ED
:100B3000471323F07F43C5F8403538BD4FF0FF30F1
:100B4000FBE700BFBA360000005001504051015091
:100B500000E100E0085001504CF6690270B5B0F1B8
:100B6000FF3F08BF10464FF02003EFF3118483F3DB
:100B70001188BFF36F8F01389042124DA8BF104605
:100B80002E6840F24715104920EAE070D1F804358C
:100B90009A1B22F07F4202F5A37205FB0020B0FBF6
:100BA000F5F005FB0060C31A23F07F431F2B98BFAD
:100BB000401920F07F40C1F8400584F31188BFF34D
:100BC0006F8F70BD0C000020005001504FF02002CC
:100BD000EFF3118382F31188BFF36F8F084AD2F8C5
:100BE0000405084A1268801A40F2471220F07F403C
:100BF000B0FBF2F083F31188BFF36F8F704700BF33
:100C0000005001500C000020312810B500F5007193
:100C100009D0134B53F82130002B1DDA03F00303E6
:100C2000023B012B18D843B2002B0CDB012200F051
:100C30001F04A2405B090B4C203344F82320BFF370
:100C40004F8FBFF36F8F064B074A43F821200021D7
:100C500002F067F8002010BD4FF0FF30FBE700BF47
:100C60000030005000E100E00001008030B54FF49A
:100C7000004448F2040585B04FF400412F4801F0CC
:100C8000FCFF21682E4801F0F8FF29682D4801F08B
:100C9000F4FF10220021684602F0BDF82368684680
:100CA00000930294FFF73EFC0120FFF76BFC00204D
:100CB000FFF754FC0020FFF779FC01210020FFF72B
:100CC00089FC214A2148D2F88C3043F44063C2F8B1
:100CD0008C302C6801F0D1FF0820FFF795FF24F03D
:100CE0000104BFF34F8FBFF36F8F64086400204689
:100CF0002146224623469FED160ADFED150A9FED99
:100D0000141ADFED131A9FED122ADFED112A9FED61
:100D1000103ADFED0F3A9FED0E4ADFED0D4A9FEDE1
:100D20000C5ADFED0B5A9FED0A6ADFED096A9FED61
:100D3000087ADFED077AFFF7C7FB00BFA537000091
:100D4000BC370000D137000000ED00E0EF370000B5
:100D5000000000002DE9F8435D4801F08EFF0021FE
:100D6000DFF8AC815B4F5C4D58F82140CA0301F5B8
:100D7000C07347F82340594802F500434E1C01F068
:100D80007CFF574B14F0100F5649574808BF1946BF
:100D900001F073FF14F0040F14BF72212D212846B7
:100DA00001F06BFF14F0020F14BF77212D212846AC
:100DB00001F063FF14F0010F14BF78212D212846A4
:100DC00001F05BFF14F4807F14BF6C212D212846B5
:100DD00001F053FF454801F050FF202E3146C3D1AA
:100DE000424801F04AFF424801F047FF0021DFF886
:100DF0002481384F384D58F821404A0301F5E073FB
:100E000047F823403B4802F500534E1C01F035FFE4
:100E1000334B14F0100F3349334808BF194601F023
:100E20002CFF14F0040F14BF72212D21284601F06D
:100E300024FF14F0020F14BF77212D21284601F062
:100E40001CFF14F0010F14BF78212D21284601F05A
:100E500014FF14F4807F14BF6C212D21284601F06B
:100E60000CFF224801F009FF202E3146C3D1002497
:100E70001E4801F002FF204801F0FFFE154B1F4DF8
:100E8000DFF89480DFF89490C3F8C04405EBC40603
:100E9000777955F83420002F14BF43464B4621463E
:100EA000174801F0EAFE57B91648013401F0E5FE93
:100EB000122CEBD10D48BDE8F84301F0DEBE3079CD
:100EC000FFF7A2FE08B11048EFE71048EDE700BFBA
:100ED000F836000000300050303700001B370000AB
:100EE000E1360000D83600008E370000863B000057
:100EF00033370000553700006937000038350000EF
:100F0000853700009137000098370000A0370000B7
:100F1000B8340000C8350000ED360000E5360000AA
:100F200004488168406A884203D003494FF08052E8
:100F30000A6070471C01002004ED00E0002320211E
:100F40000348C2180133412B82F80013F9D17047CE
:100F500000E100E0094A0A49936809685866996601
:100F600008494B6843F080534B60002383F311889A
:100F7000BFF36F8F9368986E704700BF1C0100200D
:100F80009C36000000ED00E0202080F31188BFF3C4
:100F90006F8F11498A684FF028001044EFF3098CD5
:100FA00080E8F01F0D4F4FF000664A6A8A603E608D
:100FB000506E0023536680F3118804B5064880689C
:100FC00001F0E7FEBDE8044002F1280090E8F01FC0
:100FD0008CF30988704700001C01002004ED00E03C
:100FE0001EF0040F0CBFEFF30880EFF30980816956
:100FF00031F8021C11F0FF010229FFD001B501F008
:10100000B9FE01BD38B51B4C05461B4801F035FE45
:10101000A36AD90602D5194801F02FFEA36A1A0760
:1010200002D5174801F029FEA36A9B070ED5154883
:1010300001F023FE616BA36A180607D5124801F080
:101040001CFE1DB1A36A23F08003A362094CA36AAE
:10105000DA0702D50D4801F010FEA36A9B0602D5FF
:101060000B4801F00AFEA36AA36A002043F0FF03C5
:10107000A36238BD00ED00E0563900006D39000074
:10108000A1390000B5390000CE390000E539000073
:10109000053A000038B51E4C05461E4801F0EDFD2E
:1010A000A36AD90402D51C4801F0E7FDA36A1A051A
:1010B00002D51A4801F0E1FDA36A9B050ED5184838
:1010C00001F0DBFDA16BA36A180407D5154801F0F8
:1010D000D4FD1DB1A36A23F40043A3620C4CA36AA0
:1010E000590502D5104801F0C8FDA36ADA0509D5F3
:1010F0000E4801F0C2FD064A0020936A43F47F4384
:10110000936238BDA36A9B04F5D50948F1E700BF97
:1011100000ED00E0C8380000DF380000A139000011
:10112000F13800000B390000213900003D39000082
:10113000053A000010B51C4C1C4801F09EFDA36A46
:101140009A0102D51A4801F098FDA36ADB0102D585
:10115000184801F092FDA36ADC0202D5164801F09E
:101160008CFD114CA36A180302D5144801F085FDCB
:10117000A36A590302D5124801F07FFDA36A9A03BE
:1011800002D5104801F079FD074CA36ADB0302D5B4
:101190000D4801F072FDA36A00206FEA03436FEA75
:1011A0001343A36210BD00BF00ED00E0153B00003B
:1011B0002E3B0000423B00005D3B0000883B0000EE
:1011C000A73B0000CD3B0000E83B000010B51A4CE7
:1011D0001A4801F052FDA1696369580602D5184802
:1011E00001F04BFD6369D90707D5164801F045FDAD
:1011F000636943F0FF03636110BD63699A0701D51A
:101200001148F3E763695B0701D51048EEE76369AE
:10121000180701D50E48E9E76369D90601D50D48DD
:10122000E4E763699A0601D50B48DFE763691B06AB
:10123000DED50A48DAE700BFD0ED00E0353A00001D
:101240004F3A0000603A0000773A0000963A0000FA
:10125000B23A0000D03A0000E63A0000013B00003C
:101260003D4B70B55E6801F07F43B3F17F4F05469B
:101270000C465DD111F0010041D048061BD429680D
:10128000364B37480B44012B98BF296C01F0F5FC15
:1012900014F00804304B09D0EFF389855C6814F42E
:1012A000006408D12F4801F0E8FC41E0EFF38885A5
:1012B0005B681905F6D4C6F30806F21E092A3FD862
:1012C000DFE802F005383A2D343E3E3E3E3C2648EB
:1012D00001F0D3FC204BDA6A920701D52348E2E7FC
:1012E000D86A10F080400AD0214801F0C6FC214B9A
:1012F0001B784BB10120FFF785FE06282BD029462D
:10130000BDE8704000F0D2B81B4B1B781BB1012028
:10131000FFF7C0FEF1E7194B188884B214B1FFF74C
:1013200009FFEAE7164B58690028E8D0FFF74EFF9F
:101330000020E4E70020DEE70020E9E71148B2E7FB
:1013400011481249A6F110020F2ED8BF01461048CD
:1013500001F093FCECE770BD00ED00E0A6ED0501A7
:10136000423C0000623C0000873C00009F3C0000C3
:10137000C13C000028ED00E029ED00E02AED00E08E
:10138000D0ED00E0E13C0000143C0000293C0000EE
:10139000183D0000024A536943F01003536170473F
:1013A00000ED00E043B2002B08DB012200F01F003B
:1013B00002FA00F0024A5B0942F82300704700BFBE
:1013C00000E100E043B2002B0DDB012200F01F0022
:1013D00002FA00F05B09044A203342F82300BFF30D
:1013E0004F8FBFF36F8F704700E100E043B2002BD7
:1013F00001F10101A8BF03F160434FEA4111B8BFF9
:10140000054BC9B2ABBF03F5614300F00F0083F891
:1014100000131954704700BF14ED00E02DE9F041AE
:101420008C18884617461E4604220A9B09990546D1
:1014300001F09AFE00220D49A4F1200323F00703D6
:1014400021F00101C5E91322C5E9168799610699C2
:101450001E605960079999600899D9604FF08071B2
:10146000D961AB646A66BDE8F08100BF8F290000D6
:10147000014910220A60704710ED00E0404080F3FF
:10148000118830BF704700BF404080F311884FF093
:1014900004007146014202D0EFF3098001D1EFF35D
:1014A0000880714601B5FFF7DBFE01BD38B5044683
:1014B0000D4605281AD8DFE800F00319191315178F
:1014C0000D4801F0DAFB01F035F8AA6901460B4836
:1014D00001F0D3FB29462046BDE8384000F018B89B
:1014E0000748EEE70748ECE70748EAE70146074800
:1014F00001F0C3FBE7E700BF2C3D0000CA3D000040
:101500004C3D0000723D00008C3D0000A73D0000F6
:10151000052810B50CD001F013F860B101F010F8F7
:101520000C490D4B002808BF19460C4801F0A5FBDB
:10153000FFF7A4FFFCE701F013F80028EED1084CF8
:101540000848A16801F099FBA068BDE8104000F0D0
:101550000BB800BF063E00000A3E00001B3E000024
:101560001C0100203B3E000038B505464FF020032B
:10157000EFF3118483F31188BFF36F8F01F0D5FD72
:101580000A4B9B68AB420BD1094B5A68C2F3080265
:1015900012B92046FFF7DEFC5A6842F080525A60CA
:1015A0002046BDE8384001F067BD00BF1C010020A7
:1015B00000ED00E001B572B60B4A106A00281EBFAC
:1015C0000021116201F026FD62B6EFF30580A0F163
:1015D00010004FEAC0000549014409C99847BDE819
:1015E00001400348004700001C01002004320000B5
:1015F000210F000001F0C2FB00F004F830BFFFF73C
:10160000FDBF00BF08B50E4B83F30988EFF31483C9
:1016100043F0020383F31488BFF36F8F094B0A4A28
:1016200023F07F039360BFF34F8FBFF36F8F00F002
:1016300013FD00F01BFDFFF781FC00F049FD00BF2A
:10164000A80E00200000000000ED00E010B50E4BD9
:1016500088B002930D4B0E4C03930E4B08A80493D5
:1016600002AB40F81C3D0C4A2346012100F044F92E
:1016700000230793094B0121E41A05A8059306945A
:1016800000F044F908B010BD000000200000000088
:1016900000000120060001000000002000000020E2
:1016A00010B50B680C7A23F01F0304F01F021A43D5
:1016B000CB68640923F01F03044943F0010343EAA4
:1016C00044038860CA600B6110BD00BF90ED00E06C
:1016D00030B585B09DF808200D890B684C684989A4
:1016E00065F3040261F3471200938DF8082023F09C
:1016F0001F03621E134423F01F030393084B044689
:101700001B68C3F30723013B984205DC6946FFF7DA
:10171000C7FF204605B030BD6FF01504F9E700BFE4
:1017200090ED00E02DE9F04F06460F4614460025E7
:10173000DFF8488185B0BD420BDA56F82530D3F882
:101740000490B9F1000F3CD0B9F11F0F05D86FF02C
:101750001504204605B0BDE8F08F19F01F0FF6D133
:10176000D3F800A01AF01F0FF1D1504601F097F8FE
:10177000834609EB0A00013801F091F88345E6D170
:101780001BF1160FE3D0631E5B45E0DBC8F808B021
:10179000D8F80C00C8F808B0D8F8103056F8251062
:1017A00020F01F0043F01F09D1E900321A4498428B
:1017B00002F1FF3A1AD1D14505D15FFA8BF0FFF75C
:1017C00087FF0135B7E7C8F808B0D8F80C3022F029
:1017D0001F0203F01F031A43C8F80C20E0B2FFF702
:1017E00077FF10F1160FB2D0441CEAE7C8F808B032
:1017F000D8F81020013B23F01F0302F01F0213430F
:10180000D145E0B2C8F81030E9D0FFF761FF10F120
:10181000160F9CD0C8F808B0D8F80C209DF80830F6
:10182000441C62F304038DF80830D8F810309DF89A
:1018300008205B0863F3471256F825308DF808201E
:10184000D3E900231A44009209F1FF3322F01F026A
:101850001344A3EB0A0323F01F030393D8F80030CB
:10186000E4B2C3F30723013BA342FFF670AF204667
:101870006946FFF715FF0134A3E700BF90ED00E0D4
:101880000522034B5A60BFF34F8FBFF36F8F704732
:1018900090ED00E0BFF35F8F0022014B5A6070476C
:1018A00090ED00E0104970B5104D0A682E68C2F343
:1018B0000722964214D8FFF7EDFF00240C4B0B6370
:1018C000A64205D10B4B1E70FFF7DAFF002070BD5A
:1018D0006968204601EB0411FFF7E2FE0134EFE7EF
:1018E0004FF0FF30F3E700BF90ED00E078340000E8
:1018F000AAFF44005F01002010B5034C2278FFF7D7
:1019000011FF207010BD00BF5F0100202DE9F74FCF
:10191000894607460026DFF89080DFF890A0214C2A
:101920004E4519DAD7F804B0BBF1000F36D03B684A
:101930001846019300F0B3FF019B05460BEB030033
:10194000013800F0ACFF1423854203FB06F306D0F8
:101950006FF0150248F8032003B0BDE8F08F15F1D1
:10196000160F48F80350F7D09AF80020AA42F3DD8A
:10197000A5604344A560E068197B60F30401197316
:101980002169187B490861F347101873E26822F057
:101990001F025A60226922F01F021A6101360C37B9
:1019A000BEE700BF90ED00E0100000205F010020C6
:1019B00070B50E4B0E461C780022234605460C4897
:1019C0000168C1F307218B420BDB0A4B191D186814
:1019D000FFF766FE224631462846BDE87040FFF715
:1019E000A1BE836002610133EAE700BF5F0100200E
:1019F00090ED00E010000020014B1860704700BF20
:101A0000B00E0020074B03EB8000D0F8003223F427
:101A10004033C0F80032D0F8003243EA0141C0F848
:101A20000012704700258450F8B5036801F01F04C8
:101A30009B680D461B79494944EA43140023D1F8B9
:101A400004238668D2B203F5A27051F82000C0F3D7
:101A50000420844267D122FA03F0C00763D59A00BC
:101A600002F1A04202F55042D2F8100520F0010028
:101A7000C2F81005012202FA03F3C1F80833204628
:101A80000021FFF7BFFFB068E84010F0010049D027
:101A9000F068E84010F0010044D07069E84010F0B0
:101AA00001024CD0B369EB40DB0740D4336923FA21
:101AB00005F2F36923FA05F505F0010502F00103CB
:101AC000AB420CBF022501250021244E01F5A27373
:101AD00056F8230010F003002BD18B0003F1A04334
:101AE00003F55047D7F81025240222F4473222F498
:101AF0004072C7F81025D7F8102504F4F85444EACA
:101B0000054503F551431543C7F810551860D7F83C
:101B1000103543F00103C7F81035012303FA01F132
:101B2000C6F80413F8BD0133082B8CD1A7E70325B1
:101B3000CAE701310829C9D16FF01200F2E7F16953
:101B4000336920464B4023FA05F515F0010F0CBF11
:101B500003210221FFF756FF1046E3E700D00050B3
:101B600008B5094B1A786AB901210D2019700521B1
:101B7000FFF73CFC0D20FFF715FC4FF00042034B34
:101B8000C3F80423002008BD6001002000D00050ED
:101B90002DE9F74F8046856803F47040B0F5804F1B
:101BA0001E4649D02CDCB0F5805F3DD0B0F5405FDB
:101BB0003ED060BB06F44077B7F5807F3ED0A7F5F6
:101BC000007463426341012919BFD4B2A1464FF0AA
:101BD0001F0900244FF0010B06F0010C4FEA4C07DF
:101BE00047EA0C0747EA0020DFF8C8A040EA83076D
:101BF00006F00203A14523D2002003B0BDE8F08F18
:101C0000B0F5E04F16D005DCB0F5A04F0ED06FF068
:101C10001500F2E7B0F5404F04D0B0F5504FF6D1C3
:101C20000720C7E70620C5E70120C3E70320C1E777
:101C30000420BFE70520BDE70220BBE70323C2E77E
:101C4000D8F800209268117904F01F0242EA41128C
:101C500080324AF82270A9680BFA04F2002B25D0D2
:101C60001143A9606969B0064CBF11439143696192
:101C7000A96970064CBF11439143A9612969700796
:101C80004CBF114391432961E96930064CBF0A43B7
:101C900021EA0202EA61214640460193FFF7C4FEB1
:101CA0000028AAD10134E4B2019BA3E721EA020192
:101CB000D7E700BF002584502DE9F843454E35682D
:101CC000012D5BD12F464FF00009434A93681268FB
:101CD000DC69D2F80880D3E902120A40D3E9051082
:101CE000014322EA0102D8F800101B6909695C402F
:101CF0004C4022EA040482BB3260002301279C4648
:101D0000364ED6F8042307FA03F1114211D003F13D
:101D1000A05202F5515292001168012909D103F530
:101D2000A27056F82000C2F800C0C0F30420814021
:101D30000C430133082BE4D114B3274FBB68196857
:101D4000F1B10E688B681C4203D04B6822463846BE
:101D50009847AEB131463668F4E73A420AD098F86F
:101D6000043009F01F00002140EA4310FFF74AFE4B
:101D700022EA070209F101097F00BCE70024BCE761
:101D8000012D0DD10026144B9C681B689F68D4E977
:101D900002321A40D4E905310B4322EA03020AB9A0
:101DA000BDE8F883154212D0E169236997F804C0B1
:101DB0004B40F34013F0010F06F01F000CBF03214E
:101DC000022140EA4C10FFF71DFE22EA050201360F
:101DD0006D00E4E77CD10050280F002000D00050B7
:101DE00070B54B79012B23D18B79032B20D1CC7982
:101DF0002CB1012C1CD103689B681B79C3B10A79F3
:101E000012B1022A14D10E2247F6122603689B68EB
:101E10001D680B68B3426BD027D8B3F5965F61D0CD
:101E200012D8B3F5167F4DD005D8B3F5967F74D090
:101E30006FF0220052E0B3F5966F50D0B3F5166FF5
:101E4000F6D14FF41D233FE0B3F5615F4CD004D8C9
:101E5000B3F5165FECD1324B36E0B3F5964F45D073
:101E6000B3F5E14FE4D12F4B2EE0B3F5E13F48D07D
:101E700012D84DF6C026B3423DD005D8B3F5164F63
:101E8000D6D14FF41D031FE0B3F5614F36D0B3F543
:101E9000963FCDD1244B17E0B3F5E12F37D008D8CA
:101EA000B3F5613F30D0214EB342C1D14FF08063D2
:101EB0000AE0B3F5612F2DD01D4EB342B8D14FF0DB
:101EC000805301E04FF41C33C5F824358368224366
:101ED00003C9C5F86C2583E80300002070BD4FF4EA
:101EE0009E23F1E7134BEFE7134BEDE7134BEBE7C3
:101EF0004FF40003E8E74FF46503E5E74FF46B03A5
:101F0000E2E74FF0EB73DFE74FF06C73DCE74FF085
:101F1000E863D9E74FF07063D6E74FF4A033D3E717
:101F20000050270000C0750000903A0190D00300D7
:101F300040420F0000B0130000F03A0000A04E0035
:101F4000026870B59268184B14684FF000528568AB
:101F500003219A601D260022C3F87412C3F8702270
:101F6000C4F80C651C26C4F814654FF000669E602A
:101F7000C3F86C12C3F868221B23C4F808351A236F
:101F80002946C4F81035FFF72BFF58B90823C4F8C9
:101F900000351D440123C4F81001C4F83455C4F8B9
:101FA0003835236070BD00BF0025845070B5002611
:101FB000084B53F82040013053F82050A54200D878
:101FC00070BD236820465B68984700B166600C349A
:101FD000F4E700BF88360000104B70B505461E467A
:101FE0000F4C9C4204D10E4CB44209D1002412E0A3
:101FF00062681AB122681268AA420CD00C34F0E769
:1020000063680BB90C34EFE723682846196800F0C1
:10201000C8FE0028F6D1204670BD00BF340F002056
:10202000C80E002008B50B4D4FF02002EFF31183CE
:1020300082F31188BFF36F8F01F0B4F801210446D9
:102040000228D8BF084601F0BDF82C62FFF716FA47
:10205000EAE700BF1C0100200248034A0021121ACF
:1020600000F0D9BE000000206401002008B5064839
:10207000064A0749121A00F0A1FEBDE80840054AC9
:102080000549064800F09ABEA80E0020480F00201F
:10209000B43E000000000000B43E0000000000203C
:1020A00008B50220FFF782FF074800F0E6FD032095
:1020B000FFF77CFF00F09AFA00F0EAFB034A137B7B
:1020C00023F00103137308BD673E0000B000002039
:1020D00080B5414BA2B083F308880024E0223F4B37
:1020E000012783F82220DC771C765C769C76DC76F0
:1020F0005A6A3B4E42F4E0225A625A6A394D42F41F
:1021000000225A629C63DA6892B242F0BF6242F4E3
:102110000832DA60FFF73EF9FFF7AAF907AB21466C
:102120006C22184600F077FEB06020468DF82970CA
:10213000FFF73CFF3846FFF739FF00F0EFF92A4B75
:1021400075624FF48062CDE90473CDE90244CDE9B4
:102150000044264B2649284600F02EFA6B7B344675
:1021600023F0040213F01B0F6A7304D1AB6913B997
:10217000284600F001F91F4B012205930F23CDE9FA
:10218000033200231C4E4FF4A0721C493046CDE9A7
:10219000013300931A4B00F00FFA737BE66023F0D3
:1021A00004037373174BC4E90633FFF74FFA0D4866
:1021B000A56000F0EEFD0D4B134A184682F3098826
:1021C00063B64FF0000181F31188BFF36F8F0021D8
:1021D0000022002300F0DBFBA80E002000ED00E051
:1021E0001C010020B0000020A83E0000A12000003B
:1021F00068010020AD3E000044000020680500207A
:10220000252000003401002068050020EFF3058040
:102210000D2809D828B1054B586880F40060C0F338
:10222000C02080F0010070470120FAE700ED00E0D7
:1022300008B5FEF7CBFC054B054A1B680021184486
:1022400010611846BDE8084000F0BCBF54010020F2
:102250001C010020F8B50D464FF02003EFF3118468
:1022600083F31188BFF36F8F4FF4004100270022E2
:102270000B4E0C4BC1FB00671A6130464FF4A02295
:1022800000233946FDF75EFF074B1860074B1D60C2
:10229000FFF7CEFF84F31188BFF36F8FF8BD00BF47
:1022A000FFFF04001C010020540100205001002009
:1022B0004FF02003EFF3118183F31188BFF36F8F89
:1022C000044B9A68D37B013BD37381F31188BFF32E
:1022D0006F8F70471C010020094B03F128028242D6
:1022E00005D19B688B4202D14B7BDB0607D1D1E93C
:1022F00000231A600A6853600023C1E90033704765
:102300001C01002038B50D4C024604F1280000F0F5
:10231000CCFE054600B9E568A3684AB95A7BD206E7
:1023200006D1AA6922B9DA897F2A01D9636238BD48
:102330009D4201D0FFF77CFF6562F8E71C01002099
:1023400010B54FF02003EFF3118483F31188BFF32E
:102350006F8F084B01209A68D37B0133D373FFF74B
:10236000D1FF84F31188BFF36F8FBDE8104000F0F8
:1023700092BE00BF1C010020F8B54FF02003EFF320
:10238000118483F31188BFF36F8F164A114651F8F9
:10239000283F8B420CD05BB1D66A90F90E5093F96E
:1023A0000E70AF420BDCB34202D01B68002BF6D19B
:1023B000D36A01604360D36A1860D06205E05A684E
:1023C000C0E900325A6810605860437B43F0400314
:1023D00043730020FFF796FF84F31188BFF36F8FDC
:1023E000F8BD00BF1C010020F8B504464FF02003E3
:1023F000EFF3118683F31188BFF36F8F194F0146F6
:1024000007F128052846FFF767FFBB6A3A46AB424B
:102410000CD05BB1F86A94F90E1093F90E708F42EC
:102420000BDC834202D01B68002BF6D1D36A2560F7
:102430006360D36A1C60D46205E05968C4E9003166
:1024400059680C605C60637B906843F04003637381
:10245000031B58425841FFF755FF86F31188BFF31D
:102460006F8FF8BD1C0100201449154A10B58B6808
:102470001468A34203D1BDE81040FFF7D9BE002481
:102480001460104A1268BAB1DA897F2A14D80E4A49
:1024900093F90E40126894420EDB0C4A1268934284
:1024A0000AD09A6942B90A69824203DC1846FFF7EA
:1024B0009BFFE0E7121A0A6110BD00BF1C0100205B
:1024C0004C0100205401002050010020A0360000E3
:1024D00038B504464FF02003EFF3118583F31188DC
:1024E000BFF36F8F437B5A0607D501460948FFF7B4
:1024F000F3FE637B23F040036373074B9868031B71
:1025000058425841FFF7FEFE85F31188BFF36F8FE5
:1025100038BD00BF440100201C0100200021044BF5
:10252000084603F12802C3E90A22FFF793BE00BF61
:102530001C010020014B9868704700BF1C0100205F
:10254000EFF305800D2807D838B1044B586880F4A4
:102550000060C0F3C02070470120704700ED00E02C
:10256000024B9B68187B00F0010070471C010020A3
:1025700010B502464FF02003EFF3118483F3118866
:10258000BFF36F8F437B590704D484F31188BFF3E3
:102590006F8F10BD23F00403437300F0BDFD10B135
:1025A0001046FFF7E9FE2146BDE81040014800F063
:1025B00055BD00BF6101002030B587B00E9D0446B7
:1025C00004950D9D03950C9D02950B9D01950A9D0B
:1025D0000095FEF723FF044B9B6813B9236607B0F1
:1025E00030BD1B6EFAE700BF1C0100202DE9F04F43
:1025F000284E294DB04687B0B54205F130040FD3BF
:10260000FFF756FE4FF400490027234C234EDFF816
:1026100090A0444521D307B0BDE8F04FFFF790BE2E
:1026200054F8043C059354F8103C049354F8143CBB
:10263000039354F8183C029354F81C3C019354F84B
:10264000203C009354E90A2354E90C01FFF7B4FF3E
:1026500054F8303CDD642546CEE7616A4B1C04D05B
:10266000256821B92846FFF783FF3034D1E7B34608
:10267000BC46C9FB01BC4FF4A0220023584661466A
:10268000FDF760FD5146421C05F1180000F052F8BC
:10269000EBE700BF340F0020340F0020FFFF0400E1
:1026A000B7300000034B1B680BB9FEF78FBA002050
:1026B000704700BF58010020036840B1084A5268C3
:1026C000904204D01BB19A6881680A449A604268BB
:1026D000136003685A600023C0E90033704700BFED
:1026E000C00E002038B5104B1B78002B0F4B18BFC5
:1026F0004FF0FF301C6808BF6FF000409C420AD0CA
:102700004CB1A568FFF7CEFF281A00280ADBA468A1
:10271000FFF7C8FF201A064B1B6913B19842A8BFE8
:10272000184638BD0020F6E761010020C00E0020E9
:102730001C01002070B504461646C1604FF020030E
:10274000EFF3118583F31188BFF36F8FFFF7AAFFB3
:10275000012EACBF80190130174BA0601A689A4255
:1027600001D05E6832B95A68236062605A681460AA
:102770005C600BE09068A168884216DD411A9160A8
:102780005168C4E9002151680C6054601A689A428B
:1027900006D0944204D1FFF7A5FF0021FEF7DCF933
:1027A00085F31188BFF36F8F70BD091A9642A1603F
:1027B000D9D01268D6E700BFC00E00202DE9F04B3B
:1027C0000446FFF751FE4FF02003EFF3118583F32A
:1027D0001188BFF36F8F214F214EB846DFF88490E8
:1027E0003460D9F8004032684C45D7E900BC05D0C8
:1027F00024B1A368934214DD9B1AA36000241BEB51
:1028000002004CEBE271C8E900013460FFF76AFF97
:102810002146FEF7A1F985F31188BFF36F8FBDE85C
:10282000F08B1BEB03004CEBE371D31A33600023F6
:10283000C7E90001A3602046FFF73EFF85F311883A
:10284000BFF36F8FE36898474FF02003EFF31185D4
:1028500083F31188BFF36F8FC3E700BF0000002030
:1028600058010020C00E002038B5074C074DAC427F
:1028700001D3002038BD04F114032046C4E9053318
:1028800000F03AF81C34F2E7340F0020340F002037
:1028900008B5FEF75FFABDE80840FEF7E7B940E883
:1028A00000F313F4803FD8B208BF6FF015007047F3
:1028B00070B50C254D43C66890F90B007419884219
:1028C000A8BF21464FF0200492FBF4F4B8BF715921
:1028D00002F01F0001EB8401196070BD07B501AB68
:1028E000FFF7E6FF0123019A03FA00F013680343A0
:1028F000136003B05DF804FB2DE9F8430446FF22A2
:1029000000214FF00C0E4368058900685D4394F880
:102910000AC02844E2728C4505DC00252389AB42BD
:1029200022DCBDE8F883B5FBF3F20EFB01F7D4F827
:102930000C801F2A08EB0706C8BF1F324FEA93031B
:1029400006F10409C8BF520903F10303C6E901995E
:1029500023F00303D4BFE17248F8070001F101013D
:10296000C8BF00EB8200D6E76268E3686A4320686C
:102970001E1D811886509A6820464A609A68116028
:1029800099602A460021FFF7A9FF0135C6E708B57F
:102990000446084611461A46A047FFF7CBFDFEF74E
:1029A000E3FD0020704770B50D4604464520A04762
:1029B00029465220A04729462346BDE870405220B0
:1029C00018472DE9F04F4FF0000A06460F464FF02A
:1029D000FF39D04689B01C46531E0393002505E0FD
:1029E0006DB9252800F03D813946B047039B13F8A7
:1029F000010F03930028F3D109B0BDE8F08F6428DC
:102A000062D019D839280AD8312851D22D283DD082
:102A100030283ED0252808D13946B047DEE758286F
:102A200000F0A880632800F0168139462520B047C1
:102A3000039B39461878F0E7702800F0918006D89B
:102A4000692841D06C283CD06828CFD0EDE77528A4
:102A50006DD017D87328E8D1256804F1040B2B46F4
:102A60001C4614F8010B002840F0EC80B8F1030F6D
:102A700040F000815C1BA9EB0404002C00F3E6800D
:102A80005C46ABE7782875D07A28DEE74FF003087C
:102A9000ACE7B9F1000F0EDAB8F1000F00F0E780F3
:102AA000A0F13009B8F1000F08BF4FF002089DE710
:102AB000B9F1000FF4DB0A2303FB0909A9F130097E
:102AC000F0E70AF1010A91E7BAF1000F12D1256887
:102AD0000434002D05DA39462D20B0476D4209F146
:102AE000FF3943462A46CDF8009039463046FDF777
:102AF0008DFD73E7BAF1010FE9D04FF0000C4FF0F4
:102B0000FF3B073424F0070303F10804D3E9002353
:102B100012F1004043F100018C4508BF834504D207
:102B200039463046FFF73FFF58E71546D1E7BAF17F
:102B3000000F05D122680434CDF800904346D4E755
:102B4000BAF1010FF6D0073424F0070303F10804AB
:102B5000D3E90023002B08BFB2F1004FECD3DFE72D
:102B600039463020B04739467820B0474FF0080941
:102B70004FF00108BAF1010F27DC236804340793F2
:102B80000023049310220023934602930693079B8D
:102B90000BF1FF3B4FEA8B00C0F1200CA0F12001AC
:102BA00023FA00F0049B03FA0CFC40EA0C0023FA21
:102BB00001F1084310F00F0013D1069B13B9BBF1CC
:102BC000000F2ED14FF0300C11E0073424F0070332
:102BD0001A6803F108045B6807920493D2E7059A28
:102BE000D5E709288CBF4FF0570C4FF0300C394611
:102BF00060440592B047029B069501330293BBF1F6
:102C0000000FECD1B8F1030F7FF4E8AE029BC3EBE9
:102C10004905002D7FF7E2AE39462020B047013D3F
:102C2000F7E7531E91450593E9DBB8F1010F03D196
:102C300039463020B047E2E7B8F1020FDFD139461C
:102C40002020F7E73946B047234609E739462020D8
:102C5000B047013C11E72068251D3946B0472C4696
:102C6000BCE6AA46A8464FF0FF390125BEE64FF064
:102C70000108BBE65C460546B8E60FB407B504A9F3
:102C800051F8040B0191FDF715FD03B05DF804EB5D
:102C900004B0704770474FF0502330B5D3F8085157
:102CA000D3F80423D3F8004102F00102D3F804134F
:102CB000D3F8040115B10025C3F80851B4B14FF0A1
:102CC00050230024C3F8004122B14FF050230122C9
:102CD000C3F8082348B100224FF05023C3F8042161
:102CE0008A0702D50222C3F8082330BD002AF1D09A
:102CF0004FF05023D3F80C3403F00113B3F1011F4C
:102D0000E8D1E2E708B5002201210520FEF76EFBBD
:102D10000520FEF747FB002008BD70477047FEF70F
:102D2000B3BB43B2A9B1002B12DB01215B099B00AD
:102D300003F1604303F56143D3F8802200F01F00E4
:102D400001FA00F022EA0000C3F88002D3F88032D2
:102D50007047002BFCDB01225B099B0003F1604301
:102D600003F56143D3F8801200F01F0002FA00F06F
:102D70000843E9E701460068FEF798BB202383F388
:102D80001188704708B5FEF739FCBDE80840FEF72A
:102D9000C7B807B5002101A8FEF70AFE03B05DF829
:102DA00004FB0138013910F8013F11F8012F93425B
:102DB00002D1002BF7D11A46981A7047F0B581EA74
:102DC0000004A50703460BD0013B0A4491421DD1E4
:102DD000F0BD002AFCD011F8014B013A03F8014B79
:102DE0009C07F6D10C461D1F8F183E1B032E08D8DA
:102DF0006FF00305940805FB0422A400234421443A
:102E0000E2E754F8046B45F8046FEEE711F8014B64
:102E100003F8014FDAE70346F0B5C9B29C070FD1BA
:102E20001D4641EA012444EA04449F187E1B032EF8
:102E30000CD8940803EB840413449C4209D1F0BDE0
:102E4000002AFCD003F8011B013AE7E745F8044BE0
:102E5000ECE704F8011BF0E74FF0FF30704710B5C6
:102E600004688068A46801292468C06903D15840B7
:102E70006060002010BD00334FF0010118BF012336
:102E8000D04000F001009140834214BFA160E16096
:102E9000EFE770B504688068A468C06925680129F7
:102EA0006E692C696D6880EA040084EA050404EA0E
:102EB000060480EA04001CBFD04000F00100186046
:102EC000002070BD836830B5186858B10024814275
:102ED00013D108685CB95C681860A14200D15860E1
:102EE0000020086072B9002030BD2846EFE720605E
:102EF0005868814208BF5C60F2E705680446002D0F
:102F0000F3D13AB11A680A60586819600028EAD10A
:102F10005960E9E76FF01500E6E701292DE9F04176
:102F200018BFD4B2064612BF25461F2500244FF015
:102F300001088768AC4202D90020BDE8F081FB6837
:102F400008FA04F223EA0203FB6021463046FEF74A
:102F50006BFD0028F1D10134E4B2EBE701292DE942
:102F6000F04118BFD4B2064612BF25461F250024E3
:102F70004FF001088768AC4202D90020BDE8F0811B
:102F8000FB6808FA04F21343FB6021463046FEF763
:102F90004BFD0028F2D10134E4B2ECE70B46826825
:102FA00092E8030083E803000020704703689B68F1
:102FB0001B68D3F8240118B1D3F88004C3F8800447
:102FC0007047036882689B681B68D3F8100138B1AA
:102FD000127A00200A700122C3F810011A607047AB
:102FE0004FF0FF30704782B002AA02F8011D0021A5
:102FF00003689B681B68C3F82011C3F844250122AD
:10300000C3F848259A60D3F820110029FBD0DA6074
:1030100002B07047FFF782BE437BDB0603BF8069C7
:10302000B0FA80F040090020704738B504464FF0F0
:103030002003EFF3118583F31188BFF36F8F0146EF
:103040008068FFF749F9637B23F00203637385F31C
:103050001188BFF36F8F0023A36038BD08B5FFF759
:10306000D5F820B1BDE808400846FDF773BF81F3ED
:103070001188BFF36F8F08BD08B50246FFF7C6F889
:1030800020B1BDE808401046FDF764BF82F3118807
:10309000BFF36F8F08BD4FF02003EFF3118083F370
:1030A0001188BFF36F8FFFF7E7BF0368984214BF23
:1030B00018460020704750F8103C70B50446A0F147
:1030C0001805CBB14FF02003EFF3118683F311887D
:1030D000BFF36F8F294650F8100CFFF7FDF814F876
:1030E0000B3C23F0020304F80B3C86F31188BFF37A
:1030F0006F8F002344F8103C14F80B3C284623F053
:10310000140304F80B3CFFF787FF20B12846BDE805
:103110007040FFF731B970BD437BDB0603BF8069A8
:10312000B0FA80F0400900207047036D10B50446E6
:1031300003B198472046FFF7EFFF38B12046FFF76D
:10314000C7F9637B43F00803637310BD637B9B0780
:1031500002D52046FFF769FFA369002BF1D004F1E7
:10316000180000F009F8ECE7037300234273817341
:10317000C373C0E90633704710B54FF02002EFF378
:10318000118482F31188BFF36F8F03683BB1FFF79F
:1031900093FA002084F31188BFF36F8F10BD6FF096
:1031A0001500F7E710B54FF02003EFF3118483F318
:1031B0001188BFF36F8FFFF795FA84F31188BFF37F
:1031C0006F8F10BD70B504460E464FF02003EFF32D
:1031D000118583F31188BFF36F8FFFF783FAA04245
:1031E00005DD012803DD31462046FDF7B5FC85F3FA
:1031F0001188BFF36F8F70BD7047FFFFE8CFFF7F6F
:1032000001000000000000001F2D00000000000071
:103210001F2D0000000000001F2D00000000000016
:103220001F2D0000000000001F2D00000000000006
:10323000972C0000000000001F2D0000000000007F
:103240001F2D0000000000001F2D000000000000E6
:103250001F2D0000000000001F2D000000000000D6
:103260001F2D0000000000001F2D000000000000C6
:10327000B91C0000000000001F2D0000000000002D
:103280001F2D0000000000001F2D000000000000A6
:103290001F2D0000000000001F2D00000000000096
:1032A0001F2D0000000000001F2D00000000000086
:1032B000850A0000000000001F2D00000000000033
:1032C0001F2D0000000000001F2D00000000000066
:1032D0001F2D0000000000001F2D00000000000056
:1032E0001F2D0000000000001F2D00000000000046
:1032F0001F2D0000000000001F2D00000000000036
:103300001F2D0000000000001F2D00000000000025
:103310001F2D0000000000001F2D00000000000015
:103320001F2D0000000000001F2D00000000000005
:103330001F2D0000000000001F2D000000000000F5
:103340001F2D0000000000001F2D000000000000E5
:103350001F2D0000000000001F2D000000000000D5
:103360001F2D0000000000001F2D000000000000C5
:103370001F2D0000000000001F2D000000000000B5
:103380001F2D0000000000001F2D000000000000A5
:103390001F2D0000000000001F2D00000000000095
:1033A0001F2D0000000000001F2D00000000000085
:1033B0001F2D0000000000001F2D00000000000075
:1033C0001F2D0000000000001F2D00000000000065
:1033D0001F2D0000000000001F2D00000000000055
:1033E0001F2D0000000000001F2D00000000000045
:1033F0001F2D0000000000001F2D00000000000035
:103400001F2D0000000000001F2D0000E03600000E
:10341000D506000000000000E0360000C9080000EA
:1034200000000000BA360000052D0000000000007A
:10343000C4360000052D000000000000CE3600005C
:10344000D50A000000000000E0360000A5180000CA
:1034500000000000603E0000611B000064360000B8
:10346000B3360000411F000080360000E036000047
:103470006928000000000000020000008034000005
:1034800000000000A436000006000000E0FF0F006E
:1034900000000020AC36000021000000E0FF00200A
:1034A000590900000000000000000000C1090000F0
:1034B000E5080000000000001701000007010000FF
:1034C00007010000070100000701000007010000DC
:1034D00007010000070100000701000007010000CC
:1034E00007010000070100000701000007010000BC
:1034F00007010000070100000701000007010000AC
:10350000070100000701000007010000070100009B
:10351000070100000701000007010000070100008B
:10352000070100000701000007010000070100007B
:1035300007010000070100001A38000042010000E6
:1035400021380000050100002B38000015010000A3
:1035500034380000390100003D3800000901000046
:10356000483800000A000000533800002A0100001B
:103570005B3800003A010000633800002C010000B5
:103580006B3800001C010000743800001D010000B1
:103590007D3800000A010000873800000B010000A0
:1035A000913800000F0100009C380000100100005D
:1035B000A738000011010000B23800000E01000021
:1035C000BC380000310100001701000017010000A5
:1035D000170100001701000017010000170100008B
:1035E000170100001701000007010000070100009B
:1035F00007010000070100000701000007010000AB
:10360000070100000701000007010000070100009A
:10361000070100000701000007010000070100008A
:10362000070100000701000007010000070100007A
:10363000070100000701000007010000070100006A
:103640000701000007010000911B00005F2E000031
:10365000932E0000C52E00005D2F00001B2F0000E0
:10366000000000000025845000000000C32F00006F
:10367000E72F0000AD2F0000E11D00009D2F00008E
:103680000080005001000000C80E00201C0F002028
:10369000280F0020340F0020340F0020F5FFFFFF1B
:1036A00044000020464C4153485F30005352414D86
:1036B0005F3000554152545F3000434C4F434B5FE5
:1036C00033324B00434C4F434B5F31364D007379DF
:1036D000735F636C6F636B00536563757265090993
:1036E000004E6F6E2D53656375726509004E6F6EE7
:1036F0002D53656375726500466C61736820726551
:1037000067696F6E0909446F6D61696E09095065DB
:10371000726D697373696F6E730A0025303275209C
:1037200030782530357820307825303578200900FC
:103730002563005352414D20726567696F6E090918
:10374000446F6D61696E09095065726D69737369C3
:103750006F6E730A00253032752030782530357849
:1037600020307825303578090050657269706865B9
:1037700072616C0909446F6D61696E090953746166
:103780007475730A00253032752025730909257375
:103790000009534B49500A00094552524F520A0042
:1037A000094F4B0A0053504D3A204E5320696D612A
:1037B000676520617420307825780A0053504D3AAF
:1037C000204E53204D535020617420307825780AC4
:1037D0000053504D3A204E53207265736574207625
:1037E0006563746F7220617420307825780A005305
:1037F000504D3A207072657061726520746F206A56
:10380000756D7020746F204E6F6E2D5365637572E9
:103810006520696D6167652E0A004E52465F503023
:10382000004E52465F434C4F434B004E52465F5250
:10383000544331004E52465F4E564D43004E524661
:103840005F554152544531004E52465F55415254E6
:103850004532004E52465F495043004E52465F5635
:103860004D43004E52465F465055004E52465F450E
:10387000475531004E52465F45475532004E52463D
:103880005F5457494D32004E52465F5350494D33B5
:10389000004E52465F54494D455230004E52465FED
:1038A00054494D455231004E52465F54494D4552A0
:1038B00032004E52465F5341414443004E52465FF0
:1038C0004750494F544531002A2A2A2A2A20425576
:1038D00053204641554C54202A2A2A2A2A0A0020DD
:1038E00020537461636B696E67206572726F720A30
:1038F00000202050726563697365206461746120E3
:10390000627573206572726F720A00202042464110
:103910005220416464726573733A20307825780AC6
:10392000002020496D70726563697365206461745D
:103930006120627573206572726F720A00202049DF
:103940006E737472756374696F6E2062757320652F
:1039500072726F720A002A2A2A2A2A204D50552094
:103960004641554C54202A2A2A2A2A0A002020534C
:103970007461636B696E67206572726F7220286371
:103980006F6E746578742061726561206D69676817
:1039900074206265206E6F742076616C6964290AF8
:1039A000002020556E737461636B696E67206572C9
:1039B000726F720A00202044617461204163636564
:1039C00073732056696F6C6174696F6E0A002020F2
:1039D0004D4D46415220416464726573733A203004
:1039E0007825780A002020496E73747275637469B3
:1039F0006F6E204163636573732056696F6C6174E9
:103A0000696F6E0A002020466C6F6174696E672DC5
:103A1000706F696E74206C617A792073746174655B
:103A200020707265736572766174696F6E2065725D
:103A3000726F720A002A2A2A2A2A205345435552B5
:103A400045204641554C54202A2A2A2A2A0A002079
:103A500020416464726573733A20307825780A00D7
:103A60002020496E76616C696420656E74727920DD
:103A7000706F696E740A002020496E76616C69640B
:103A800020696E74656772697479207369676E6105
:103A9000747572650A002020496E76616C69642035
:103AA000657863657074696F6E2072657475726E87
:103AB0000A0020204174747269627574696F6E2007
:103AC000756E69742076696F6C6174696F6E0A0037
:103AD0002020496E76616C6964207472616E73692E
:103AE00074696F6E0A0020204C617A7920737461CA
:103AF000746520707265736572766174696F6E0AA1
:103B00000020204C617A792073746174652065729D
:103B1000726F720A002A2A2A2A2A205553414745E1
:103B2000204641554C54202A2A2A2A2A0A002020BD
:103B30004469766973696F6E206279207A65726F65
:103B40000A002020556E616C69676E6564206D65A2
:103B50006D6F7279206163636573730A002020536F
:103B60007461636B206F766572666C6F7720286373
:103B70006F6E746578742061726561206E6F742059
:103B800076616C6964290A0020204E6F20636F7093
:103B9000726F636573736F7220696E73747275638D
:103BA00074696F6E730A002020496C6C6567616CE4
:103BB000206C6F6164206F66204558435F52455406
:103BC00055524E20696E746F2050430A00202049E0
:103BD0006C6C6567616C20757365206F6620746816
:103BE0006520455053520A002020417474656D7061
:103BF0007420746F206578656375746520756E64D4
:103C00006566696E656420696E7374727563746944
:103C10006F6E0A005265736572766564204578633D
:103C2000657074696F6E20280053707572696F75C6
:103C30007320696E746572727570742028495251D0
:103C4000200020205320696E737472756374696F4D
:103C50006E20616464726573733A20203078257831
:103C60000A00524554544F4241534520646F6573D6
:103C7000206E6F74206D61746368204558435F52F5
:103C8000455455524E0A002A2A2A2A2A20484152CF
:103C900044204641554C54202A2A2A2A2A0A002028
:103CA00020427573206661756C74206F6E20766596
:103CB00063746F72207461626C6520726561640A5E
:103CC0000020204661756C7420657363616C6174BB
:103CD000696F6E20287365652062656C6F77290AAD
:103CE000002A2A2A2A2A204465627567206D6F6E91
:103CF00069746F7220657863657074696F6E2028CF
:103D00006E6F7420696D706C656D656E7465642985
:103D1000202A2A2A2A2A0A002A2A2A2A2A2025731D
:103D200020256429202A2A2A2A2A0A002A2A2A2A1D
:103D30002A204861726477617265206578636570D6
:103D400074696F6E202A2A2A2A2A0A002A2A2A2A15
:103D5000204B65726E656C20416C6C6F6361746999
:103D60006F6E204661696C75726521202A2A2A2AA5
:103D70000A002A2A2A2A2A204B65726E656C204F77
:103D80004F505321202A2A2A2A2A0A002A2A2A2A7C
:103D90002A204B65726E656C2050616E696321202C
:103DA0002A2A2A2A2A0A002A2A2A2A20556E6B6ED3
:103DB0006F776E20466174616C204572726F72205D
:103DC000256421202A2A2A2A0A0043757272656E08
:103DD0007420746872656164204944203D20257018
:103DE0000A4661756C74696E6720696E73747275CA
:103DF0006374696F6E2061646472657373203D2023
:103E0000307825780A0049535200657373656E74E3
:103E100069616C2074687265616400466174616CEC
:103E2000206661756C7420696E20257321205370A3
:103E3000696E6E696E672E2E2E0A00466174616C83
:103E4000206661756C7420696E20746872656164A7
:103E5000202570212041626F7274696E672E0A00FE
:103E60004750494F5F30002A2A2A2A2A20426F6F82
:103E700074696E67205A6570687972204F53207696
:103E8000312E31342E39392D6E6373312D726331F9
:103E90002D342D6739346237643561666665656136
:103EA000202A2A2A2A2A0A006D61696E0069646C38
:103EB00065000000A32900000090D003592E0000E7
:103EC00000C201000001030000000000C00E00203D
:103ED000C00E00200C3400000000000000000000B4
:103EE0006C340000000000000000000048340000B6
:103EF000000000000000000024340000A034000096
:103F00000000000030340000AC340000000000006D
:103F1000603400006C360000B40E0020183400003D
:103F200000000000000000003C3400000000000021
:103F30000000000054340000483600002400002037
:103F4000340F0020340F00200000000000000000AB
:043F50000F0000005E
:10800000C8360220F5A2000069C0010059A1000095
:1080100059A1000059A1000059A1000059A1000078
:1080200059A1000059A1000059A10000BD9C000009
:1080300059A1000059A10000659C00001999000099
:10804000B5A20000B5A20000B5A20000B5A20000D4
:10805000B5A20000B5A20000B5A20000B5A20000C4
:10806000B5A20000B5A20000B5A20000B5A20000B4
:10807000B5A20000B5A20000B5A20000B5A20000A4
:10808000B5A20000B5A20000B5A20000B5A2000094
:10809000B5A20000B5A20000B5A20000B5A2000084
:1080A000B5A20000B5A20000B5A20000B5A2000074
:1080B00089B7000023C70100B5A20000B5A20000E7
:1080C000B5A20000B5A20000B5A20000B5A2000054
:1080D000B5A20000B5A20000B5A20000B5A2000044
:1080E000B5A20000B5A2000045C70100B5A200007E
:1080F000B5A20000B5A20000B5A20000B5A2000024
:10810000B5A20000B5A20000B5A20000B5A2000013
:10811000B5A20000B5A20000B5A20000B5A2000003
:10812000B5A20000B5A20000B5A20000B5A20000F3
:10813000B5A20000B5A20000B5A20000B5A20000E3
:10814000B5A200007BB972B90029BEBF00204FF074
:10815000004106E008BF00281CBF6FF000414FF04F
:10816000FF3000F0C7B9ADF1080C6DE904CE00296D
:1081700009DB002B1ADB00F04DF8DDF804E0DDE947
:10818000022304B07047404261EB4101002B1BDB2E
:1081900000F040F8DDF804E0DDE9022304B04042DD
:1081A00061EB4101524263EB43037047524263EB80
:1081B000430300F02FF8DDF804E0DDE9022304B00A
:1081C000404261EB41017047524263EB430300F0D0
:1081D00021F8DDF804E0DDE9022304B0524263EB4C
:1081E0004303704753B94AB9002908BF00281CBF90
:1081F0004FF0FF314FF0FF3000F07CB9ADF1080CCB
:108200006DE904CE00F006F8DDF804E0DDE90223B4
:1082100004B070472DE9F0478C46089D04468A4615
:10822000002B4AD18A42174662D9B2FA82F64EB181
:10823000C6F1200E01FA06F3B740B44020FA0EFE54
:108240004EEA030A4FEA1748230C1FFA87F9BAFBD4
:10825000F8FE08FB1EAA0EFB09F243EA0A439A4203
:108260000BD9FB180EF1FF312CBF012000209A42E0
:1082700002D9002800F02A818E469A1AA3B2B2FBD6
:10828000F8F008FB102200FB09F943EA0244A1457B
:1082900007D93C1900F1FF3302D2A14500F2108149
:1082A0001846A4EB090440EA0E4000211DB1F44039
:1082B0000023C5E90043BDE8F0878B4208D9002DB3
:1082C00000F0F2800021C5E9000C0846BDE8F08707
:1082D000B3FA83F100294ED16345C0F0E8808242B1
:1082E00040F2E5800846002DE5D0C5E9004AE2E706
:1082F00002B9FFDEB2FA82F6002E40F099808B1AA6
:108300004FEA124E1FFA82F801214FEA144CB3FBD8
:10831000FEF20EFB123008FB02F94CEA004CE1457C
:1083200008D917EB0C0C02F1FF3302D2E14500F241
:10833000CA801A46ACEB090CA3B2BCFBFEF00EFBE4
:1083400010CC08FB00F843EA0C44A0450ED93C19B8
:1083500000F1FF332CBF4FF0010C4FF0000CA04593
:1083600003D9BCF1000F00F0A8801846A4EB080464
:1083700040EA02409AE7C1F120048B4002FA01FE74
:108380000CFA01F6E24020FA04F72CFA04FC00FA99
:1083900001F813433E431F0C320C1FFA83F9BCFB58
:1083A000F7F007FB10CC00FB09FA42EA0C4CE2455F
:1083B00008D913EB0C0C00F1FF3202D2E24500F2B7
:1083C00089801046ACEB0A0CB6B2BCFBF7FA07FB8F
:1083D0001ACC0AFB09F946EA0C42914506D99A18CB
:1083E0000AF1FF3601D291457AD8B2464AEA0040F6
:1083F000A2EB0902A0FB0E67BA42B446B94602D30B
:1084000007D1B04505D2B6EB0E0C67EB030301387C
:108410009946002D6BD0B8EB0C0362EB090202FA0F
:1084200004F4CB40CA4000211C43C5E9004242E7A6
:10843000B740C6F1200201FA06F3B44021FA02FC6B
:108440004FEA174E20FA02F21FFA87F8BCFBFEF142
:108450001A430EFB11CC01FB08F0130C43EA0C4C41
:10846000604507D917EB0C0C01F1FF3301D26045D1
:1084700033D81946ACEB000C92B2BCFBFEF00EFBFD
:1084800010CC00FB08F342EA0C4C634507D917EB0C
:108490000C0C00F1FF3201D2634525D81046ACEB3D
:1084A000030340EA014130E72946284603E7841ADE
:1084B0006CEB030301209A4615E702383C4455E76C
:1084C00002383C44EDE6023ABC4433E7AEF1020E1A
:1084D0003B44D2E602389C4474E70239BC44C9E705
:1084E000AAF1020A1A4481E70238BC44D7E72946B8
:1084F000E1E600BF704700BF70B491E87800B2E8D1
:1085000002105B1854EB0C04B2E802104D4156EB1C
:108510000C0680E878008041013070BC704770B470
:1085200091E87800B2E802105B1A74EB0C04B2E830
:1085300002108D4176EB0C0680E8780080414042C5
:1085400070BC70472DE9F00791E8F807B2E8021017
:108550005B1854EB0C04B2E802104D4156EB0C06CC
:10856000B2E802104F4158EB0C08B2E8021059EB88
:1085700001095AEB0C0A80E8F80780410130BDE898
:10858000F00770472DE9F00791E8F807B2E802100C
:108590005B1A74EB0C04B2E802108D4176EB0C060A
:1085A000B2E802108F4178EB0C08B2E8021079EBC8
:1085B00001097AEB0C0A80E8F80780414042BDE8E7
:1085C000F00770472DE9F007524290E87800B1E8D3
:1085D00080071740DB1918EA020854EB080419EA6F
:1085E000020955EB09051AEA020A56EB0A0678C099
:1085F00090E87800B1E8800717407B4118EA02084C
:1086000054EB080419EA020955EB09051AEA020AB3
:1086100056EB0A0678C080410130BDE8F00770478C
:108620002DE9F007524290E87800B1E88007174042
:10863000DB1B18EA020874EB080419EA020975EB5F
:1086400009051AEA020A76EB0A0678C090E8780073
:10865000B1E880071740BB4118EA020874EB080430
:1086600019EA020975EB09051AEA020A76EB0A060D
:1086700078C080414042BDE8F007704790E8300084
:1086800091E8C000A31B1340E41AF618EB1B13403B
:10869000ED1AFF1830C0C0C17047F0B55242FFF765
:1086A000EDFFFFF7EBFFFFF7E9FFFFF7E7FFF0BD97
:1086B0002DE9F0073AC91668A1FB069A4FF0000CA5
:1086C000E3FB06AC4FF00007E4FB06C74FF00008E1
:1086D000E5FB067840F8049B56684FF00009E1FB83
:1086E00006A91CEB090C4FF0000949EB0909E3FB53
:1086F00006C917EB09074FF0000949EB0909E4FB2C
:10870000067918EB09084FF0000949EB0909E5FB68
:10871000068940F804AB96684FF0000AE1FB06CAF0
:1087200017EB0A074FF0000A4AEB0A0AE3FB067A46
:1087300018EB0A084FF0000A4AEB0A0AE4FB068A23
:1087400019EB0A094FF0000A4AEB0A0AE5FB069A00
:1087500040F804CBD6684FF0000CE1FB067C18EB28
:108760000C084FF0000C4CEB0C0CE3FB068C19EBE7
:108770000C094FF0000C4CEB0C0CE4FB069C1AEBC4
:108780000C0A4FF0000C4CEB0C0CE5FB06AC80E83F
:108790008017BDE8F00770470A462DE9F04F41EC1D
:1087A000140A92EC080A1EC910EE100AA1FB007808
:1087B0004FF00009E2FB00894FF0000AE3FB009A4A
:1087C0004FF0000BE4FB00AB12EE100A4FF0000C70
:1087D000E1FB00BC4FF0000EE2FB00CE4FF00005C5
:1087E000E3FB00E54FF00006E4FB005605EE107ACF
:1087F00010EE900A4FF00007E1FB008719EB070924
:108800004FF0000747EB0707E2FB00971AEB070A58
:108810004FF0000747EB0707E3FB00A71BEB070B35
:108820004FF0000747EB0707E4FB00B712EE900A92
:108830001CEB070C4FF0000747EB0707E1FB00C7F5
:108840001EEB070E4FF0000747EB0707E2FB00E7C0
:10885000ED194FF0000747EB0707E3FB0057F61948
:108860004FF0000747EB0707E4FB006705EE908A2F
:1088700011EE100A4FF00008E1FB00981AEB080A0D
:108880004FF0000848EB0808E2FB00A81BEB080BC0
:108890004FF0000848EB0808E3FB00B81CEB080C9D
:1088A0004FF0000848EB0808E4FB00C813EE100A7C
:1088B0001EEB080E4FF0000848EB0808E1FB00E84B
:1088C00015EB08054FF0000848EB0808E2FB0058DC
:1088D00016EB08064FF0000848EB0808E3FB0068B9
:1088E00017EB08074FF0000848EB0808E4FB007896
:1088F00006EE109A11EE900A4FF00009E1FB00A974
:108900001BEB090B4FF0000949EB0909E2FB00B929
:108910001CEB090C4FF0000949EB0909E3FB00C906
:108920001EEB090E4FF0000949EB0909E4FB00E9D1
:1089300013EE900A15EB09054FF0000949EB090900
:10894000E1FB005916EB09064FF0000949EB090954
:10895000E2FB006917EB09074FF0000949EB090931
:10896000E3FB007918EB09084FF0000949EB09090E
:10897000E4FB008906EE90AA14EE901A01F11001B2
:108980001EC910EE100A4FF0000AE1FB00BA1CEB02
:108990000A0C4FF0000A4AEB0A0AE2FB00CA1EEB7F
:1089A0000A0E4FF0000A4AEB0A0AE3FB00EA15EB55
:1089B0000A054FF0000A4AEB0A0AE4FB005A12EEDD
:1089C000100A16EB0A064FF0000A4AEB0A0AE1FB0E
:1089D000006A17EB0A074FF0000A4AEB0A0AE2FBAB
:1089E000007A18EB0A084FF0000A4AEB0A0AE3FB88
:1089F000008A19EB0A094FF0000A4AEB0A0AE4FB65
:108A0000009A07EE10BA10EE900A4FF0000BE1FB4F
:108A100000CB1EEB0B0E4FF0000B4BEB0B0BE2FBF6
:108A200000EB15EB0B054FF0000B4BEB0B0BE3FBD7
:108A3000005B16EB0B064FF0000B4BEB0B0BE4FB54
:108A4000006B12EE900A17EB0B074FF0000B4BEB8D
:108A50000B0BE1FB007B18EB0B084FF0000B4BEB13
:108A60000B0BE2FB008B19EB0B094FF0000B4BEBF0
:108A70000B0BE3FB009B1AEB0B0A4FF0000B4BEBCD
:108A80000B0BE4FB00AB07EE90CA11EE100A4FF09F
:108A9000000CE1FB00EC15EB0C054FF0000C4CEB6F
:108AA0000C0CE2FB005C16EB0C064FF0000C4CEBE0
:108AB0000C0CE3FB006C17EB0C074FF0000C4CEBBD
:108AC0000C0CE4FB007C13EE100A18EB0C084FF0C2
:108AD000000C4CEB0C0CE1FB008C19EB0C094FF07B
:108AE000000C4CEB0C0CE2FB009C1AEB0C0A4FF058
:108AF000000C4CEB0C0CE3FB00AC1BEB0C0B4FF035
:108B0000000C4CEB0C0CE4FB00BC08EE10EA11EE80
:108B1000900A4FF0000EE1FB005E16EB0E064FF0E0
:108B2000000E4EEB0E0EE2FB006E17EB0E074FF041
:108B3000000E4EEB0E0EE3FB007E18EB0E084FF01E
:108B4000000E4EEB0E0EE4FB008E13EE900A19EBB6
:108B50000E094FF0000E4EEB0E0EE1FB009E1AEBDD
:108B60000E0A4FF0000E4EEB0E0EE2FB00AE1BEBBA
:108B70000E0B4FF0000E4EEB0E0EE3FB00BE1CEB97
:108B80000E0C4FF0000E4EEB0E0EE4FB00CE14EE7A
:108B9000100AA0EC075A80E8E05FBDE8F08F00BF44
:108BA00030B44FF0000310F8014B11F8015B013AAB
:108BB00084EA050443EA0403F5D1A3F101034FEA73
:108BC000D37030BC70474FF0000310F8012B01390F
:108BD00043EA0203F9D1A3F101034FEAD3707047CE
:108BE00011F8013B00F8013B013AF9D1704700222E
:108BF00000F8012B0139FBD1704700BF2DE9F007C8
:108C000091E8F807B2E802105B1854EB0C04B2E8E4
:108C100002104D4156EB0C06B2E802104F4158EBE2
:108C20000C08B2E8021059EB01095AEB0C0A894111
:108C3000B3F1FF3374F1FF3475F1FF3576F10006BF
:108C400077F1000778F1000879F101097AF1FF3A2C
:108C500051F100014A425B184C414D4156F100066A
:108C600057F1000758F1000859EB02095AEB010AC5
:108C700080E8F807BDE8F00770472DE9F00791E8B4
:108C8000F807B2E802105B1A74EB0C04B2E80210A9
:108C90008D4176EB0C06B2E802108F4178EB0C08A0
:108CA000B2E8021079EB01097AEB0C0A89414A42D9
:108CB0005B184C414D4156F1000657F1000758F141
:108CC000000859EB02095AEB010A80E8F807BDE8F1
:108CD000F00770470A462DE9F04F41EC140A92EC78
:108CE000080A1EC910EE100AA1FB00784FF0000917
:108CF000E2FB00894FF0000AE3FB009A4FF0000B03
:108D0000E4FB00AB12EE100A4FF0000CE1FB00BCDC
:108D10004FF0000EE2FB00CE4FF00005E3FB00E554
:108D20004FF00006E4FB005605EE107A10EE900AB4
:108D30004FF00007E1FB008719EB07094FF0000730
:108D400047EB0707E2FB00971AEB070A4FF0000713
:108D500047EB0707E3FB00A71BEB070B4FF00007F0
:108D600047EB0707E4FB00B712EE900A1CEB070C79
:108D70004FF0000747EB0707E1FB00C71EEB070EAC
:108D80004FF0000747EB0707E2FB00E7ED194FF054
:108D9000000747EB0707E3FB0057F6194FF0000702
:108DA00047EB0707E4FB006705EE908A11EE100A17
:108DB0004FF00008E1FB00981AEB080A4FF000089A
:108DC00048EB0808E2FB00A81BEB080B4FF000087B
:108DD00048EB0808E3FB00B81CEB080C4FF0000858
:108DE00048EB0808E4FB00C813EE100A1EEB080E5F
:108DF0004FF0000848EB0808E1FB00E815EB080518
:108E00004FF0000848EB0808E2FB005816EB080694
:108E10004FF0000848EB0808E3FB006817EB080771
:108E20004FF0000848EB0808E4FB007806EE109AC3
:108E300011EE900A4FF00009E1FB00A91BEB090BB2
:108E40004FF0000949EB0909E2FB00B91CEB090CE2
:108E50004FF0000949EB0909E3FB00C91EEB090EBD
:108E60004FF0000949EB0909E4FB00E913EE900A11
:108E700015EB09054FF0000949EB0909E1FB005921
:108E800016EB09064FF0000949EB0909E2FB0069FE
:108E900017EB09074FF0000949EB0909E3FB0079DB
:108EA00018EB09084FF0000949EB0909E4FB0089B8
:108EB00006EE90AA14EE901A01F110011EC910EEF0
:108EC000100A4FF0000AE1FB00BA1CEB0A0C4FF04D
:108ED000000A4AEB0A0AE2FB00CA1EEB0A0E4FF038
:108EE000000A4AEB0A0AE3FB00EA15EB0A054FF019
:108EF000000A4AEB0A0AE4FB005A12EE100A16EBCB
:108F00000A064FF0000A4AEB0A0AE1FB006A17EB77
:108F10000A074FF0000A4AEB0A0AE2FB007A18EB54
:108F20000A084FF0000A4AEB0A0AE3FB008A19EB31
:108F30000A094FF0000A4AEB0A0AE4FB009A07EE1E
:108F400010BA10EE900A4FF0000BE1FB00CB1EEBC5
:108F50000B0E4FF0000B4BEB0B0BE2FB00EB15EB9A
:108F60000B054FF0000B4BEB0B0BE3FB005B16EB21
:108F70000B064FF0000B4BEB0B0BE4FB006B12EE00
:108F8000900A17EB0B074FF0000B4BEB0B0BE1FBC1
:108F9000007B18EB0B084FF0000B4BEB0B0BE2FBCD
:108FA000008B19EB0B094FF0000B4BEB0B0BE3FBAA
:108FB000009B1AEB0B0A4FF0000B4BEB0B0BE4FB87
:108FC00000AB07EE90CA11EE100A4FF0000CE1FB67
:108FD00000EC15EB0C054FF0000C4CEB0C0CE2FB1D
:108FE000005C16EB0C064FF0000C4CEB0C0CE3FB9A
:108FF000006C17EB0C074FF0000C4CEB0C0CE4FB77
:10900000007C13EE100A18EB0C084FF0000C4CEB30
:109010000C0CE1FB008C19EB0C094FF0000C4CEB35
:109020000C0CE2FB009C1AEB0C0A4FF0000C4CEB12
:109030000C0CE3FB00AC1BEB0C0B4FF0000C4CEBEF
:109040000C0CE4FB00BC08EE10EA11EE900A4FF0A5
:10905000000EE1FB005E16EB0E064FF0000E4EEB2D
:109060000E0EE2FB006E17EB0E074FF0000E4EEBFC
:109070000E0EE3FB007E18EB0E084FF0000E4EEBD9
:109080000E0EE4FB008E13EE900A19EB0E094FF062
:10909000000E4EEB0E0EE1FB009E1AEB0E0A4FF097
:1090A000000E4EEB0E0EE2FB00AE1BEB0E0B4FF074
:1090B000000E4EEB0E0EE3FB00BE1CEB0E0C4FF051
:1090C000000E4EEB0E0EE4FB00CE53EC172A18EE0A
:1090D000104A12EB0A0253EB0B0354EB0C0455EB52
:1090E0000E05002040F1000012EB0B0253EB0C03C5
:1090F00054EB0E0455EB0E0546410020474158EB5A
:10910000000859EB0A0940F10000B2EB0E0273F1BE
:10911000000374F1000475EB0A0576EB0B0677EBA0
:109120000C0778EB0A0879EB0C0960F10000B5EB4D
:109130000B0576EB0C0677EB0E0778EB0B0879EB5B
:109140000E0960F100005FEAE07C7FEA0C0CDCF1C4
:10915000000EB2EB0C0273EB0C0374EB0C0475F114
:10916000000576F1000677F1000778EB0E0879EB41
:109170000C0960F100005FEAE07CDCF1000E12EB0C
:109180000C0253EB0C0354EB0C0455F1000556F1A3
:10919000000657F1000758EB0E0859EB0C0940F197
:1091A00000005FEAE07CDCF1000E12EB0C0253EBF6
:1091B0000C0354EB0C0455F1000556F1000657F171
:1091C000000758EB0E0859EB0C095BEC15AA51ECA3
:1091D000160A1AEB060A5BEB070B50EB080051EB83
:1091E00009015FF0000C4CF1000C1AEB070A5BEB75
:1091F000080B50EB090051EB090152EB0C025FF038
:10920000000C53EB0C0354EB0C0475414CF1000CB7
:10921000BAEB090A7BF1000B70F10000B141BA41D1
:1092200073EB0803B44175EB08056CF1000CC91B26
:1092300072EB080273EB0903BC4175EB09056CF195
:10924000000C5FEAEC787FEA0808D8F10009BAEB75
:10925000080A7BEB080B70EB080071F1000172F15A
:10926000000273F1000374EB090475EB08056CF15F
:10927000000C5FEAEC78D8F100091AEB080A5BEB06
:10928000080B50EB080051F1000152F1000253F1BC
:10929000000354EB090455EB08054CF1000C5FEAA0
:1092A000EC78D8F100091AEB080A5BEB080B50EBDD
:1092B000080051F1000152F1000253F1000354EB98
:1092C000090455EB080514EE107AA7E8000C87E8AE
:1092D0003F00BDE8F08F00BF0146014812F099BE83
:1092E00003FF010010B5084C0146084812F091FE3A
:1092F000224607490748172312F08BFE2046BDE897
:109300001040172112F092BED8FE0100B8FE0100F5
:10931000530D0200E6FE0100014812F07ABE00BFC4
:1093200021FF01002DE9F04F87B0837A00AF9B0049
:109330000A3303F4FF63ADEB030D0546436868464B
:10934000033323F00303036004460120C7F80CD065
:10935000814221D2287C0E4610F00100904601D0B7
:1093600012F0A4FB0446002E1FDAC023514A5249D2
:10937000524812F04EFE524812F04BFEC0214D48AA
:1093800012F054FE4FF0FF342146287C12F097FB78
:109390001C37BD46BDE8F08F236801309B080333BE
:1093A00023F0030344F8043FD2E7FB68298953F80C
:1093B0002630D5F800B003FB08FABB60013B03EB95
:1093C0000A027B606B680BEB0A094B439A420CD391
:1093D0003C49A423374A394812F01BFE3A4812F0A0
:1093E00018FEA421334812F021FE42463146284699
:1093F00012F03FFB0C23EA68214603FB06231A1DEB
:109400004BF80A209A68C9F804209A68C2F80090BC
:10941000C3F80890287C12F052FB287C10F0010061
:1094200001D012F043FB0446002EADD007F1140327
:1094300042463146284612F006FB042390FBF3F324
:109440007A699B001068D84000F00F000F289BD16C
:109450004FF00009CB4628F003033B603B68B5F8AA
:1094600008C003EB0902BB68696803FB02FA01FB51
:109470000CF17B680AEB0300884211D23146284682
:1094800012F005FB2A6802EB0A0152F80A004B6849
:10949000186052F80A00436042F80AB0C1F804B0FC
:1094A00009F10109B9F1040FD8D1013E98FBF9F88F
:1094B00059E700BF3DFF0100530D0200E6FE010029
:1094C000A1FF010084FF01009EFF01000B68013332
:1094D0000B60014B1B681847285902202DE9F04FFB
:1094E00085B00E9C9B46012CB8BF0124012B0CBFFC
:1094F0003023202315468046894601260A2700226C
:10950000DFF870A0019402930AF101040AB9AA4598
:109510001ED2B5FBF4F049463030C0470122013677
:10952000B5FBF4F10A23013F012F04FB1155BAFBEF
:10953000F3FAE9D1494605F13000C047BBF1030F0A
:1095400003D1019B9C1B002C0FDC05B0BDE8F08F04
:10955000019BBB42E4DBBBF1020FE1D84946029814
:1095600003920136C047039ADAE749462020C047F4
:10957000013CE8E7FFC99A3B014B1860704700BF08
:1095800028590220002313B502AC44F8043D0246DA
:109590000B460348214612F0E0FB02B010BD00BFAD
:1095A000CD94000010B54FF02003EFF3118483F346
:1095B0001188BFF36F8F00F013F80122064BC3F838
:1095C00040254FF0FF32054B9A62DA6284F311882E
:1095D000BFF36F8F002010BD0090034000ED00E04E
:1095E000074AD2F8883043F47003C2F88830BFF3DA
:1095F0004F8FBFF36F8F034B034A1A60704700BF52
:1096000000ED00E02C5902200090D00338B505464B
:1096100048B90C490C4811230C4A12F0FAFC1121EC
:109620000A4812F003FD0A4C22684AB1094906486B
:109630001223064A12F0EDFC1221044812F0F6FC47
:10964000256038BDBD0B0200E6FE0100C0FF010031
:10965000080002201E0002000A2838B50446074D03
:1096600004D128680D2143685B6898472868E1B2F7
:1096700043685B689847204638BD00BF0C00022055
:1096800010B5044C204601F091FC2046BDE8104086
:10969000FFF772BF5996000008B5044802F054FB6A
:1096A000034B1860FFF7ECFF002008BD38000200F4
:1096B0000C00022010B54FF02003EFF3118283F36A
:1096C0001188BFF36F8F154C237833B982F311885B
:1096D000BFF36F8F6FF0440010BD013BDBB223700E
:1096E00033B182F31188BFF36F8F6FF00F00F3E790
:1096F0000B4B0121187838B1217082F31188BFF328
:109700006F8F6FF00A00E7E7197082F31188BFF3DB
:109710006F8F044A11601870DEE700BF7A1E0220C6
:10972000791E02200450004010B54FF02002EFF3E4
:10973000118382F31188BFF36F8F134C207890B19F
:1097400083F31188BFF36F8F104AD2F81C34D2F81C
:10975000182403F0030343F48033934314BF6FF0E2
:109760004300002010BD0122227083F31188BFF353
:109770006F8F064BC3F80401C3F818150221C3F814
:1097800004139A60E0E700BF781E022000500040FA
:1097900038B5204BD3F80851D3F80423D3F800018F
:1097A00002F00102D3F80443D3F804111DBB78B9C9
:1097B00042BBB1B940F2451317491848184A12F094
:1097C00028FCBDE8384040F24511154812F02EBC87
:1097D0000020C3F800011AB101220E4BC3F8082380
:1097E00041B100220B4BC3F80421A20702D502228B
:1097F000C3F8082338BD0025C3F808510028E7D175
:10980000002AEDD0D3F80C3403F00113B3F1011F9B
:10981000E6D1E1E700500040A8000200E6FE0100AA
:109820004A0002002DE9F0414FF02003EFF31182CE
:1098300083F31188BFF36F8F304B18781F46441C99
:109840001C70D8B182F31188BFF36F8F3B784BB98E
:109850002B492C4860232C4A12F0DBFB60212A485C
:1098600012F0E4FB294BD3F80C3403F00113B3F1ED
:10987000011F0CBF00206FF043000CE0244D95F851
:109880000080B8F1000F08D0187082F31188BFF380
:109890006F8F6FF00A00BDE8F08101262E7082F311
:1098A0001188BFF36F8F194C21B3052000F0A2FB84
:1098B000C4F80081D4F80433C4F804632660D4F8F3
:1098C00000219AB10022DB0758BF0123C4F8002110
:1098D0004FF0200258BFC4F808330E4B0520C3F8E0
:1098E000802100F077FB00232B70AFE720BF40BF43
:1098F00020BFE4E7C4F800112660F4E77A1E0220D6
:109900003F000200E6FE01004A0002000050004055
:10991000791E022000E100E010B5064C06492246FF
:109920000648172312F075FB2046BDE810401721AA
:1099300012F07CBBE5000200530D0200E6FE0100C0
:10994000002238B5234BC3F840214FF02003EFF33A
:10995000118583F31188BFF36F8F1F4803F002FE58
:1099600060B91E494E231E4A1E4812F052FB1E4883
:1099700012F04FFB4E211A4812F058FB164803F024
:109980000FFE144B194AD3F8044540F247131168EF
:109990001148641A24F07F44B4FBF3F403FB04136E
:1099A000136003F0EDFD60B9114961230C4A0D48C5
:1099B00012F02FFB0F4812F02CFB6121084812F027
:1099C00035FB85F31188BFF36F8F2046BDE8384023
:1099D00004F0EEB8005001401400022083010200A0
:1099E0003A010200E6FE0100980102001000022088
:1099F000AD010200C401020038B51B4802F0A4F911
:109A000070B3436802211B689847002440F2471353
:109A1000164D4FF40012C5F80845C5F840354FF40F
:109A20008033C5F84433C5F80433114B01211C6061
:109A3000104B1520C3F88021224600F0EFFA1520C4
:109A400000F0C8FA012320460B4A13602B60D5F8BA
:109A5000043503F2471323F07F43C5F8403538BD82
:109A60004FF0FF30FBE700BFC7000200005001408D
:109A70004051014000E100E0085001404CF669030C
:109A8000B0F1FF3F08BF184670B5441E9C42A8BF06
:109A90001C4624EAE4744FF02003EFF3118583F3AE
:109AA0001188BFF36F8F234803F05CFD60B9224932
:109AB0004E23224A224812F0ACFA224812F0A9FAA8
:109AC0004E211E4812F0B2FA1A4803F069FD1E49F1
:109AD0001E4A0E6840F24711D2F80435981B20F058
:109AE0007F4000F5A37001FB0404B4FBF1F401FB1B
:109AF0000464E31A23F07F431F2B98BF641824F0FB
:109B00007F44C2F840450B4803F03AFD60B9104964
:109B100061230A4A0A4812F07CFA0E4812F079FAD8
:109B20006121064812F082FA85F31188BFF36F8F26
:109B300070BD00BF14000220830102003A01020040
:109B4000E6FE0100980102001000022000500140D2
:109B5000AD010200C401020038B54FF02003EFF35D
:109B6000118583F31188BFF36F8F1B4803F0FAFC54
:109B700060B91A494E231A4A1A4812F04AFA1A488A
:109B800012F047FA4E21164812F050FA124803F02C
:109B900007FD164B1048D3F80445154B1B68E41A13
:109BA00040F2471324F07F44B4FBF3F403F0E8FCE5
:109BB00060B9104961230A4A0A4812F02AFA0E488D
:109BC00012F027FA6121064812F030FA85F3118865
:109BD000BFF36F8F204638BD1400022083010200BE
:109BE0003A010200E6FE0100980102000050014027
:109BF00010000220AD010200C40102000448816887
:109C0000406A884203D003494FF080520A6070478F
:109C1000F806022004ED00E0002320210348C218CA
:109C20000133412B82F80013F9D1704700E100E0C5
:109C3000094A0A49936809685866996608494B6851
:109C400043F080534B60002383F31188BFF36F8F81
:109C50009368986E704700BFF806022070D5010027
:109C600000ED00E0202080F31188BFF36F8F1149D1
:109C70008A684FF028001044EFF3098C80E8F01F49
:109C80000D4F4FF000664A6A8A603E60506E0023B6
:109C9000536680F3118804B50648806812F0EBF92A
:109CA000BDE8044002F1280090E8F01F8CF3098819
:109CB00070470000F806022004ED00E01EF0040FDB
:109CC0000CBFEFF30880EFF30980816931F8021CC3
:109CD00011F0FF010229FFD001B512F0BDF901BD5D
:109CE00038B51E4C05461E4812F093F9A36AD904F4
:109CF00002D51C4812F08DF9A36A1A0502D51A483C
:109D000012F087F9A36A9B050ED5184812F081F965
:109D1000A16BA36A180407D5154812F07AF91DB192
:109D2000A36A23F40043A3620C4CA36A590502D52D
:109D3000104812F06EF9A36ADA0509D50E4812F040
:109D400068F9064A0020936A43F47F43936238BD62
:109D5000A36A9B04F5D50948F1E700BF00ED00E0D8
:109D6000D7010200EE01020000020200140202000C
:109D70002E02020044020200600202007902020088
:109D800010B51C4C1C4812F044F9A36A9A0102D584
:109D90001A4812F03EF9A36ADB0102D5184812F006
:109DA00038F9A36ADC0202D5164812F032F9114CD8
:109DB000A36A180302D5144812F02BF9A36A5903B9
:109DC00002D5124812F025F9A36A9A0302D5104869
:109DD00012F01FF9074CA36ADB0302D50D4812F0FD
:109DE00018F9A36A00206FEA03436FEA1343A362E2
:109DF00010BD00BF00ED00E0CA030200E303020053
:109E0000F7030200120402003D0402005C04020099
:109E1000820402009D04020038B5244C0546244803
:109E200012F0F7F8A36AD90602D5224812F0F1F829
:109E3000A36A1A0702D5204812F0EBF8A36A9B0721
:109E40000ED51E4812F0E5F8616BA36A180607D517
:109E50001B4812F0DEF81DB1A36A23F08003A36251
:109E6000124CA36AD90702D5164812F0D2F8A36A99
:109E70009A0602D5144812F0CCF8A36ADB060ED578
:109E800012494FF49E73124A124812F0C2F8124857
:109E900012F0BFF84FF49E710D4812F0C7F8034A54
:109EA0000020936A43F0FF03936238BD00ED00E0A9
:109EB000A9020200C002020000020200F402020035
:109EC0000D0302002403020079020200530D020078
:109ED00044030200E6FE01009003020038B52D4B5A
:109EE00005465C6801F07F43B3F17F4F05D0002049
:109EF0002946BDE8384000F041B9C807F7D4490603
:109F000002D5254812F085F8C4F30804E21E092A98
:109F100035D8DFE802F0052E302B343434343432B7
:109F20001E4812F076F81B4BDA6A920703D51C48DC
:109F300012F06FF8DBE7DB6A5B00D8D5194812F046
:109F400068F8194B1B782BB10120FFF765FF062835
:109F5000CED138BD154B1B781BB10120FFF7C0FED9
:109F6000F5E7134B1B889BB2002BC0D0FFF708FF0F
:109F7000EDE70020E9E70020F0E70E48D8E70E48BB
:109F80000E49A4F110020F2CD8BF01460C4812F064
:109F900040F8ACE700ED00E0F70402001B0502000A
:109FA000330502005505020028ED00E029ED00E030
:109FB0002AED00E075050200C9040200DE0402007B
:109FC000AC050200024A536943F010035361704725
:109FD00000ED00E043B2002B08DB012200F01F007F
:109FE00002FA00F0024A5B0942F82300704700BF02
:109FF00000E100E043B2002B0DDB012200F01F0066
:10A0000002FA00F05B09044A203342F82300BFF350
:10A010004F8FBFF36F8F704700E100E070B54C1CAD
:10A02000072C05460E460ED97223104A10491148D6
:10A0300011F0EFFF31461048072211F0EAFF7221BC
:10A040000A4811F0F3FF6BB2002BA8BF03F1604385
:10A050004FEA4414B8BF094BE4B2ABBF03F5614308
:10A0600005F00F0583F800435C5570BDC005020084
:10A0700011060200E6FE01002C06020014ED00E0CD
:10A0800008B572B6044B186A18B100221A6212F0B1
:10A090006AFF62B608BD00BFF80602202DE9F8434A
:10A0A0000B9E05460F2E894690461F4602D11E4B39
:10A0B0009F4214D006F110031E2B10D93F231B4AD8
:10A0C0001B491C4811F0A5FF31461B486FF00F03D8
:10A0D0000E2211F09EFF3F21144811F0A7FF0C9BA8
:10A0E00004223146284612F0E3FF002209EB08045F
:10A0F0001249A4F1680323F0070321F00101C5E927
:10A100001322C5E91698996108991F605960099949
:10A110001A6699600A99D9604FF08071D961AB6471
:10A120006A66BDE8F88300BFA1BD000061060200B9
:10A13000AE060200E6FE010035070200F1BC010098
:10A14000014910220A60704710ED00E0404080F3A2
:10A15000118830BF704700BF404080F311884FF036
:10A1600004007146014202D0EFF3098001D1EFF300
:10A170000880714601B5FFF7B1FE01BD38B5044650
:10A180000D4605281AD8DFE800F003191913151732
:10A190000D4811F03EFF03F08FF8AA6901460B4805
:10A1A00011F037FF29462046BDE8384000F018B8C6
:10A1B0000748EEE70748ECE70748EAE701460748A3
:10A1C00011F027FFE7E700BF66070200040802005E
:10A1D00086070200AC070200C6070200E107020082
:10A1E000052810B50CD003F08BF960B103F088F9A5
:10A1F0000C490D4B002808BF19460C4811F009FF07
:10A20000FFF7A4FFFCE703F08BF90028EED1084C20
:10A210000848A16811F0FDFEA068BDE8104000F0FC
:10A220000BB800BF400802004408020055080200B5
:10A23000F80602207508020038B504464FF02003E6
:10A24000EFF3118583F31188BFF36F8F037BDB0777
:10A250000CD512492523124A124811F0DAFE124891
:10A2600011F0D7FE25210E4811F0E0FE204612F035
:10A2700000FF0E4B9B68A3420BD10D4B5A68C2F3F3
:10A28000080212B92846FFF7D3FC5A6842F0805200
:10A290005A602846BDE8384012F0ACBEED08020016
:10A2A0009A080200E6FE01001B090200F8060220DF
:10A2B00000ED00E001B572B60B4A106A00281EBF1F
:10A2C0000021116212F04FFE62B6EFF30580A0F19B
:10A2D00010004FEAC0000549014409C99847BDE88C
:10A2E0000140034800470000F806022088D1010021
:10A2F000FD9B000011F0B4FE00F004F830BFFFF742
:10A30000FDBF00BF08B5164B83F30988EFF3148334
:10A3100043F0020383F31488BFF36F8F114A124B8B
:10A3200022F07F029A60BFF34F8FBFF36F8FD3F895
:10A33000882042F47002C3F888204FF00042C3F82E
:10A340003422BFF36F8FB0EE400ABFF36F8F01F07E
:10A3500041FD01F049FDFFF75FFC01F077FD00BF13
:10A36000084002200080000000ED00E010B50E4B18
:10A3700088B002930D4B0E4C03930E4B08A8049328
:10A3800002AB40F81C3D0C4A2346012100F05EF967
:10A3900000230793094B0121E41A05A805930694AD
:10A3A00000F078F908B010BD0000022000000000A5
:10A3B000000004200600010000000220000002202E
:10A3C00010B50B680C7A23F01F0304F01F021A4328
:10A3D000CB68640923F01F03044943F0010343EAF7
:10A3E00044038860CA600B6110BD00BF90ED00E0BF
:10A3F00030B585B09DF808200D890B684C684989F7
:10A4000065F3040261F3471200938DF8082023F0EE
:10A410001F03621E134423F01F030393084B0446DB
:10A420001B68C3F30723013B984205DC6946FFF72D
:10A43000C7FF204605B030BD6FF01504F9E700BF37
:10A4400090ED00E02DE9F04F06460F46144600253A
:10A45000DFF8488185B0BD420BDA56F82530D3F8D5
:10A460000490B9F1000F3CD0B9F11F0F05D86FF07F
:10A470001504204605B0BDE8F08F19F01F0FF6D186
:10A48000D3F800A01AF01F0FF1D1504611F0D2FA04
:10A49000834609EB0A00013811F0CCFA8345E6D176
:10A4A0001BF1160FE3D0631E5B45E0DBC8F808B074
:10A4B000D8F80C00C8F808B0D8F8103056F82510B5
:10A4C00020F01F0043F01F09D1E900321A449842DE
:10A4D00002F1FF3A1AD1D14505D15FFA8BF0FFF7AF
:10A4E00087FF0135B7E7C8F808B0D8F80C3022F07C
:10A4F0001F0203F01F031A43C8F80C20E0B2FFF755
:10A5000077FF10F1160FB2D0441CEAE7C8F808B084
:10A51000D8F81020013B23F01F0302F01F02134361
:10A52000D145E0B2C8F81030E9D0FFF761FF10F173
:10A53000160F9CD0C8F808B0D8F80C209DF8083049
:10A54000441C62F304038DF80830D8F810309DF8ED
:10A5500008205B0863F3471256F825308DF8082071
:10A56000D3E900231A44009209F1FF3322F01F02BD
:10A570001344A3EB0A0323F01F030393D8F800301E
:10A58000E4B2C3F30723013BA342FFF670AF2046BA
:10A590006946FFF715FF0134A3E700BF90ED00E027
:10A5A0000522034B5A60BFF34F8FBFF36F8F704785
:10A5B00090ED00E0BFF35F8F0022014B5A607047BF
:10A5C00090ED00E070B5194C194E22683568C2F361
:10A5D0000722954215D940F20313164A1649174827
:10A5E00011F017FD22682946C2F30722144811F022
:10A5F00010FD104840F2031111F018FD4FF0FF302C
:10A6000070BDFFF7D7FF0F4B23630024A54205D190
:10A610000D4B1D70FFF7C4FF0020F1E77168204665
:10A6200001EB0411FFF7CCFE0134EFE790ED00E001
:10A6300038D40100BE090200530D0200E6FE0100FD
:10A64000190A0200AAFF44007B1E022038B50C4CF8
:10A650000D462278FFF7F6FE207016300FD1C92381
:10A66000084A0949094811F0D4FC2946084811F064
:10A67000D0FCBDE83840C921024811F0D7BC38BD34
:10A680007B1E0220BE090200530D0200E6FE0100FF
:10A69000630902002DE9F74F0F4680460026DFF8D8
:10A6A000C490DFF8C4A02A4CBE4202DB03B0BDE870
:10A6B000F08FD8F804B0BBF1000F45D0D8F80030C7
:10A6C0001846019311F0B6F9019B05460BEB030008
:10A6D000013811F0AFF91423854203FB06F314D0BF
:10A6E0006FF0150249F80320D9231A4A1A491B486A
:10A6F00011F08FFC39461A4811F08BFCD92115480E
:10A7000003B0BDE8F04F11F091BC15F1160F49F8F8
:10A710000350E9D09AF80020AA42E5DDA5604B4439
:10A72000A560E068197B60F3040119732169187B47
:10A73000490861F347101873E26822F01F025A605B
:10A74000226922F01F021A61013608F10C08ABE7FA
:10A7500090ED00E0BE090200530D0200E6FE01008C
:10A760008F090200180002207B1E022070B5164BD4
:10A770000C461D7800222B46064614480168C1F39A
:10A7800007218B421BDB124B191D1868FFF718FEBF
:10A790002A4621463046FFF755FE163013D1E823EE
:10A7A0000C4A0D490D4811F034FC21460C4811F0BB
:10A7B00030FCBDE87040E821064811F037BC8360EA
:10A7C00002610133DAE770BD7B1E022090ED00E0EC
:10A7D00018000220BE090200530D0200E6FE01002F
:10A7E000360902002DE9F04F1F4600239346C9B0F9
:10A7F000CDE90C0104939BF800000BF1010548B171
:10A80000252879D0DDE90C319847013006D14FF089
:10A81000FF330493049849B0BDE8F08FAB46049B26
:10A820000133CDE90437059FE5E7232C5DD052D8ED
:10A83000002CEFD0202C08BF4FF001095D46AB463D
:10A840001BF8014BBD48214611F0D3FC0028ECD188
:10A850002A2C59D13A683B1D002A0392BEBF5242AE
:10A86000039201221F466C78B8BF069205F1020BD5
:10A87000039BC92B28BFC82303932E2C69D19BF8B7
:10A8800000302A2B62D13D680BF1010B0437C92D32
:10A89000A8BF4FF0FF359BF800400BF1010B21469C
:10A8A000A74811F0A6FC18B19BF800400BF1010B72
:10A8B000672C7CDC652C80F2E080472C4CDC452C3E
:10A8C00080F2DB80002CA5D0252C00F03583C82C2D
:10A8D00040F33C839BE72D2C0BD0302C07D02B2C46
:10A8E000079B08BF01230793A8E70126A6E7029468
:10A8F000A4E701230693A1E74FF000092023CDE947
:10A90000069902934E469AE7A4F13003092B03906F
:10A91000B3D80A22AB461BF8010BA0F13003092B78
:10A920000446A5D8039B5D4602FB0300A0F130035B
:10A930000393EFE7934600FB0535303D5A4612F886
:10A94000013BA3F130010929F4D9A0E700250A2031
:10A95000F4E74FF0FF35A2E7632C6FD032DC582CC0
:10A96000B5D13B1D05933968002E00F0DC8247F617
:10A9700030030DF15607ADF854302B4610223846FF
:10A9800011F0CEFC582C06D10DF1530212F8013F04
:10A99000002B40F0CA820DF15408002EA7EB0808E6
:10A9A000404414BF4FF002094FF0000929E0702C19
:10A9B00000F094822BDC6E2C00F0538200F357825F
:10A9C000692C84D13C683B1D002C059342DA2D2371
:10A9D000B4F1004F8DF8543041D061420DF155086B
:10A9E0002B4640460A2211F09BFC079B804415A889
:10A9F000A8EB0000002B3DD1B9F1000F01D14FEAC7
:10AA0000D4790135029B18BF2023029380E0752C76
:10AA100000F08082782CA4D0732C7FF458AF0026ED
:10AA20003B1D396805938B5D002B00F06682013673
:10AA3000C82EF8D1002D80F2628266E23B1D05939C
:10AA40003B6801268DF8543000238DF855304FF0C7
:10AA500000091CE2079B23B12B238DF854302146BB
:10AA6000BCE7B9F1000F01D02023F6E721460DF134
:10AA70005408B5E7DDF81C90C3E7073727F0070750
:10AA800007F108030593D7E900C7FB0243EA5C53CB
:10AA900023F000410B464FEACC22CDE9102340F2CF
:10AAA000FF731046C7F30A589845CDE90001604688
:10AAB00048D1DDE90012002877F10003B8BF2D234B
:10AAC00015A8AEBF03468DF854300DF155030A4367
:10AAD000A4F1410403F1030825D1192C1DD8492202
:10AAE0001A704E225A7046229A700022DA70079B22
:10AAF000A8EB0000002B40F05582B9F1000F07D100
:10AB00009DF85410A1F12D03D3F1000949EB03097D
:10AB1000C8283FF77CAE0646B9E169221A706E225A
:10AB20005A706622E0E7192C99BF4E2241216E220D
:10AB3000612194BF1A701A705970D5E74D0A02004E
:10AB4000530A0200462CDDE9002342EA080243EAE8
:10AB5000E87308BF6624134343D0DDE900230028CF
:10AB600043F00043CDE9102377F10003A8F2FE384B
:10AB700039DA2D238DF854300DF1550A0023009356
:10AB800018F1020F3EDBB8F1000F79DC10A808F1D4
:10AB9000010811F0EDFBB8F1040FF7D1002D24F0FE
:10ABA0002003B8BF0625472B40F09780002E40F0C9
:10ABB00092802B1C18BF01230893009B033304DBF6
:10ABC000009A6B1C9A4240F38D80672C0CBF652461
:10ABD000452405F10108102398450F93A8BF984616
:10ABE00089E04FF00008079B0BB12B23C2E7B9F1B6
:10ABF000000F01D02023BDE70DF1540ABEE710A8D5
:10AC000011F0B6FBDDE9107C00230B930023CDF897
:10AC100028C0A94ADDE90A018B4208BF824208F137
:10AC20000108ECD30522A7FB0201CDE90801099B2D
:10AC300002FB0C334FF0000C0993DDE90823CDE94A
:10AC40001023009B013B0093002300216FF0004084
:10AC5000099A994208BF904207D2BCF1000F8FD0E9
:10AC6000DDE90823CDE910238AE7DDE908239218FE
:10AC70005B41CDE9082308F1FF384FF0010CE3E711
:10AC800010A811F088FB4FF0000C009B08F1FF3872
:10AC900001330093DDE91023CDE9082300230021CF
:10ACA0006FF00040099A994208BF904208D2BCF167
:10ACB000000F3FF468AFDDE90823CDE9102362E718
:10ACC000DDE9082392185B41CDE9082308F1FF383C
:10ACD0004FF0010CE2E700236EE70023662C089397
:10ACE0007FF477AF009B13EB05084BD51023662448
:10ACF0004FF000080F9300224FF0006348A961E96C
:10AD0000362318F1FF383FD2DDE91023DDE91201C7
:10AD1000171843EB01083A464346CDE910230023B8
:10AD200008F07042134308D010A811F034FB10A8AB
:10AD300011F01EFB009B01330093662C0AF1010801
:10AD400040D1009B002B29DD534498460FA910A841
:10AD500011F051FB0AF8010BC245F7D10023009313
:10AD600006B95DB12E2346464FF0300A88F8003010
:10AD700008EB0503B34215D10135A844089B002B0D
:10AD800039D160E0662426E708460A9111F003FBFA
:10AD90000A99084611F0ECFA0A99B2E730238AF8CA
:10ADA0000030DDE7009A2AB1013286F801A0009256
:10ADB0000136DFE70FA910A80A9311F01CFB0A9BCC
:10ADC0007070F5E70FA910A811F015FB302818BF17
:10ADD000009B8AF800001CBF03F1FF33009306B903
:10ADE0003DB12E230AF102088AF801304544454559
:10ADF0002ED1089B43B118F8012C08F1FF33302AFB
:10AE00002DD02E2A08BF984624F02003452B1AD1B6
:10AE1000009B0A22002BBBBF5B4200932B232D23F8
:10AE200088F80130009B88F8004093FBF2F303F1AF
:10AE3000300188F80210009908F1040802FB13178A
:10AE4000303708F8017C002315A888F800304EE65A
:10AE50000FA910A811F0CFFA08F8010BC7E7984620
:10AE6000C9E73B1D0593049A3B681A60DBE43B1D70
:10AE70000593396816B330238DF8543059BB01352A
:10AE8000029B18BF202389468DF855100293039B1F
:10AE9000B34240F38580069B15AD002B58D020238C
:10AEA000039AAB550136B242FAD1DDE9033215AC53
:10AEB00013441D46A41A6FE03233333315A80DF145
:10AEC00054082B460822A0EB080811F029FA404448
:10AED0004FF0000995E50DF15500F0E73B1D059396
:10AEE00047F630033968ADF85430102208230DF1CD
:10AEF000560011F015FA0230EAE7002D02DBAE42EF
:10AF0000A8BF2E46002E3FF48EAC324615A811F095
:10AF1000B9F99CE53B1D05930A222B46396815A813
:10AF200011F0FEF9D4E715AF27E5A3F16101192966
:10AF30009CBF203B137029E50D9920460C9B984738
:10AF400001303FF464AC049B0133049305976AE439
:10AF5000039B721C9C1B2819294611F07CF9069B47
:10AF6000029A202A18BF4B4606931C44069BA34214
:10AF70009BDA069B1A46029BAB5413460133069399
:10AF8000F4E7049B0D99E05C0C9B984701303FF47B
:10AF90003EAC049B01330493049BAB42F1D142E4E9
:10AFA000039682E7DDF81C90B2E500BF014B186004
:10AFB000704700BF305902200CB41FB509B90DF11C
:10AFC0000300CDE9020107AB069A02A905480193E7
:10AFD000FFF708FC0022029B1A7005B05DF804EB35
:10AFE00002B0704733C4010024218379044A01FB75
:10AFF00003231B6AC01A034BC0105843704700BF9D
:10B00000905A0220ABAAAAAA10B524248379094A2F
:10B0100004FB0323DB690A685C6823689A4294BFD7
:10B020000A600B60FFF7E0FFD4E9002302FB003069
:10B0300010BD00BF905A022070B5164684680D46B8
:10B0400061B922491C23224A224810F0E2FF22481B
:10B0500010F0DFFF1C211E4810F0E8FF6B6863B999
:10B060001E491D231A4A1B4810F0D3FF1C4810F03C
:10B07000D0FF1D21164810F0D9FF23685BB10022D4
:10B080009D4213D12B685AB962682360954200D162
:10B09000636000232B6076B9002070BD0B46EFE79C
:10B0A000136063689D4208BF6260F2E719681A4640
:10B0B0000029F3D13EB123682B6060682560002829
:10B0C000EAD16560E9E76FF01500E6E7A80A02003B
:10B0D000580A0200E6FE0100B10A0200C00A02009E
:10B0E000D20A020010B5074C0749224607484FF420
:10B0F000E27310F08EFF2046BDE810404FF4E2717D
:10B1000010F094BFF50A02004E0B0200E6FE0100AB
:10B110001F2838B504460D4601D9FFF7E3FF08485C
:10B1200000EB8400D0F8003223F44033C0F8003242
:10B13000D0F8003243EA0543C0F8003238BD00BF02
:10B14000002584402DE9F041036801F01F049B684D
:10B150000D461B79484E44EA43140023D6F80423D5
:10B160008768D2B203F5A27156F82110C1F3042109
:10B170008C4266D122FA03F1C90762D59A0002F126
:10B18000804202F54432D2F8101521F00101C2F8D4
:10B190001015012202FA03F3C6F8083320460021F5
:10B1A000FFF7B6FFB868E84010F0010047D0F86834
:10B1B000E84010F0010042D07869E84010F0010842
:10B1C0004BD0BB69EB40DB073FD43B69FA69EB40EE
:10B1D00022FA05F503F0010305F00105AB420CBFAF
:10B1E00002250125002202F5A27356F8230010F073
:10B1F00003002CD1930003F1804303F54433D3F8CB
:10B200001015240221F4473121F44071C3F81015C0
:10B21000D3F8101504F4F85444EA05450D431749D2
:10B22000C3F8105541F82200D3F8101541F0010180
:10B23000C3F81015012303FA02F2C6F80423BDE88F
:10B24000F0810133082B8DD1A8E70325CAE701322D
:10B25000082AC8D16FF01200F1E73B69FA6920466D
:10B26000534023FA05F515F0010F0CBF032102210D
:10B27000FFF74EFF4046E2E7001003400011034095
:10B2800008B5094B1A786AB90121312019700521D6
:10B29000FEF7C4FE3120FEF79DFE4FF00042034B47
:10B2A000C3F80423002008BD7C1E022000100340C8
:10B2B0002DE9F74F0746846803F47040B0F5804FDE
:10B2C0001D464AD02DDCB0F5805F3ED0B0F5405F22
:10B2D0003FD068BB05F44076B6F5807F3FD0A6F539
:10B2E000007673427341012919BF5FFA82F9C8469B
:10B2F0004FF01F084FF000094FF0010A05F0010C54
:10B300004FEA4C0646EA0C0646EA002040EA83066D
:10B3100005F002030193C84523D2002003B0BDE825
:10B32000F08FB0F5E04F16D005DCB0F5A04F0ED091
:10B330006FF01500F2E7B0F5404F04D0B0F5504F74
:10B34000F6D10720C6E70620C4E70120C2E70320A4
:10B35000C0E70420BEE70520BCE70220BAE70323CC
:10B36000C1E73B689B68197909F01F0343EA411B59
:10B37000BBF11F0F01DDFFF7B5FE194A0BF180038A
:10B3800042F82360019A0AFA09F3A1682AB3194323
:10B39000A1606169A8064CBF194399436161A16925
:10B3A0006A064CBF19439943A161216968074CBFE4
:10B3B000194399432161E1692A064CBF0B4321EAF5
:10B3C0000303E36149463846FFF7BCFE0028A5D1D8
:10B3D00009F101025FFA82F99DE721EA0301D7E74B
:10B3E000002584402DE9F047524F3E68012E74D16C
:10B3F000B0464FF0000A504A93681268DC69D2F8F0
:10B400000890D3E902251540D3E905210A4325EA2E
:10B410000205D9F800201B6912695C40544025EAF6
:10B420000404002D46D13D60002301279E46434D74
:10B43000DFF814C1D5F8042307FA03F111420FD045
:10B4400003EB0C0292001168012909D103F5A270E7
:10B4500055F82000C2F800E0C0F3042081400C43FE
:10B460000133082BE6D1002C39D0334883681D689E
:10B47000ADB380462F68DFF8D490DFF8D4A0AB6876
:10B480001C4213D06B6863B951463D234A462C4891
:10B4900010F0BFFD2B4810F0BCFD3D21484610F0D8
:10B4A000C5FD6B682246294640469847BFB13D46D8
:10B4B0003F68E4E715EA080F0AD099F804300AF06B
:10B4C0001F00002140EA4310FFF722FE25EA08058D
:10B4D0000AF1010A4FEA4808A3E70024A4E7012E75
:10B4E0000ED10027144B9D681B68D3F80880D5E95E
:10B4F00002341C40D5E90532134324EA03040CB995
:10B50000BDE8F087264212D02B69EA6998F804C09A
:10B510005340FB4013F0010F07F01F000CBF032145
:10B52000022140EA4C10FFF7F3FD24EA060401373C
:10B530007600E4E77C110340F85902200010034034
:10B54000E6FE0100D20A020040C40010580A0200C0
:10B55000E90A020070B54B79012B23D18B79032BBB
:10B5600020D1CC792CB1012C1CD103689B681B79AC
:10B57000C3B10A7912B1022A14D10E2247F612265B
:10B5800003689B681D680B68B3426BD027D8B3F57E
:10B59000965F61D012D8B3F5167F4DD005D8B3F5BC
:10B5A000967F74D06FF0220052E0B3F5966F50D0C2
:10B5B000B3F5166FF6D14FF41D233FE0B3F5615F8D
:10B5C0004CD004D8B3F5165FECD1324B36E0B3F56E
:10B5D000964F45D0B3F5E14FE4D12F4B2EE0B3F5B4
:10B5E000E13F48D012D84DF6C026B3423DD005D831
:10B5F000B3F5164FD6D14FF41D031FE0B3F5614FDD
:10B6000036D0B3F5963FCDD1244B17E0B3F5E12FFB
:10B6100037D008D8B3F5613F30D0214EB342C1D105
:10B620004FF080630AE0B3F5612F2DD01D4EB34279
:10B63000B8D14FF0805301E04FF41C33C5F82435E6
:10B640008368224303C9C5F86C2583E80300002002
:10B6500070BD4FF49E23F1E7134BEFE7134BEDE77B
:10B66000134BEBE74FF40003E8E74FF46503E5E71E
:10B670004FF46B03E2E74FF0EB73DFE74FF06C73CF
:10B68000DCE74FF0E863D9E74FF07063D6E74FF49B
:10B69000A033D3E70050270000C0750000903A01A6
:10B6A00090D0030040420F0000B0130000F03A00B9
:10B6B00000A04E0070B50646002201210820FEF7CA
:10B6C000ADFC0820FEF786FC4FF000523368B568E9
:10B6D0009B6803211C681A4B1D209A600022C3F846
:10B6E0007412C3F87022C4F80C051C20C4F81405A9
:10B6F0004FF000609860C3F86C12C3F868221B23F7
:10B70000C4F808351A232946C4F810353046FFF727
:10B7100021FFA0B90823C4F8003505F10C03C4F8D3
:10B720001001C4F834350123AA68C4F8383592688A
:10B730002360C4F84425C4F84805A360E36070BDE5
:10B740000025844000220E4BF0B51C680D4B1646B8
:10B750001F46BD58B91885420DD075B14D680832E5
:10B76000651BB542C4BF2E460B46502AF1D119467F
:10B77000013C18605C600846F0BD0B46F7E700BF6F
:10B780004C00022058000220684620F007018D4638
:10B7900019B510F060FC0D4BD3E8EF2F0132C3E870
:10B7A000E12F0029F8D106F0D9FB094B1C6824B120
:10B7B000201D01F0BDFD2468F9E7FEF761FCFEF7EE
:10B7C0001DFABDE819408546704700BF4C000220B5
:10B7D000500002202DE9F0430D4689B011F080FCA5
:10B7E0002B680646002B0F4603D101F0B7FC3C2026
:10B7F0006CE0B8BF4FF0FF334FF00102B8BF2B60D1
:10B80000002102A801F05EFD0DF104084FF02003B5
:10B81000EFF3118983F31188BFF36F8F01F04CFDB3
:10B82000FFF790FF324C4368226893424FF00003C9
:10B8300008D101932F4B5A68002A4AD1C3E90088E6
:10B84000012300E0426089F31188BFF36F8F002B62
:10B850003BD0296802A801F0B3FD4FF02003EFF3BD
:10B86000118983F31188BFF36F8F0021214B1A6870
:10B870005AB1424538D1019800292FD15968186032
:10B88000914200D158600023019301F015FDFFF7AC
:10B8900059FF2368436089F31188BFF36F8F2C68C9
:10B8A000631C12D011F01CFC861B61EB0707E31729
:10B8B000A21B63EB07031946002A71F1000310462F
:10B8C000B8BF00202860002891D0002009B0BDE852
:10B8D000F083C2F80080C3F80480B1E708605868BC
:10B8E000904208BF5960CEE711461268C0E700BF1A
:10B8F0004C000220500002204FF08052014BC3F850
:10B900000021704700E100E04FF08052014BC3F886
:10B910008021704700E100E04FF00052014BC3F876
:10B920000021704700E100E04FF00052014BC3F8E6
:10B930008021704700E100E008B50023074AC2E912
:10B940000033074AD2E8EF1FC2E8E03F0028F9D1F0
:10B9500010F092FFBDE8084010F083BF50000220B5
:10B960004C00022008B50248FDF750FE002008BD3B
:10B970001CD50100B0F58D7F0DD040F20223984216
:10B980002AD001282AD1142924D0192922D0042907
:10B9900024D1042313E0013905291FD801A353F84A
:10B9A00021F000BFBDB90000C5B90000C9B9000051
:10B9B000CDB9000093B90000D1B900000223136093
:10B9C000002070470523FAE70623F8E70723F6E788
:10B9D0000123F4E71160F3E70129F9D04FF0FF30BC
:10B9E000704700BF154B70B51D68154C154B1E6890
:10B9F00023684BB9144915487E23154A10F009FBFA
:10BA00007E21134810F012FB2368DB6A4BB9114901
:10BA10000E487F230E4A10F0FCFA7F210C4810F0EC
:10BA200005FB23683246DC6A284600230A49A04702
:10BA3000BDE87040094B186811F090BA54590220C3
:10BA400008000220A8000220B60B0200E6FE01005A
:10BA5000630B0200C10B02009D1E02206C0102203C
:10BA60002DE9F0431F4DADF2044D4FF480620021EB
:10BA7000684610F034FC2E461B4F2B68D7F8008028
:10BA80004BB91A491A4869231A4A10F0C2FA6921B7
:10BA9000184810F0CBFA33685B6A4BB91649144862
:10BAA0006A23144A10F0B5FA6A21124810F0BEFA5F
:10BAB000336840465C6A4FF4806200236946A047C1
:10BAC000B0F10008D9DD0024DFF830904445D4D02F
:10BAD000D9F800001DF80410436801345B689847EA
:10BAE000F4E700BF0800022054590220B60B020000
:10BAF000E6FE0100630B0200E50B02006C01022070
:10BB0000012230B5314B87B031481A7000F01CF972
:10BB1000304D286018B96FF00D0007B030BD436894
:10BB20009B68002B46D12A685368002B46D12A4CCB
:10BB300023684BB929492A4819232A4A10F069FA7F
:10BB40001921284810F072FA23681B684BB926495E
:10BB500023481A23234A10F05CFA1A21214810F0D6
:10BB600065FA236840F201221B680021662098478D
:10BB70001E4B1F4A18601368013003F10103136064
:10BB8000C9D000241B4B1C4A1C60C3E901240A23B2
:10BB90004FF4C062CDE902431849194BCDE9044482
:10BBA000CDE90044174801F059FD286811F0D6F995
:10BBB0002046B2E798470028B5D0ACE79B6C002B35
:10BBC000B5D0114910469847B1E700BF9E1F02202B
:10BBD000380002006C01022008000220B60B0200AF
:10BBE000E6FE0100630B0200D20B02005459022052
:10BBF000BC000220AC000220E5B90000C8200220F1
:10BC000061BA0000C00002200DBC00004368F7B517
:10BC10005B6C054603B198476B685B6B6BB128465C
:10BC2000984750B1344C354E6B689B692BB101225B
:10BC30000DF107012846984708B903B0F0BD226806
:10BC40009DF80710531C2229236018D07F2901D0AA
:10BC5000082918D102B1013A022B38BF022300276C
:10BC60002748023B875423603378002BDCD1254BD7
:10BC70001B78032BD8D8DFE803F012123038307865
:10BC800080F001003070B3F5807F03D94FF48073EA
:10BC90002360C9E7002BFBD0194B9954E4E71A4AFB
:10BCA000D35C8B42C0D1194B18684368DB6A03B17F
:10BCB00098471749D1E8EF3F43F00102C1E8E02F70
:10BCC0000028F7D1DB0703D40839124811F07BF9BB
:10BCD000114B22681A600023DAE7094B1A4412F864
:10BCE000013C002BA0D00A29DCE7054B1A4412F8CE
:10BCF000013C0D2B98D1F6E7B80002209D1F0220D1
:10BD00009D1E02209E1F0220F60B02006C010220E5
:10BD1000B40002203C070220A800022070B50026D3
:10BD2000084B53F82040013053F82050A54200D86A
:10BD300070BD236820465B68984700B166600C348C
:10BD4000F4E700BF5CD50100104B70B505461E46F8
:10BD50000F4C9C4204D10E4CB44209D1002412E095
:10BD600062681AB122681268AA420CD00C34F0E75B
:10BD700063680BB90C34EFE723682846196810F0A4
:10BD80004EFA0028F6D1204670BD00BF285A022086
:10BD900080590220014B986854307047F806022001
:10BDA00008B50B4D4FF02002EFF3118382F3118899
:10BDB000BFF36F8F01F068FE012104460228D8BF4F
:10BDC000084601F0A7FE2C62FEF7C0F9EAE700BFC3
:10BDD000F80602200248034A0021121A10F07FBA26
:10BDE00000000220C420022008B50648064A074980
:10BDF000121A10F047FABDE80840054A05490648FE
:10BE000010F040BA28590220D85A0220D41102005A
:10BE100000000000D41102000000022008B502203A
:10BE2000FFF77CFF074810F0F4F80320FFF776FFD8
:10BE300001F070FCFDF770FA034A137B23F0010355
:10BE4000137308BDF90B02001C02022080B53B4BA6
:10BE5000B2B083F308880024E022394B012783F82D
:10BE60002220DC771C765C769C765A6A354E42F44A
:10BE7000E0225A62FEF7A6F8FEF762F907AB214608
:10BE8000AC22184610F02BFAB06020468DF82970CD
:10BE9000FFF744FF3846FFF741FF2B4D01F052F901
:10BEA0002A4B75624FF48052CDE90473CDE9024408
:10BEB000CDE90044264B2749284601F039FB6B7B2E
:10BEC000344623F0040213F01B0F6A7304D1AB69EC
:10BED00013B9284600F0CAFD1F4B012205930F231A
:10BEE000CDE9033200231D4E4FF4A0721C493046A9
:10BEF000CDE9013300931B4B01F01AFB737BE66025
:10BF000023F004037373184BC4E90633FEF72EFACB
:10BF10000D48A56010F0AFF80D4B144A184682F397
:10BF2000098863B64FF0000181F31188BFF36F8F6A
:10BF30000021002200230FF0DBFE00BF084002209A
:10BF400000ED00E0F80602201C0202203A0C02007C
:10BF50001DBE0000C82602203F0C02007001022016
:10BF6000C8360220A1BD000010070220C8360220FA
:10BF700070B500240A4B0B48834201D3002070BDEA
:10BF800000211A699D685C61A94201D11C33F3E765
:10BF90005E6901311660DE685A613244F4E700BF21
:10BFA000285A0220605A022038B5074C074DAC428F
:10BFB00001D3002038BD04F114032046C4E9053341
:10BFC0000FF084FD1C34F2E7605A02207C5A0220F4
:10BFD0002DE9F04F064685B00D4617461C46EFF397
:10BFE00005830D2B05D8002B5DD0384B5B681A05F7
:10BFF00059D4002C4AD10022354B9046F31A354AC9
:10C000009B1002FB03FA06F1140B5FFA8AFA009503
:10C0100003AB02AA394630460FF0A3FD10F10B0F17
:10C020000BD1009503AB02AA394630460FF099FDBB
:10C0300010F10B0F08BF6FF00B006B79029A85F8B7
:10C0400004A062F303036B716B68039A62F31F33FE
:10C050006B60C0B1BCB110F10C0F14D14FF02003D4
:10C06000EFF3118083F31188BFF36F8F2246594697
:10C0700000F056FF631CCAD001F048FEB8EB000484
:10C08000C5D56FF00A0005B0BDE8F08F124939231D
:10C09000124A13480FF0BDFF12480FF0BAFF3921C2
:10C0A0000E480FF0C3FF002CA5DD01F02FFE4FF46A
:10C0B000004C002180460C484FF4A0220023CCFB0A
:10C0C0000401FCF73FF818EB000295E700ED00E0F3
:10C0D000605A0220B76DDBB68B0C0200440C0200E4
:10C0E000E6FE01009EFF0100FFFF040070B504782A
:10C0F00002684178234DC4EBC404A400120B01F084
:10C100000F012819FDF70EF94FF02003EFF3118608
:10C1100083F31188BFF36F8F1B4801F023FA60B9D6
:10C120001A494E231A4A1B480FF073FF1A480FF0A2
:10C1300070FF4E2116480FF079FF134801F030FAD6
:10C1400004F11400284410F074FF28B13146BDE812
:10C1500070400D4800F096BA0B4801F011FA60B932
:10C160000E4961230A4A0B480FF053FF0C480FF0A9
:10C1700050FF612106480FF059FF86F31188BFF385
:10C180006F8F70BD605A0220F40602208301020006
:10C190003A010200E6FE010098010200AD01020032
:10C1A000C40102000146014810F0DFBE605A0220BF
:10C1B000034B01469B68186E08B110F0D6BE70475D
:10C1C000F80602202DE9F84304460E4690469946AB
:10C1D00000F108054FF02003EFF3118783F3118876
:10C1E000BFF36F8F284601F0BDF960B932494E2385
:10C1F000324A33480FF00DFF32480FF00AFF4E214C
:10C200002E480FF013FF284601F0CAF9B9F1000FCC
:10C210002CD00820FFF7CCFFC0B9284601F0B0F9B8
:10C2200060B929496123254A25480FF0F2FE2748C5
:10C230000FF0EFFE612121480FF0F8FE87F311881F
:10C24000BFF36F8F6FF00B00BDE8F8830123C0F8D8
:10C2500004800360036803F003035EB9226813439C
:10C2600003606368206073B960600CE0C8F80090F8
:10C270004046EFE7326832F0030215D1626803608E
:10C2800062B9C4E90000042104F10C0010F067FF5A
:10C290002846394600F0F6F90020D5E7136803F088
:10C2A000030303431360DFE713430360336803F0C2
:10C2B000030318433060E6E7830102003A010200FD
:10C2C000E6FE010098010200AD010200C401020077
:10C2D0002DE9F04F044689B00F4600F108054FF0F4
:10C2E0002003EFF3118883F31188BFF36F8F284683
:10C2F00001F038F960B967494E23674A67480FF083
:10C3000088FE67480FF085FE4E2163480FF08EFED1
:10C31000284601F045F9206820B30368626823F0DD
:10C320000303904208BF63602360012110F036FED2
:10C330000646284601F024F960B95A496123564A55
:10C3400056480FF066FE58480FF063FE61215248D0
:10C350000FF06CFE88F31188BFF36F8F304609B081
:10C36000BDE8F08F2846AFB901F00AF960B94D4930
:10C370006123494A49480FF04CFE4B480FF049FEF3
:10C38000612145480FF052FE88F31188BFF36F8F8B
:10C390000026E3E701F0F4F860B9424961233E4A20
:10C3A0003E480FF036FE40480FF033FE61213A4818
:10C3B0000FF03CFE88F31188BFF36F8F00222346F5
:10C3C000042103A801F0EAFD7A1C02D010F07CFEE3
:10C3D00083464FF00009DFF8C080DFF8C0A0069B5D
:10C3E000A7EB09026FF31033012103A8069301F0B4
:10C3F0002BFE08B10B30CBD14FF02003EFF31182AD
:10C4000083F31188BFF36F8F2846019201F0AAF8D9
:10C4100060B920494E23424650460FF0FAFD2048AD
:10C420000FF0F7FD4E2140460FF000FE284601F0C8
:10C43000B7F8206838B10368626823F003039042BC
:10C44000236008BF6360012110F0A8FD064628465E
:10C4500001F096F860B913496123424650460FF047
:10C46000D8FD11480FF0D5FD612140460FF0DEFDEB
:10C47000019B83F31188BFF36F8F002E7FF46EAFA3
:10C480007B1CACD010F020FEA0EB0B094F45A6DAC8
:10C490007EE700BF830102003A010200E6FE0100D0
:10C4A00098010200AD010200C4010200EFF3058013
:10C4B0000D2809D828B1054B586880F40060C0F3F6
:10C4C000C02080F0010070470120FAE700ED00E095
:10C4D00008B5FDF741FB054B054A1B6800211844D0
:10C4E00010611846BDE8084001F014BB3407022073
:10C4F000F8060220036810B504465BB906490748F0
:10C5000040F28313064A0FF084FD40F28311044881
:10C510000FF08CFD206810BD9A0D0200E6FE0100B0
:10C52000550D0200F8B507460D464FF02003EFF316
:10C53000118483F31188BFF36F8F1F4801F012F845
:10C5400060B91E494E231E4A1E480FF062FD1E4868
:10C550000FF05FFD4E211A480FF068FD164801F0FC
:10C560001FF84FF4004600220021184B18481A61AA
:10C57000C6FB07014FF4A0220023FBF7E3FD154B98
:10C580001860154B1D60FFF7A3FF0B4800F0F8FF84
:10C5900060B9124961230A4A0A480FF03AFD10486F
:10C5A0000FF037FD612106480FF040FD84F311883C
:10C5B000BFF36F8FF8BD00BF2C070220830102007C
:10C5C0003A010200E6FE010098010200F80602208E
:10C5D000FFFF04003407022030070220AD010200F3
:10C5E000C401020038B504464FF02003EFF3118573
:10C5F00083F31188BFF36F8F1B4800F0B3FF60B95E
:10C600001A494E231A4A1B480FF003FD1A480FF02F
:10C6100000FD4E2116480FF009FD134800F0C0FF41
:10C6200004F10800FFF766FF214600F0E3F8637BA2
:10C630000D4823F00203637300F0A2FF60B90F49B5
:10C6400061230B4A0B480FF0E4FC0D480FF0E1FCAE
:10C65000612107480FF0EAFC85F31188BFF36F8F63
:10C660000023A36038BD00BF2C0702208301020015
:10C670003A010200E6FE010098010200AD0102004D
:10C68000C401020010B502460C46FFF70FFFA8B127
:10C69000104600F075FF60B913497823134A144817
:10C6A0000FF0B7FC13480FF0B4FC78210F480FF0DF
:10C6B000BDFC2046BDE81040FDF7BABA104600F0B8
:10C6C0005FFF60B908496123084A09480FF0A1FCDF
:10C6D00008480FF09EFC612104480FF0A7FC84F38A
:10C6E0001188BFF36F8F10BDAD0102003A01020047
:10C6F000E6FE0100C401020038B54FF02003EFF35D
:10C70000118583F31188BFF36F8F2D4800F02AFF46
:10C7100060B92C494E232C4A2C480FF07AFC2C4847
:10C720000FF077FC4E2128480FF080FC244800F0E1
:10C7300037FFEFF305830D2B04D893B1254B5B68CE
:10C740001B050ED424494FF48073244A1F480FF070
:10C7500060FC23480FF05DFC4FF480711F480FF020
:10C7600065FC204CA268D27B012A0ED11E4940F202
:10C7700001131A4A15480FF04CFC19480FF049FCF8
:10C7800040F2011115480FF051FCA268D37B013B28
:10C79000D3730B4800F0F4FE60B9144961230A4AD0
:10C7A0000A480FF036FC12480FF033FC61210648AE
:10C7B0000FF03CFC85F31188BFF36F8F38BD00BFCD
:10C7C0002C070220830102003A010200E6FE01006C
:10C7D0009801020000ED00E0F80C0200AA0C020033
:10C7E0009EFF0100F8060220050D0200AD010200C7
:10C7F000C4010200124B10B503F1280282420C461C
:10C8000005D19B688B4202D14B7BDB0617D10D4BC8
:10C810001B689C420BD10C490C484FF423730C4A03
:10C820000FF0F7FB4FF4237109480FF0FFFBD4E939
:10C8300000231A60226853600023C4E9003310BD4E
:10C84000F806022074D50100D00D0200E6FE0100BA
:10C85000550D020038B504464FF02003EFF3118563
:10C8600083F31188BFF36F8F1D4800F07BFE60B922
:10C870001C494E231C4A1D480FF0CBFB1C480FF0EF
:10C88000C8FB4E2118480FF0D1FB154800F088FE78
:10C8900004F10800FFF72EFE2146FFF7ABFF637B94
:10C8A0000F4823F00203637300F06AFE60B9114978
:10C8B00061230D4A0D480FF0ACFB0F480FF0A9FBA8
:10C8C000612109480FF0B2FB85F31188BFF36F8F28
:10C8D000002304F11800A360BDE8384001F088B8D7
:10C8E0002C070220830102003A010200E6FE01004B
:10C8F00098010200AD010200C401020038B5154CD8
:10C90000024604F1280010F08EFB054600B9E568E8
:10C91000CAB9A36863B910497F23104A10480FF0C1
:10C9200078FB10480FF075FB7F210C480FF07EFB61
:10C93000A3685A7BD20606D1AA6922B9DA897F2A6E
:10C9400001D9636238BDA368AB4201D0FFF7C0FDD7
:10C950006562F7E7F8060220B10D0200550D0200EE
:10C96000E6FE01009EFF010038B5334CA268D27B81
:10C9700072B9324940F22123314A32480FF049FB63
:10C9800031480FF046FB40F221212D480FF04EFBBD
:10C99000EFF305830D2B04D893B12C4B5B681B057B
:10C9A0000ED42B4940F22223254A26480FF031FBB2
:10C9B00025480FF02EFB40F2222121480FF036FBD4
:10C9C0004FF02003EFF3118583F31188BFF36F8FCE
:10C9D000204800F0C7FD60B91F494E231F4A19487F
:10C9E0000FF017FB1E480FF014FB4E211B480FF0F1
:10C9F0001DFB184800F0D4FDA2680120D37B013351
:10CA0000D373FFF77BFF134800F0BAFD60B91549F7
:10CA10006123124A0B480FF0FCFA13480FF0F9FAA1
:10CA200061210E480FF002FB85F31188BFF36F8F71
:10CA3000BDE8384010F0EDBAF80602202D0D0200D6
:10CA4000550D0200E6FE01009EFF010000ED00E032
:10CA5000F80C02002C070220830102003A010200B8
:10CA600098010200AD010200C4010200F8B50446BD
:10CA70004FF02003EFF3118583F31188BFF36F8F1D
:10CA80002F4800F06FFD60B92E494E232E4A2F48E3
:10CA90000FF0BFFA2E480FF0BCFA4E212A480FF0D3
:10CAA000C5FA274800F07CFD2A4B1B689C420BD13D
:10CAB0002949264840F27623284A0FF0AAFA40F284
:10CAC000762126480FF0B2FA254A02F12801D2E970
:10CAD0000A308B420BD053B194F90E6093F90E706B
:10CAE000B7420ADC984202D01B68002BF6D1C4E999
:10CAF0000010D36A1C60D46205E05A68C4E90032B1
:10CB00005A6814605C60637B002043F040036373E9
:10CB1000FFF7F4FE0A4800F033FD60B911496123C4
:10CB2000094A0A480FF075FA0F480FF072FA6121AE
:10CB300005480FF07BFA85F31188BFF36F8FF8BDBE
:10CB40002C070220830102003A010200E6FE0100E8
:10CB50009801020074D50100D00D0200550D0200AD
:10CB6000F8060220AD010200C401020050F8103C9A
:10CB700070B50446A0F11805002B40D04FF02003FB
:10CB8000EFF3118683F31188BFF36F8F244800F011
:10CB9000E9FC60B923494E23234A24480FF039FAAF
:10CBA00023480FF036FA4E211F480FF03FFA1C4879
:10CBB00000F0F6FCA4F11000FFF79CFC2946FFF7FB
:10CBC00019FE14F80B3C164823F0020304F80B3C42
:10CBD00000F0D6FC60B917496123134A13480FF0DF
:10CBE00018FA15480FF015FA61210F480FF01EFAD8
:10CBF00086F31188BFF36F8F002344F8103C14F8BC
:10CC00000B3C284623F0140304F80B3C10F0E0F929
:10CC100020B12846BDE87040FFF728BF70BD00BFB7
:10CC20002C070220830102003A010200E6FE010007
:10CC300098010200AD010200C4010200F8B50446EB
:10CC40004FF02003EFF3118583F31188BFF36F8F4B
:10CC5000334800F087FC60B932494E23324A3348EA
:10CC60000FF0D7F932480FF0D4F94E212E480FF0CB
:10CC7000DDF92B4800F094FC21462E48FFF7BAFD61
:10CC80002D4B1B689C420BD12C49284840F276233F
:10CC90002B4A0FF0BEF940F2762129480FF0C6F971
:10CCA000284A02F12801D2E90A308B420BD053B155
:10CCB00094F90E6093F90E70B7420ADC834202D0F9
:10CCC0001B68002BF6D1C4E90010D36A1C60D46243
:10CCD00005E05968C4E9003159680C605C60637B09
:10CCE000906843F040036373031B58425841FFF7B9
:10CCF00005FE0B4800F044FC60B9134961230A4A61
:10CD00000A480FF086F911480FF083F961210648AF
:10CD10000FF08CF985F31188BFF36F8FF8BD00BF5A
:10CD20002C070220830102003A010200E6FE010006
:10CD3000980102002007022074D50100D00D0200E6
:10CD4000550D0200F8060220AD010200C4010200E8
:10CD50001449154A10B58B681468A34203D1BDE885
:10CD60001040FFF7B5BB00241460104A1268BAB136
:10CD7000DA897F2A14D80E4A93F90E401268944239
:10CD80000EDB0C4A126893420AD09A6942B90A69CA
:10CD9000824203DC1846FFF751FFE0E7121A0A61EE
:10CDA00010BD00BFF8060220280702203407022029
:10CDB0003007022074D5010038B504464FF0200337
:10CDC000EFF3118583F31188BFF36F8F1D4800F0D7
:10CDD000C9FB60B91C494E231C4A1D480FF019F9C4
:10CDE0001C480FF016F94E2118480FF01FF915488E
:10CDF00000F0D6FB637B5A0607D521461648FFF79D
:10CE0000F9FC637B23F040036373144B9868031BA6
:10CE100058425841FFF772FD0A4800F0B1FB60B973
:10CE20000F496123094A0A480FF0F3F80D480FF043
:10CE3000F0F8612105480FF0F9F885F31188BFF388
:10CE40006F8F38BD2C070220830102003A010200D7
:10CE5000E6FE01009801020020070220F8060220E9
:10CE6000AD010200C401020070B504460D4616462D
:10CE7000FFF7A2FF637B43F002036373002D2DD005
:10CE8000214BA5601B689C420BD12049204840F2F1
:10CE90007623204A0FF0BDF840F276211D480FF0AE
:10CEA000C5F82B689D420CD05BB194F90E2093F924
:10CEB0000E1091420CDC69688B4202D01B68002B7B
:10CEC000F5D16B68256063606B681C606C6005E081
:10CED0005A68C4E900325A6814605C60731C12D04E
:10CEE0004FF4004500210C484FF4A022C5FB060179
:10CEF0000023FBF727F90949421C04F11800BDE89B
:10CF0000704000F0CFBC70BD74D50100D00D0200A0
:10CF1000E6FE0100550D0200FFFF04006DCB00008E
:10CF2000F8B50646214D224CA868FFF79DFFAB6877
:10CF300030462360FCF77CFE06464FF02003EFF3FB
:10CF4000118783F31188BFF36F8F1A4800F00AFB33
:10CF500060B919494E23194A19480FF05AF819486F
:10CF60000FF057F84E2115480FF060F8114800F007
:10CF700017FB2368AA680F489A4204BF0023236066
:10CF800000F0FEFA60B9104961230C4A0C480FF01A
:10CF900040F80E480FF03DF8612108480FF046F8C0
:10CFA00087F31188BFF36F8F3046F8BDF806022073
:10CFB000280702202C070220830102003A01020008
:10CFC000E6FE010098010200AD010200C40102006A
:10CFD00038B505460C4611460E4A90680E4A106058
:10CFE0001A46FFF741FF284600F0CAFA60B90B491C
:10CFF00078230B4A0B480FF00CF80B480FF009F898
:10D00000782107480FF012F82046BDE83840FCF7B9
:10D010000FBE00BFF806022028070220AD01020063
:10D020003A010200E6FE0100C401020038B50446E0
:10D030004FF02003EFF3118583F31188BFF36F8F57
:10D04000394800F08FFA60B938494E23384A3948D8
:10D050000EF0DFFF38480EF0DCFF4E2134480EF0B2
:10D06000E5FF314800F09CFA20460FF0DCFF044653
:10D070002D4800F085FA60B9304961232C4A2D48CB
:10D080000EF0C7FF2E480EF0C4FF612128480EF0B5
:10D09000CDFF85F31188BFF36F8F002C41D04FF087
:10D0A0002003EFF3118583F31188BFF36F8F1E48C0
:10D0B00000F058FA60B91D494E231D4A1D480EF074
:10D0C000A8FF1D480EF0A5FF4E2119480EF0AEFF37
:10D0D000154800F065FA04F10800FFF70BFA214645
:10D0E000FFF788FB637B104823F00203637300F0B3
:10D0F00047FA60B9114961230D4A0E480EF089FFC5
:10D100000F480EF086FF612109480EF08FFF85F36E
:10D110001188BFF36F8F002304F11800A36000F0A3
:10D1200067FC204638BD00BF2C07022083010200A7
:10D130003A010200E6FE010098010200AD01020082
:10D14000C40102000021044B084603F12802C3E990
:10D150000A22FFF7E7B900BFF8060220F8B5EFF39F
:10D1600005830D2B04D893B1444B5B681B050ED48B
:10D17000434940F27E33434A43480EF04AFF434856
:10D180000EF047FF40F27E313E480EF04FFF404D1B
:10D19000404EA9683268914264D04FF02003EFF30B
:10D1A000118783F31188BFF36F8F3B4800F0DAF9E2
:10D1B00060B93A494E233A4A33480EF02AFF3948BB
:10D1C0000EF027FF4E2136480EF030FF324800F0B7
:10D1D000E7F9A9683448FFF70DFBAC6833689C4257
:10D1E0000BD13249284840F27623264A0EF011FF2F
:10D1F00040F2762123480EF019FFD5E90A312A4A78
:10D2000093420BD053B194F90E0093F90E6086420D
:10D210000ADC994202D01B68002BF6D1C4E9002138
:10D22000EB6A1C60EC6205E05A68C4E900325A6897
:10D2300014605C600120FFF761FB174800F0A0F963
:10D2400060B91B496123164A0F480EF0E2FE1948E7
:10D250000EF0DFFE612112480EF0E8FE87F3118820
:10D26000BFF36F8F4FF02003EFF3118083F311882A
:10D27000BFF36F8FBDE8F840FCF7DABC00ED00E0CB
:10D28000F80C0200550D0200E6FE01009EFF0100B1
:10D29000F806022074D501002C0702208301020049
:10D2A0003A0102009801020020070220D00D02007E
:10D2B000AD010200C4010200014B9868704700BF35
:10D2C000F806022070B504460E46154662B91249AA
:10D2D0004623124A12480EF09CFE12480EF099FEA8
:10D2E00046210E480EF0A2FEB5420CD20E4947234D
:10D2F0000A4A0B480EF08DFE0C480EF08AFE4721BC
:10D3000006480EF093FE04F11003C4E90265C4E977
:10D310000044C4E9043370BD240E0200E10D020094
:10D32000E6FE0100300E0200470E02005E0E020013
:10D3300070B504464FF02003EFF3118683F3118894
:10D34000BFF36F8F194800F00DF960B918494E23EB
:10D35000184A19480EF05DFE18480EF05AFE4E218C
:10D3600014480EF063FE114800F01AF92046FFF74A
:10D370005DFE054670B1437BDB0603D183690BB9C3
:10D38000FFF774FB0023AB663146BDE870400748E9
:10D39000FFF778B9D4E902329A4218BF013302216B
:10D3A000A36004F110000FF0DAFEEDE73807022069
:10D3B000830102003A010200E6FE0100980102002A
:10D3C00070B505460E46EFF305830D2B04D88BB1DF
:10D3D000344B5B681B050DD466B133498C23334A4B
:10D3E00033480EF016FE33480EF013FE8C212F4802
:10D3F0000EF01CFE4FF02003EFF3118483F311882D
:10D40000BFF36F8F2C4800F0ADF860B92B494E2365
:10D410002B4A27480EF0FDFD2A480EF0FAFD4E215A
:10D4200027480EF003FE244800F0BAF8AB68C3B1F9
:10D43000013BAB60204800F0A3F860B922496123AA
:10D440001F4A1B480EF0E5FD20480EF0E2FD612169
:10D450001B480EF0EBFD84F31188BFF36F8F0020A3
:10D4600070BDBEB9144800F08BF860B9164961234D
:10D47000134A0F480EF0CDFD14480EF0CAFD61218D
:10D480000F480EF0D3FD84F31188BFF36F8F6FF058
:10D490000F00E5E733462A462146BDE870400648BE
:10D4A000FFF796BD00ED00E0830E0200E10D0200E3
:10D4B000E6FE01009EFF0100380702208301020002
:10D4C0003A01020098010200AD010200C40102000D
:10D4D00010B5084C4FF0FF334FF4806220460649E8
:10D4E00000F074F904F1140004490FF0C1FD0020AC
:10D4F00010BD00BF3C07022008400220AA0E020017
:10D50000EFF305800D2807D838B1044B586880F434
:10D510000060C0F3C02070470120704700ED00E0BC
:10D52000024B9B68187B00F001007047F806022050
:10D5300030B587B00E9D044604950D9D03950C9D56
:10D5400002950B9D01950A9D0095FCF7A7FD044BE4
:10D550009B6813B9236607B030BD1B6EFAE700BFA6
:10D56000F8060220006838B1044B00F003001B7D70
:10D57000C01A18BF0120704701207047F80602202A
:10D58000064A117D936802680B439A424FF00003EC
:10D5900006BF036001201846704700BFF80602204E
:10D5A000024A117D93680B4303607047F80602201E
:10D5B00038B504464FF02003EFF3118583F311884B
:10D5C000BFF36F8F1E48FFF7CDFF60B91D494E2393
:10D5D0001D4A1E480EF01DFD1D480EF01AFD4E217D
:10D5E00019480EF023FD1648FFF7DAFF637B5A0750
:10D5F00015D41348FFF7C4FF60B916496123124AD6
:10D6000012480EF006FD14480EF003FD61210E488D
:10D610000EF00CFD85F31188BFF36F8F38BD23F03A
:10D620000403637320460FF01AFD10B12046FFF784
:10D630001DFA2946BDE838400148FFF723B800BF6E
:10D64000FC070220830102003A010200E6FE01000D
:10D6500098010200AD010200C40102002DE9F04171
:10D6600086B004460E4617469846119DEFF3058393
:10D670000D2B04D893B1204B5B681A050ED41F49BB
:10D680004FF4D9731E4A1F480EF0C3FC1E480EF01B
:10D69000C0FC4FF4D9711A480EF0C8FC0023059362
:10D6A000109B3A4604930F9B314603930E9B2046F2
:10D6B00002930D9B01930C9B00934346FFF738FFA9
:10D6C0006B1C03D035B92046FFF772FF204606B029
:10D6D000BDE8F0814FF4004600210C484FF4A02231
:10D6E0000023C6FB0501FAF72DFD0949421C04F190
:10D6F000180000F0D7F8E9E700ED00E0F80C0200B0
:10D70000B30E0200E6FE0100F90E0200FFFF040066
:10D710006DCB00002DE9F04F284E294DB04687B063
:10D72000B54205F130040FD3FEF7E6FF4FF4004990
:10D730000027234C234EDFF890A0444521D307B0A7
:10D74000BDE8F04FFFF710B954F8043C059354F8C6
:10D75000103C049354F8143C039354F8183C02937F
:10D7600054F81C3C019354F8203C009354E90A23DC
:10D7700054E90C01FFF7DCFE54F8303CDD6425462B
:10D78000CEE7616A4B1C04D0256821B92846FFF713
:10D790000FFF3034D1E7B346BC46C9FB01BC4FF4A0
:10D7A000A022002358466146FAF7CCFC5146421CA1
:10D7B00005F1180000F076F8EBE700BF285A0220C8
:10D7C000285A0220FFFF04006DCB00002DE9F04134
:10D7D000054686B098460E4617460FF0EBFB002034
:10D7E00005F11404CDE90400CDE90208CDE90050AB
:10D7F0003146064B3A462046FFF730FF20460449A3
:10D8000006B0BDE8F0410FF033BC00BF05BD01001C
:10D810001E0F0200034B1B680BB9FCF79DB90020DB
:10D82000704700BF0008022038B5104B1B78002B52
:10D830000F4B18BF4FF0FF301C6808BF6FF000405F
:10D840009C420AD04CB1A568FFF7E4FF281A0028D3
:10D850000ADBA468FFF7DEFF201A064B1B6913B131
:10D860009842A8BF184638BD0020F6E79F1F022047
:10D8700058590220F8060220036840B1084A52684D
:10D88000904204D01BB19A6881680A449A60426849
:10D89000136003685A600023C0E90033704700BF7B
:10D8A0005859022003682DE9F04704460E461546F4
:10D8B00063B143494D23434A43480EF0AAFB434812
:10D8C0000EF0A7FB4D213F480EF0B0FB012DB8BF75
:10D8D0000125E6604FF02003EFF3118883F31188F0
:10D8E000BFF36F8F3A48FFF73DFE60B939494E23C9
:10D8F000394A35480EF08DFB38480EF08AFB4E2130
:10D9000035480EF093FB3248FFF74AFEFFF782FFDF
:10D91000334E28443568A060B54205D0294FDFF862
:10D92000CC90DFF8A4A035B9736826606360736893
:10D930001C6074601BE0AB68002B0CDA4946562370
:10D940003A4650460EF065FB20480EF062FB562129
:10D9500038460EF06BFBAA68A3689A4228DDD31AFA
:10D96000AB606B68C4E900536B681C606C60336823
:10D97000B34206D09C4204D1FFF756FF0021FCF7CA
:10D980007DF81348FFF7FCFD60B916496123124A80
:10D990000D480EF03EFB14480EF03BFB61210E4893
:10D9A0000EF044FB88F31188BFF36F8FBDE8F0875A
:10D9B0009B1AA3607368AB42B6D02D68B3E700BF73
:10D9C0006F0F0200280F0200E6FE01009EFF01001B
:10D9D00004080220830102003A01020098010200BB
:10D9E00058590220AD010200C40102008F0F02004D
:10D9F00038B504464FF02003EFF3118583F3118807
:10DA0000BFF36F8F1948FFF7ADFD60B918494E237A
:10DA1000184A19480EF0FDFA18480EF0FAFA4E218D
:10DA200014480EF003FB1148FFF7BAFD2368D3B189
:10DA30002046FFF721FF00240C48FFF7A1FD60B945
:10DA40000F4961230B4A0C480EF0E3FA0D480EF023
:10DA5000E0FA612107480EF0E9FA85F31188BFF377
:10DA60006F8F204638BD6FF01504E5E704080220EB
:10DA7000830102003A010200E6FE01009801020063
:10DA8000AD010200C401020038B54FF02003EFF3EE
:10DA9000118583F31188BFF36F8F1748FFF762FD7D
:10DAA00060B916494E23164A16480EF0B2FA1648C7
:10DAB0000EF0AFFA4E2112480EF0B8FA0E48FFF7FA
:10DAC0006FFDFFF7B1FE04460B48FFF759FD60B943
:10DAD0000E4961230A4A0B480EF09BFA0C480EF0DF
:10DAE00098FA612106480EF0A1FA85F31188BFF378
:10DAF0006F8F204638BD00BF04080220830102005A
:10DB00003A010200E6FE010098010200AD010200A8
:10DB1000C401020070B504460E464FF02003EFF337
:10DB2000118583F31188BFF36F8F1A48FFF71AFD31
:10DB300060B919494E23194A19480EF06AFA194872
:10DB40000EF067FA4E2115480EF070FA1148FFF7F3
:10DB500027FDFFF769FEA04205DD012803DD314600
:10DB60002046FBF78BFF0B48FFF70AFD60B90E4913
:10DB700061230A4A0A480EF04CFA0C480EF049FAA2
:10DB8000612106480EF052FA85F31188BFF36F8FBA
:10DB900070BD00BF04080220830102003A010200A8
:10DBA000E6FE010098010200AD010200C40102007E
:10DBB0002DE9F04B0446FFF7CBF84FF02003EFF3CD
:10DBC000118583F31188BFF36F8F4648FFF7CAFCB6
:10DBD00060B945494E23454A45480EF01AFA454872
:10DBE0000EF017FA4E2141480EF020FA424F434EF4
:10DBF000B9463C48DFF81081FFF7D2FC3460D8F812
:10DC0000004032684445D7E900BC05D024B1A36880
:10DC1000934225DD9B1AA36000241BEB02004CEB12
:10DC2000E271C9E900013460FFF7FEFD2146FBF710
:10DC300025FF2C48FFF7A4FC60B9314961232B4A2A
:10DC40002B480EF0E6F92F480EF0E3F96121274842
:10DC50000EF0ECF985F31188BFF36F8FBDE8F08B00
:10DC60001BEB03004CEBE371D31A33600023C7E9CD
:10DC70000001A3602046FFF7FFFD1A48FFF780FC74
:10DC800060B91F496123194A19480EF0C2F91D48AD
:10DC90000EF0BFF9612115480EF0C8F985F311881F
:10DCA000BFF36F8FE368204698474FF02003EFF3F0
:10DCB000118583F31188BFF36F8F0A48FFF752FC79
:10DCC00060B909494E23094A09480EF0A2F90948EA
:10DCD0000EF09FF94E2105480EF0A8F90148FFF714
:10DCE0005FFC8CE704080220830102003A01020075
:10DCF000E6FE010098010200000002200008022058
:10DD0000AD010200C4010200585902202DE9F04182
:10DD10004FF02003EFF3118683F31188BFF36F8F69
:10DD20001A48FFF71FFC60B919494E23194A1A48CF
:10DD30000EF06FF919480EF06CF94E2115480EF0EF
:10DD400075F91248FFF72CFCFBF706FF144BD3E9DB
:10DD5000004527180D4845F10008FFF711FC60B990
:10DD6000104961230B4A0C480EF053F90E480EF08F
:10DD700050F9612107480EF059F986F31188BFF375
:10DD80006F8F38464146BDE8F08100BF040802208D
:10DD9000830102003A010200E6FE01009801020040
:10DDA00000000220AD010200C40102002DE9F84389
:10DDB00014240F46904604FB0104454DDFF84C91B6
:10DDC000444E002F01DABDE8F8830023A360637B93
:10DDD00003F00F03042B39D8DFE803F0452A03389A
:10DDE0001C00236963B93C4996232A4630460EF04D
:10DDF00010F93A480EF00DF9962128460EF016F962
:10DE0000226882B363681A60226853600023C4E901
:10DE1000003328E02369002BF2D131499A232A46A6
:10DE200030460EF0F6F82F480EF0F3F89A21E4E7AA
:10DE30002369002BE4D12C499E232A4630460EF05C
:10DE4000E8F82A480EF0E5F89E21D6E74946A523D2
:10DE50002A4630460EF0DDF825480EF0DAF8A52106
:10DE600028460EF0E3F82348FFF78AFB60B9224901
:10DE70006123224A30460EF0CCF821480EF0C9F852
:10DE800061211E480EF0D2F888F31188BFF36F8F1E
:10DE90004FF02003EFF3118883F31188BFF36F8FE6
:10DEA0001448FFF75FFB60B916494E23134A30460A
:10DEB0000EF0AFF814480EF0ACF84E210F480EF0FB
:10DEC000B5F80C48FFF76CFB013F143C79E700BF45
:10DED0009E0F0200E6FE0100E20F0200FC0F0200AE
:10DEE000111002002D1002003E1002005B10020013
:10DEF0007210020008080220AD0102003A0102007F
:10DF0000C40102008301020098010200530D0200C7
:10DF1000836870B505460E4653B31C6874B91B4937
:10DF200040F25B131A4A1B480EF073F81A480EF0C1
:10DF300070F840F25B1116480EF078F80022AB68DA
:10DF40001A71637B9A0713D5236A02331AD02046CD
:10DF5000FEF780FC082E0CBF6FF003030023A366BE
:10DF6000637BDB0604D1A36913B92046FEF77EFD6F
:10DF70000020EB68A860C3F30432164366F3103345
:10DF8000EB6070BD6FF00A00FBE700BF2F110200CD
:10DF90009E0F0200E6FE010054110200F8B504468F
:10DFA0000F461D46164662B11F492A231F4A2048C4
:10DFB0000EF02FF81F480EF02CF82A211B480EF007
:10DFC00035F80F2F0CD91C492B23184A18480EF08E
:10DFD00020F81A480EF01DF82B2114480EF026F8F0
:10DFE00065B917492C23114A11480EF012F815484B
:10DFF0000EF00FF82C210D480EF018F80022637B6C
:10E00000A26067F303036373E368256162F310336F
:10E01000E360C3F3074366F34103A373E38962F349
:10E020008F03E381F8BD00BF881002009E0F02003D
:10E03000E6FE0100A8100200CE100200F21002005D
:10E0400002110200151102002DE9F04F054687B0BC
:10E050008B469046EFF305830D2B04D883B1A64B76
:10E060005B681B050CD4A549C123A54AA5480DF042
:10E07000D0FFA5480DF0CDFFC121A1480DF0D6FF7E
:10E0800065B9A249C2239E4A9E480DF0C2FFA0482E
:10E090000DF0BFFFC2219A480DF0C8FFBBF1000F81
:10E0A0000CDC9C49C323964A96480DF0B2FF9A486F
:10E0B0000DF0AFFFC32192480DF0B8FF974B2C46EF
:10E0C0009B684FF00009029301234FF0FF36DFF801
:10E0D00054A2934F8DF80C30D9453FDB4FF020030D
:10E0E000EFF3118483F31188BFF36F8F8D48FFF72F
:10E0F00039FA60B98C494E23894A82480DF089FF6C
:10E100008A480DF086FF4E2185480DF08FFF854827
:10E11000FFF746FA9DF80C30002B40F01F8128468F
:10E1200022463146FFF742FE7E48FFF729FA60B9E2
:10E130007F4961237A4A73480DF06BFF7D480DF0EB
:10E1400068FF612176480DF071FF84F31188BFF3F9
:10E150006F8F0024204607B0BDE8F08F4FF02003FA
:10E16000EFF3118283F31188BFF36F8F5046019252
:10E17000FFF7F8F960B96C494E233A4661480DF053
:10E1800048FF6A480DF045FF4E2138460DF04EFF1E
:10E190005046FFF705FA637B03F00F03042B26D8E4
:10E1A000DFE803F0071F0325190023699B68002B94
:10E1B0002ED1B8F1000F37D09DF80C30002B33D0A2
:10E1C000637B03F00F03042B00F28880DFE803F089
:10E1D0005B7346865F0023691B68002BE9D004222D
:10E1E00017E023699B68002BE3D0012211E0502344
:10E1F000434A514943480DF00CFF617B4F4801F001
:10E200000F010DF006FF50213D480DF00FFFD0E744
:10E2100002220021E368A160C3F30430024362F3E9
:10E220001033E3608DF80C105046FFF7A9F960B980
:10E230003F4961233A4633480DF0EBFE3D480DF06F
:10E24000E8FE612138460DF0F1FE019B83F3118851
:10E25000BFF36F8F09F1010914343DE7236963B9F6
:10E2600037497523264A27480DF0D3FE35480DF06F
:10E27000D0FE752122480DF0D9FE2146206902AA60
:10E2800010300EF03DFF02ABA3600136CCE72369EE
:10E2900063B92D4979231A4A1A480DF0BAFE2B4862
:10E2A0000DF0B7FE792116480DF0C0FE206902AAD4
:10E2B00021460C30E5E7236963B925497D23104ADF
:10E2C00010480DF0A6FE23480DF0A3FE7D210C485A
:10E2D0000DF0ACFE02AA21462069D2E78423084A49
:10E2E000154908480DF095FE1B480DF092FE84215B
:10E2F00003480DF09BFEC6E700ED00E0F80C0200BD
:10E300009E0F0200E6FE01009EFF01007311020055
:10E310008911020098110200A7110200F8060220DC
:10E320003A0102000808022083010200980102005D
:10E33000AD010200C4010200530D0200B61102003B
:10E34000E20F0200FC0F0200111002002D1002006B
:10E350003E1002005B1002007210020000238DF8D4
:10E360000C30B8F1000F17D12B48FFF709F960B94D
:10E370002A4961232A4A2B480DF04BFE2A480DF00A
:10E3800048FE612126480DF051FE84F31188BFF349
:10E390006F8F6FF00A04DDE604AA214643461E484B
:10E3A000CDE90422FEF714FE04464FF02003EFF3FC
:10E3B000118783F31188BFF36F8F1748FFF7D2F8E7
:10E3C00060B91A494E23164A16480DF022FE184825
:10E3D0000DF01FFE4E2112480DF028FE0E48FFF7EB
:10E3E000DFF828463A463146FFF7E0FC0A48FFF7D7
:10E3F000C7F860B909496123094A0A480DF009FEC6
:10E4000009480DF006FE612105480DF00FFE87F367
:10E410001188BFF36F8F9DE608080220AD0102004E
:10E420003A010200E6FE0100C4010200830102007D
:10E430009801020008B5074B1A6842F000421A60C2
:10E440001B68DB0702D4FAF747FF08BDFAF74AFF5B
:10E4500008BD00BF0C08022010B5084C23684BB95A
:10E460000123236000F01AF82368002B01DB02234C
:10E47000236010BD0F20FAF72FFF10BD0C080220FB
:10E480000FB408B52D200EF06EF9BDE808404FF02E
:10E49000FF3004B0704700BFFFF7CCBFF0B593B0BA
:10E4A00004F0E0FC20B92A4901A804F04FFD18B19E
:10E4B000FFF7C0FF13B0F0BDFDF73EFA03F0B4FD67
:10E4C00002460028F4D120234FF4804008214FF465
:10E4D000405C204FCDE910221F4E03930593079314
:10E4E0001E4D1F4C1F4A204B09900D900DEB010053
:10E4F000CDF82CC0CDE90E1102970496069508942C
:10E500000A920C9300F080FB0028D1D103F0A0FB0D
:10E510000028CDD105F0A8F90028C9D102F0BEF934
:10E520000028C5D105F0B4FB0028C1D105F08AFF51
:10E530000028BDD102F0D2F80028B9D100F0A4F82B
:10E540000028B5D101F04EF90028B3D0B0E700BFE4
:10E5500058D60100000001204000012020000120C9
:10E56000607001206000012060300120022808B5A1
:10E570000ED01DD90A280BD0662821D140F20123E4
:10E580009A4224D040F202239A4219D1114808BD80
:10E59000A2F582720A2A18D8012340F203410E48DC
:10E5A00003FA02F20A4200F1280318BF184608BD18
:10E5B000012805D140F203239A4201D1074808BD42
:10E5C00016200EF0D0F8002008BD034808BD04480E
:10E5D00008BD00BF18D60100A0D50100F0D501008C
:10E5E00078D5010038B5054603F044FC044678B9F7
:10E5F0001F4BAB430AD01F4BAB4333D11E4838BD32
:10E60000012B16D140F203239A4212D11B4838BD88
:10E6100083680269022B11D0F2D90A2B0ED0662B27
:10E6200007D140F201239A421AD040F202239A42C3
:10E63000E4D016200EF097F8002038BDA2F58272C3
:10E640000A2A0BD8012340F203410D4803FA02F2D3
:10E650000A4200F1280418BF204638BD084838BDDA
:10E66000084838BD09200EF07EF8204638BD00BFAE
:10E670003254764900009A7818D60100F0D501008E
:10E68000A0D5010078D5010070B586B01D4902A85B
:10E6900004F05CFC00BB0146044640F20122662007
:10E6A00005F0E4F8184E00280546306010DB1748E6
:10E6B0000DF0ADFD2346024614492846019400940E
:10E6C00005F084F8054611480DF0A1FDA84207D0D9
:10E6D0000524204606B070BD6924204606B070BDF2
:10E6E0003068CDE9004403A923460A2205F050F919
:10E6F0000128EDDD03A8022205490DF09DFD00284B
:10E70000E7D0E5E7645902206059022070D6010085
:10E710007CD60100014B1860704700BF1C18022016
:10E72000F0B56C4B83B01B78002B00F0AD806A4BCA
:10E730001C68A26863689A422DD04BF6EF63ADF86F
:10E74000003023786E468DF80430636805219A42C4
:10E750002ABF27699F1ABF1A9A4294BF0025E5680D
:10E76000BFB288BF5B1B304688BF9DB2ADF8027058
:10E770000EF08DF8BDF80210A0680EF088F8A368BE
:10E7800022691F44974208BFE368A76008BFA360DF
:10E79000002D40F08D80514B1C68A26863689A423E
:10E7A0002CD04BF6EF63ADF8003023786E468DF831
:10E7B0000430636805219A422ABF27699F1ABF1A4D
:10E7C0009A4294BF0025E568BFB288BF5B1B304604
:10E7D00088BF9DB2ADF802700EF059F8BDF8021076
:10E7E000A0680EF054F8A36822691F44974208BF3E
:10E7F000E368A76008BFA360002D48D1384B1C68B0
:10E80000A26863689A422BD04BF6EF63ADF80030F4
:10E8100023786E468DF80430636805219A422ABF3A
:10E8200027699F1ABF1A9A4294BF0025E568BFB2B4
:10E8300088BF5B1B304688BF9DB2ADF802700EF0FA
:10E8400026F8BDF80210A0680EF021F8A36822692E
:10E850001F44974208BFE368A76008BFA3600DB9D3
:10E8600003B0F0BD30460521ADF802500EF00FF8B0
:10E87000BDF80210E0680EF00AF8BDF80220E36867
:10E880001344A36003B0F0BDFDF74EF84FE7052138
:10E890003046ADF802500DF0FAFFBDF80210E06806
:10E8A0000DF0F5FFBDF80220E3681344A360A5E76F
:10E8B00005213046ADF802500DF0E9FFBDF8021019
:10E8C000E0680DF0E4FFBDF80220E3681344A360A4
:10E8D00061E700BFA01F02201818022010180220B4
:10E8E0001418022000222DE9F04FB04B83B01B68B2
:10E8F00019695C69187C1A74587C5A74987C9A74EB
:10E90000D87CDA74187D1A75587D5A75987D9A7579
:10E91000D87DDA75B9B10139032914D8DFE811F0CF
:10E92000D6000301040016000125032000226FF029
:10E930005F019F4C25701C7A1872587A5A72987A27
:10E940009A72DA7AD97203B0BDE8F08F04210022FE
:10E950006FF05F001C7A1972597A5A7294499C7A46
:10E960009A72DC7AD8720A700B78002B00F017814B
:10E97000904B1C68A26863689A422DD04BF6EF63F7
:10E98000ADF8003023786E468DF8043063680521B9
:10E990009A422ABF27699F1ABF1A9A4294BF00253C
:10E9A000E568BFB288BF5B1B304688BF9DB2ADF83B
:10E9B00002700DF06CFFBDF80210A0680DF067FF4B
:10E9C000A36822691F44974208BFE368A76008BF95
:10E9D000A360002D40F0D280774B1C68A26863686A
:10E9E0009A422DD04BF6EF63ADF8003023786E4697
:10E9F0008DF80430636805219A422ABF27699F1A5F
:10EA0000BF1A9A4294BF0025E568BFB288BF5B1B5E
:10EA1000304688BF9DB2ADF802700DF038FFBDF8EA
:10EA20000210A0680DF033FFA36822691F449742CB
:10EA300008BFE368A76008BFA360002D40F08D8089
:10EA40005E4B1C68A26863689A423FF47CAF4BF649
:10EA5000EF63ADF8003023786E468DF804306368BC
:10EA600005219A422ABF27699F1ABF1A9A4294BF6A
:10EA70000025E568BFB288BF5B1B304688BF9DB2EA
:10EA8000ADF802700DF003FFBDF80210A0680DF0A4
:10EA9000FEFEA36822691F44974208BFE368A7608F
:10EAA00008BFA360002D3FF44EAF05213046ADF8FE
:10EAB00002500DF0ECFEBDF80210E0680DF0E7FE2C
:10EAC000BDF80220E3681344A3603CE7384A11789C
:10EAD00009B100211170A568002D39D04FF0000C4C
:10EAE000DFF8D4A0DFF8CCB03449E1466646624690
:10EAF000D1F800E0DAF80080DBF8007008E0632964
:10EB000016D0612904BF074601260132AA4213D05C
:10EB1000911C04EB8101486801786229EFD180469D
:10EB20004FF00109F1E7FCF7F7FE03B0BDE8F08F05
:10EB300086464FF0010CE8E7A6BBB9F1000F01D003
:10EB4000CAF80080BCF1000F02D01C4AC2F800E0F5
:10EB5000012000226FF05F01EDE605213046ADF89F
:10EB600002500DF094FEBDF80210E0680DF08FFE2B
:10EB7000BDF80220E3681344A36061E70521304635
:10EB8000ADF802500DF083FEBDF80210E0680DF004
:10EB90007EFEBDF80220E3681344A3601CE7FCF787
:10EBA000C3FEE5E6CBF80070C7E700BF1C180220E3
:10EBB000A01F02201818022010180220141802208A
:10EBC000014B1878704700BFA01F0220002070473B
:10EBD0000B4BD3E90023134498420DD282420BD849
:10EBE00010B5044600F0E0FC40B1064A84600260C3
:10EBF000BDE8104000F020BC04F0F6BA10BD00BF24
:10EC0000201802200100020000282BD030B589B066
:10EC100001AA6946044600F025FB034640B1134AA9
:10EC200004F1280003C882E80300184609B030BD8B
:10EC3000DDE90012204600F04BF803460028EED133
:10EC40000B4B0C490C480D4A03930D4D0D4B049191
:10EC500005900D4902A807930695029203F06EFBFA
:10EC60000346DCE70E231846704700BF2018022039
:10EC700039F5000009F60000F9F1000039F4000050
:10EC8000D1EB0000CDEB00002818022060B108B5E0
:10EC90004368DBB2022B0ED003681B0C022B05D09D
:10ECA000042B0ED0002008BD00207047806804F0BF
:10ECB0009BFA002008BD0146BDE80840034803F068
:10ECC00027BA024803F09AFB002008BD281802204A
:10ECD000002800F0FF802DE9F04F056895B0002D69
:10ECE00000F0EE808368002B00F0EA800769002FB7
:10ECF00000F0E680846A002C00F0E28044681B2C5F
:10ED000040F2E380C4680B2C40F2DF80D0F814E0BE
:10ED1000BEF1170F40F2D980002604466F48CDE9B6
:10ED20000012DFF8D8A16E490680A06BDFF8D0C1D1
:10ED3000DFF8D081DFF8D0B1DFF8D09172460E60F5
:10ED4000CAF8000031463846CCF80060CBF80030F5
:10ED5000C8F80060C9F800600DF0C1FAE3693846F0
:10ED60003B60A3697B60FFF7D5FC01224FF0040CE8
:10ED70005C4B5D49C3F810560968802004915B49DB
:10ED8000DDF810E0C3F8146609682E7003916E7008
:10ED9000EE70AA700399A16ADBF800E06960E16A8D
:10EDA000019CA960EC60009C5149AF61C5F814E07A
:10EDB0002C61C3F890250C68A1F592610594059C1F
:10EDC000C3F898C5D1F898444FF480670694069C20
:10EDD0001024C3F8A045D1F8A044464D0794079CE1
:10EDE0004024C3F8A845D1F8A8440894089CC3F867
:10EDF000AC05D1F8AC0409900998C3F80061086823
:10EE00000A900A98C3F8086188680B900B98C3F8B9
:10EE1000106108690C900C98C3F8186188690D900E
:10EE20000D98C3F81C61C86901F501710E900E9828
:10EE3000D3F804031043C3F804030C682E480F945E
:10EE40000F9CD3F8044344EA0C04C3F804430C6851
:10EE50001094109CD3F8044344F01004C3F8044306
:10EE60000C681194119CD3F8044344F04004C3F897
:10EE700004430C681294129CD3F8044344F08004B9
:10EE8000C3F80443DAF8003009685B011391DBB280
:10EE90001399C8F8002080F82A33C0F884714760BD
:10EEA0000296C5F81066D5F810360293029BD8F882
:10EEB0000030012BFBD0D9F8000015B0BDE8F08F71
:10EEC0004CF20E0015B0BDE8F08F4CF2090015B001
:10EED000BDE8F08F4CF20E00704700BF701E02209C
:10EEE0003818022000A0024010A6024014A60240DA
:10EEF00090A502400050004000E100E030180220E0
:10EF00003C18022034180220401802202C1802203D
:10EF10002DE9F0474FF48065A94C86B0C4F88450C1
:10EF2000BFF34F8FBFF36F8FA64EC4F88451D6F84E
:10EF30000C331F0669D4A34BD3F80C23D00775D428
:10EF4000D3F80C2312F0400259D1D3F80C1349071F
:10EF500041D59D4F3968012900F0C9809B4BDFF8EE
:10EF600094821F683A6872B300210C4602E00134B3
:10EF7000944226D207EBC405AB68002BF7D06E682D
:10EF8000F6B2012EF3D16868B8F80030B3EB104F39
:10EF9000EDD16A68013322F0FF0242F002026A609A
:10EFA000A868A8F80030FFF771FE314628B96B68F1
:10EFB00023F0FF0343F003036B603A68013494428B
:10EFC000D8D30029CFD100217E4A814BC2F8081145
:10EFD0001B680393039B7B4BD3F80C33DB0643D4B2
:10EFE0004FF480617B4B764A1B685B01DBB282F891
:10EFF0002A33C2F88411516006B0BDE8F0870622BA
:10F00000714B1A6006B0BDE8F087FFF76BFCFFF7A5
:10F01000D7FD002866D1704BC6F81C011B68019310
:10F02000019B684BD3F80C23D00789D500216B4A8C
:10F03000C3F80011126803240292029AD3F814361E
:10F040006149A3F50043013B022B8CBF0323644AB3
:10F050000C6098BF52F82330624A1846136006B01D
:10F06000BDE8F047FFF718BA5F4BDFF888811F68EB
:10F070003A6872B300210C4602E00134944226D271
:10F0800007EBC405AB68002BF7D06E68F6B2012E13
:10F09000F3D16868B8F80030B3EB104FEDD16A686F
:10F0A000013322F0FF0242F002026A60A868A8F869
:10F0B0000030FFF7EBFD314628B96B6823F0FF0302
:10F0C00043F003036B603A6801349442D8D30029BB
:10F0D000CFD100213B4A454BC2F810111B68049365
:10F0E000049B7DE7E02384F82A3365608AE738498A
:10F0F000C3F808213E4A0B681268059393683A48A2
:10F1000032490360D2F80480059AC1F800808BB1BF
:10F11000B8F1000F0ED01B68102B03D8D8F80010E0
:10F12000102909D94CF2060303222E4918460B6018
:10F130003A6094E71023F7E7DFF8B89059B300205E
:10F1400008F1040A044602E001348C4221D2E500B1
:10F1500008EB05039A68002AF6D05E68F6B2012E25
:10F16000F2D1D3F804C0B9F80020B2EB1C4FEBD1B8
:10F170005968013221F0FF0141F00201596098689D
:10F18000A9F80020FFF782FD68B13046D8F80010DA
:10F19000DAE70028D2D102200E4B4FF48061084AF2
:10F1A0001B68386021E75AF80530304623F0FF032A
:10F1B00043F003034AF80530D8F80010C4E700BF55
:10F1C00000E100E000A002403418022038180220BC
:10F1D00008A10240301802201CA1024000A10240F8
:10F1E00080D601002C1802203C18022010A10240F9
:10F1F00040180220701E022030B4184B1C6825688D
:10F200006DB1A368834227D0002302E08968814260
:10F2100019D00133DA00AB4204EB0201F6D1104BF6
:10F220001C6825686DB1A368834215D0002302E0F5
:10F230008968814207D00133DA009D4204EB020164
:10F24000F6D130BC70470432A35823F0FF0343F0DB
:10F250000303A35030BC70470422F5E73C1802209A
:10F2600038180220002800F0B880002900F0B5808E
:10F27000002A00F0B2802DE9F04F046A85B0002C1E
:10F2800000F0A680406A002800F0A28042F6874580
:10F290004FF0000A554EA84286F800A040F2A08028
:10F2A0000827DFF88091204616460D464422514635
:10F2B000C9F800400DF013F8D9F8002004F1440318
:10F2C000DFF8648182F801A082F802A082F803A02E
:10F2D0001770184644225146C8F800300CF0FFFF62
:10F2E000D8F8002004F18803DFF840B1177082F8E5
:10F2F00001A082F802A082F803A018464FF4007221
:10F300005146CBF800300CF0EAFF394B04F5227C73
:10F31000C3F800C0514660464FF400720CF0DFFFA6
:10F320004FF4205C06214FF0010E4FF401304FF4F2
:10F330008832304B04F591645C602F4CC3F808C0F0
:10F340009981A3F800E019461C612C4BDFF8E0C05E
:10F3500020612B48636003F5C073A060C4F800C04F
:10F360002848E360626103F0F1FD002832D14FF0DC
:10F37000020C2024D9F80010DBF8002029601C4B77
:10F38000D8F80010DFF8ACE01F4D3160CEF8002057
:10F390001B681E4902F500722A601D4E1D4A1E4D53
:10F3A0000B6003F500731D4933602880C2F814C553
:10F3B00009681B4B03910399C2F81C7519683B44FB
:10F3C00002910299C2F824451B680193019B01E058
:10F3D0004CF2070005B0BDE8F08F4CF20E0070470C
:10F3E0004CF2040005B0BDE8F08F00BFA11F022061
:10F3F0006C180220581802207C180220800004009B
:10F400000001040044180220501802204C18022069
:10F410004818022000A00240721E022014A50240DB
:10F420001CA50240781802207018022074180220CF
:10F43000400008005418022000285ED070B4334BFE
:10F4400083B01A68324B82421ED81B68314983420E
:10F45000096803D8304C2468844246D881420ED9CA
:10F460002E4B1B78002B4BD1831A2D499E099B06EE
:10F470000A682C4C4FF003014FF0020514D04CF2F7
:10F48000100003B070BC70471B689842F7D3224A43
:10F4900012689042F3D20121C31A234A9E099B06A7
:10F4A0000D461268214CEAD14368DBB29D421FD160
:10F4B000202002EBC60253681D4D03F47F432E88C3
:10F4C00043F0010343EA0643536000BF0138FCD117
:10F4D0000122184B43F8212022682B880192019ABF
:10F4E00001332B8003B070BC70478142D3D9B7E79A
:10F4F0004CF2070003B070BC70474CF20E0070472E
:10F500004CF20F0003B070BC704700BF54180220CB
:10F510004C1802205018022048180220A11F022077
:10F52000781802200CA002407018022004A00240AB
:10F53000721E022000A00240184B1B7863BBF0B47F
:10F54000174A03F0FF001468164B25681E68A5B122
:10F550000746C10063185A68D2B2032A04D19F60DB
:10F560005A6822F0FF025A605A6812F0FF0F01D168
:10F570009B682BB10130A842EBD10020F0BC704752
:10F5800006EB801021448860436823F0FF0343F0BA
:10F5900002034360F0BC704700207047A11F0220A7
:10F5A0007818022074180220F0B4154A154B14681C
:10F5B0001E682568ADB100200746C10063185A686F
:10F5C000D2B2032A04D19F605A6822F0FF025A6027
:10F5D0005A6812F0FF0F01D19B682BB101308542B0
:10F5E000EBD10020F0BC704706EB8010214488600E
:10F5F000436823F0FF0343F001034360F0BC70470E
:10F60000701802206C180220034B1B780BB903F012
:10F61000E1BD0020704700BFA11F02200B7870B52C
:10F620000646EBB1084600240A46202B154612D0A8
:10F630001370013410F8013F0A191546002BF4D15C
:10F64000002408462C700CF01EFD064B53F82630A3
:10F650005860204670BD10F8013F002BE5D1EFE760
:10F660000D46EDE7981902200B7870B50646EBB110
:10F67000084600240A46202B154612D01370013488
:10F6800010F8013F0A191546002BF4D10024084B4D
:10F690002C70084653F826500CF0F5FC28602046E4
:10F6A00070BD10F8013F002BE5D1EFE70D46EDE707
:10F6B0009819022008B58022002102480CF00FFEA4
:10F6C000002008BD98180220F0B51F4C83B00646F4
:10F6D0001E4920460CF070FD10BB054601468022F5
:10F6E00020460CF0FCFD1A4B0195186880222B4631
:10F6F0000095214604F04CF9074616480CF087FDAA
:10F700008742054614DB0246214612480CF094FD60
:10F7100070B93046611903B0BDE8F040FFF7CABFC9
:10F720002046802200210CF0DAFD002003B0F0BD5D
:10F7300009480CF06CFD0449024607480CF07CFDBA
:10F740004FF0FF30F2E700BF981802208CD601007E
:10F75000941802207CD6010094D60100F0B51C4C10
:10F7600083B080220021064620460CF0B8FD00231D
:10F77000184A21461068CDE90033802204F008F9C8
:10F78000074615480CF043FD874218DB0546024644
:10F79000214611480CF050FD88B961193046FFF739
:10F7A0003DFF30B10D4B53F826301A685A6003B054
:10F7B000F0BD304603B0BDE8F040FFF785BF084814
:10F7C0000CF025FD0249024605480CF035FDE9E73D
:10F7D00098180220941802209CD601009819022043
:10F7E00094D601004FF0FF3310B5094C28220021B8
:10F7F000084823600CF073FD40F2012200216620CE
:10F8000004F034F800282060B4BF0320002010BDAD
:10F8100094180220981902202DE9F041662882B040
:10F8200040F0CA80B1F5007F40F0AD8040F2022385
:10F830009A4240F0A880634C25684DB36368002B62
:10F8400000F09D80A368002B00F09B80E368002BF4
:10F8500000F09F802369002B00F09D806369002BDE
:10F8600000F0A680A369002B00F0A480E369002BC0
:10F8700000F09380236A53B1636A092543B10C20D9
:10F880000CF071FF4FF0FF3002B0BDE8F0810825A9
:10F89000782003F075FC44F825000028EFD078228A
:10F8A00000210CF01CFD012103264FF0FF3054F81D
:10F8B00025308022996054F8253000211E67586059
:10F8C00041480CF00CFD414F414A80213E48FBF776
:10F8D00073FB3D48D7F8008000260CF098FC3346B7
:10F8E0000246394940460196009603F06FFF804674
:10F8F00035480CF08CFC404521D1DFF8E0803146E2
:10F90000802240460CF0EBFC38683346CDE90066B7
:10F910004146802204F03CF807462E480CF077FC64
:10F92000874206463BDB024641462A480CF084FCEF
:10F93000A8BB08EB06012846FFF796FE78B154F8FD
:10F94000250003F03BFC7822002154F825000CF040
:10F95000C6FC00234FF0FF3044F8253094E72846DA
:10F96000FFF7B2FE0028EAD1022254F8253045F014
:10F97000F14040F4D0109A6002B0BDE8F08101255A
:10F9800086E7022584E716200CF0EDFE4FF0FF30ED
:10F990007AE703257CE704257AE7072578E70E4810
:10F9A0000CF035FC0D4902460B480CF045FCC6E74F
:10F9B00005256DE706256BE72F200CF0D4FE4FF0F0
:10F9C000FF3061E7981902201819022094180220CC
:10F9D00018D7010028D7010094D6010098180220FA
:10F9E0002DE9F04F83B0002900F01E81642A914672
:10F9F00000F21A810446084688460CF008FC642888
:10FA000000F212818B4BA34340F0068124F0F144B5
:10FA100024F4D014092C00F3FF80874F57F82430CA
:10FA2000002B00F0F9809A68002A00F0F580002C85
:10FA3000C0F2F2809B68022B40F0EE807F4E802265
:10FA4000002130460CF04BFC7D4A80213046FBF70C
:10FA5000B3FA57F824300546C0F180011B68794A93
:10FA60003018FBF7A9FA57F8243005441B6F03F050
:10FA70000302032A00F0BD809B074CBF724B734BFF
:10FA8000C5F180017019724AFBF796FA0544C5F179
:10FA90008001701943466F4AFBF78EFA0544802DAA
:10FAA00000F3BA80DFF8C4A16448DAF800500CF023
:10FAB000AEFB002302460193284600935F4903F002
:10FAC00085FE05465D480CF0A2FBA84240F0A480EC
:10FAD0002046FFF7F9FD0546002840F09D800146CD
:10FAE000802256480CF0FBFB5B4A80215348FBF711
:10FAF00063FA57F82430C0F180011B68574A30443C
:10FB0000FBF75AFA4D48DAF800B00CF080FB2B46B0
:10FB10000246019500954949584603F057FE0546AF
:10FB200046480CF074FBA84276D12046FFF7CCFD86
:10FB30000546002870D1032157F824304A469960C1
:10FB400057F8240041460C300CF09CFB29468022DB
:10FB50003A480CF0C4FB424A80213848FBF72CFAA3
:10FB600057F82430C0F180011B683C4A3044FBF751
:10FB700023FA3248DAF800800CF049FB2B460246A3
:10FB8000019500952D49404603F020FE05462B487F
:10FB90000CF03DFBA84202D12046FFF7DFFD80229A
:10FBA000002126480CF09BFB2E4A80212348FBF7BE
:10FBB00003FA0023C0F180010546224A3018FBF702
:10FBC000FBF957F824300544C5F180015B6F1D4AED
:10FBD0007019FBF7F1F957F82430291870180C3315
:10FBE000C1F180011A4AFBF7E7F9002003B0BDE834
:10FBF000F08FC5F180011C4B154A7019FBF7DCF939
:10FC00000544C5F1800170194346124AFBF7D4F947
:10FC10000544802D7FF746AF09200CF0A4FD4FF07E
:10FC2000FF3003B0BDE8F08F0E200CF09CFD4FF0CC
:10FC3000FF30DBE700009A7898190220181902209B
:10FC4000B4D60100C0D60100DCD60100E4D6010024
:10FC5000CCD60100D4D60100E8D60100F4D60100CC
:10FC6000F8D6010008D70100C4D60100941802207C
:10FC70002DE9F041454B82B083437BD120F0F14424
:10FC800024F4D014092C75DC414D55F824000028CB
:10FC900070D08368002B6DD0002C6BDB8368032B46
:10FCA0000DD003F08BFA7822002155F824000CF0D7
:10FCB00016FB002045F8240002B0BDE8F081354E67
:10FCC0008022002130460CF00AFB334A8021304666
:10FCD000FBF772F955F82430C0F180011B682F4AF8
:10FCE0003044DFF8C080FBF767F93046D8F8007081
:10FCF0000CF08DFA0023024631463846CDE9003338
:10FD000003F064FD074630460CF081FAB84237D163
:10FD10002046FFF7D9FC074690BB014680223046BB
:10FD20000CF0DDFA1E4A80213046FBF745F955F804
:10FD30002430C0F180011B68184A3044FBF73CF9BD
:10FD40003046D8F800800CF062FA3B460246019734
:10FD500000973146404603F039FD074630460CF027
:10FD600056FAB8420CD12046FFF7AEFC40B955F820
:10FD7000240096E709200CF0F6FC4FF0FF309BE7DB
:10FD800023200CF0F0FC4FF0FF3095E700009A784C
:10FD90009819022018190220A8D60100F4D60100F3
:10FDA000B4D60100941802202DE9F04140F202245B
:10FDB000A14202D1511E012906D916200CF0D3FC14
:10FDC0004FF0FF30BDE8F081002BF6D006990029F6
:10FDD000F3D03C49814301D00920EFE720F0F14402
:10FDE00024F4D014092CF7DC374D55F824100029E1
:10FDF000F2D088680028EFD0002CEDDB022A8A6858
:10FE000037D1032A56D1069A042AD6D1DFF8C88002
:10FE10001B684F6F80224B67404600210CF05FFA51
:10FE20002A4A80214046FBF7C7F80123C0F1800130
:10FE30000646274A4044FBF7BFF855F824300644ED
:10FE4000C6F180015B6F224A08EB0600FBF7B4F8AD
:10FE500055F82430311808EB01000C33C1F1800152
:10FE60001C4AFBF7A9F855F824304FF0FF305F67C4
:10FE7000A4E7FAB18A68032A1CD08A68042A19D038
:10FE8000069A9008421E012A97D8069A920794D1A2
:10FE90001A68022A10D00A2A8FD10222022806D11B
:10FEA0005B68022B0AD00A2B87D142F002020A6754
:10FEB000002083E70E2081E70122EFE742F00102F4
:10FEC000F5E700BF00009A789819022008D70100D2
:10FED000C0D60100CCD601001819022010B540F29E
:10FEE0000224A14202D1511E012905D916200CF08D
:10FEF0003AFC4FF0FF3010BD002BF7D0029B002BD7
:10FF0000F4D0234B834305D009200CF02CFC4FF098
:10FF1000FF3010BD20F0F14020F4D0100928F3DCB0
:10FF20001C4B53F82030002BEED099680029EBD001
:10FF30000028E9DB0299022A09689A6803D1032A9A
:10FF40001FD00E20D3E7002AFBD09A68042AF8D0ED
:10FF5000072901F00302C9D9002AC7D11B6F9907ED
:10FF600003D50A21012202980160DB0704D5022390
:10FF7000029941F822300132029B92001A6000205F
:10FF8000B5E70429B2D15B6F029A00201360AEE797
:10FF900000009A7898190220002900F09B83F0B5A0
:10FFA000A24C022883B00D46236800F093800A28F3
:10FFB0003ED01BB19B68032B00F0268163681BB108
:10FFC0009B68032B00F00F81A3681BB19B68032B78
:10FFD00000F0F880E3681BB19B68032B00F0E18020
:10FFE00023691BB19B68032B00F0228163691BB15D
:10FFF0009B68032B00F06081A3691BB19B68032BF6
:020000040001F9
:1000000000F04981E3691BB19B68032B00F032814A
:10001000236A1BB19B68032B00F01B81636A1BB131
:100020009B68032B00F0AC804FF0FF3003B0F0BDB5
:100030001BB19B68032B00F0198363681BB19B689D
:10004000032B00F0E182A3681BB19B68032B00F037
:10005000BB82E3681BB19E68032E00F0D681236942
:100060001BB19B68032B00F0E98163691BB19B689E
:10007000032B00F0FB81A3691BB19B68032B00F0ED
:100080000D82E3691BB19B68032B00F01F82236A7A
:100090001BB19B68032B00F03382636A002BC3D033
:1000A0009B68032BC0D128460CF0B1F80646606A65
:1000B0000C300CF0ACF88642B6D1616A28460C319F
:1000C0000CF0ADF80028AFD1636A1A6F9207ABD578
:1000D00009261AE11BB19B68032B00F0E1826368DB
:1000E0001BB19B68032B00F0A982A3681BB19B681E
:1000F000032B00F04F82E3681BB19E68032E00F0D3
:10010000EC8023691BB19B68032B00F0308163698D
:100110001BB19B68032B00F04481A3691BB19B6852
:10012000032B00F05881E3691BB19B68032B00F09F
:100130000182236A1BB19B68032B00F01382636A60
:10014000002B3FF471AF9B68032B7FF46DAF284603
:100150000CF05DF80646606A0C300CF058F88642E8
:100160007FF462AF616A28460C310CF058F8002821
:100170007FF45AAF636A1A6FD2077FF555AFA7E7CE
:1001800028460CF044F80646606A0C300CF03FF844
:1001900086427FF449AF616A28460C310CF03FF883
:1001A00042E728460CF033F80646E0680C300CF0C5
:1001B0002EF886427FF414AFE16828460C310CF02B
:1001C0002EF80DE728460CF022F80646A0680C3001
:1001D0000CF01DF886427FF4FDAEA16828460C3174
:1001E0000CF01DF8F6E628460CF011F8064660689B
:1001F0000C300CF00CF886427FF4E6AE61682846BD
:100200000C310CF00CF8DFE608460CF000F806465E
:1002100020680C300BF0FBFFB0427FF4CFAE2168BA
:1002200028460C310BF0FBFFC8E600BF98190220EE
:1002300028460BF0ECFF064620690C300BF0E7FF78
:1002400086427FF4D3AE216928460C310BF0E7FFDC
:10025000CCE628460BF0DBFF0646206A0C300BF09C
:10026000D6FF86427FF4DAAE216A28460C310BF0C5
:10027000D6FFD3E628460BF0CAFF0646E0690C30ED
:100280000BF0C5FF86427FF4C3AEE16928460C310E
:100290000BF0C5FFBCE628460BF0B9FF0646A06987
:1002A0000C300BF0B4FF86427FF4ACAEA169284657
:1002B0000C310BF0B4FFA5E628460BF0A8FF06466C
:1002C00060690C300BF0A3FF86427FF495AE616944
:1002D00028460C310BF0A3FF8EE628460BF097FF63
:1002E0000746E0680C300BF092FF87427FF409AFBD
:1002F000E16828460C310BF092FF00287FF401AF33
:10030000E3681A6FD1077FF5FCAE5868431C7FF491
:100310008DAEB94D8022002128460BF0E0FFB74A90
:1003200080212846FAF748FE54F82630C0F18001B3
:10033000B34A1B682844FAF73FFEB24B28461F68B1
:100340000BF065FF0023024629463846CDE900330D
:1003500003F03CFA074628460BF059FFB84202D199
:100360003046FFF7FBF954F8263058685EE6284619
:100370000BF04DFF064620690C300BF048FF86421B
:100380007FF4C5AE216928460C310BF048FF0028E8
:100390007FF4BDAE23691A6FD2077FF5B8AE04268D
:1003A000B3E728460BF033FF064660690C300BF0CC
:1003B0002EFF86427FF4B1AE616928460C310BF006
:1003C0002EFF00287FF4A9AE63691A6FD7077FF567
:1003D000A4AE052699E728460BF019FF0646A0694A
:1003E0000C300BF014FF86427FF49DAEA1692846C5
:1003F0000C310BF014FF00287FF495AEA3691A6F3F
:10040000D6077FF590AE06267FE728460BF0FFFE65
:100410000746E0680C300BF0FAFE87427FF41FAE0F
:10042000E16828460C310BF0FAFE00287FF417AE85
:10043000E3681A6F91073FF568AF10E628460BF0A6
:10044000E6FE064620690C300BF0E1FE86427FF4A2
:100450000CAE216928460C310BF0E1FE00287FF438
:1004600004AE23691A6F920799D4FEE528460BF073
:10047000CEFE064660690C300BF0C9FE86427FF462
:10048000FAAD616928460C310BF0C9FE00287FF4F3
:10049000F2AD63691A6F97079BD4ECE528460BF021
:1004A000B6FE0646A0690C300BF0B1FE86427FF422
:1004B000E8ADA16928460C310BF0B1FE00287FF4AD
:1004C000E0ADA3691A6F96079DD4DAE528460BF0D4
:1004D0009EFE0646E0690C300BF099FE86427FF4E2
:1004E000D6ADE16928460C310BF099FE00287FF467
:1004F000CEADE3691A6F90077FF5C9AD072604E713
:1005000028460BF084FE0646206A0C300BF07FFE76
:1005100086427FF4C2AD216A28460C310BF07FFE83
:1005200000287FF4BAAD236A1A6F91077FF5B5AD45
:100530000826EAE628460BF06AFE0646E0690C301B
:100540000BF065FE86427FF4F4ADE16928460C317C
:100550000BF065FE00287FF4ECADE3691A6FD0075D
:10056000CCD4E6E528460BF052FE0646206A0C3055
:100570000BF04DFE86427FF4E2AD216A28460C3135
:100580000BF04DFE00287FF4DAAD236A1A6FD10715
:10059000CED4D4E528460BF03AFE0646A0680C30CF
:1005A0000BF035FE86427FF4A6ADA16828460C31DB
:1005B0000BF035FE00287FF49EADA3681A6FD007BC
:1005C0007FF599AD0226A0E628460BF020FE0646F0
:1005D000A0680C300BF01BFE86427FF43AADA16898
:1005E00028460C310BF01BFE00287FF432ADA368C7
:1005F0001A6F9007E6D42CE518190220F8D60100EE
:10060000F4D601009418022028460BF000FE06469E
:1006100060680C300BF0FBFD86427FF414AD61681E
:1006200028460C310BF0FBFD00287FF40CAD63680D
:100630001A6F96077FF507AD012666E628460BF090
:10064000E6FD064660680C300BF0E1FD86427FF463
:100650004CAD616828460C310BF0E1FD00287FF4B9
:1006600044AD63681A6FD607E6D43EE508460BF042
:10067000CEFD064620680C300BF0C9FD86427FF4A3
:10068000DCAC216828460C310BF0C9FD0646002879
:100690007FF4D3AC23681A6F97073FF536AECCE4EE
:1006A00008460BF0B4FD064620680C300BF0AFFD99
:1006B00086427FF414AD216828460C310BF0AFFD63
:1006C000064600287FF40BAD23681A6FD7073FF565
:1006D0001CAE04E54FF0FF30704700BFF0B53B4C57
:1006E000C7B0266816BB0127394827600BF08FFD7D
:1006F0000546C0F5807331464FF4807206A8029318
:100700000BF0EDFD2A46324906A80BF0BBFD06AA08
:10071000009702AB2A4420212E4802F08BFD0646AA
:1007200038B100232320236047B0F0BD0E2047B02E
:10073000F0BD2220029B27601D4406AF06AB785512
:100740002B4440F20122022166205E7003F08EF8F5
:10075000071EE6DB20480BF05AFD334602461E49D1
:10076000CDE90066384603F031F8023503A9334677
:100770000A22CDE90066384603F00AF9CDE90066A1
:1007800006A92A463346384603F020F8A84203D08B
:10079000384603F0B5F8C4E7CDE9006633460A22CF
:1007A00003A9384603F0F4F80128F1DD03A802227A
:1007B0000A490BF041FD05460028E9D102233846DD
:1007C000236003F09DF82846AEE700BFC019022061
:1007D00034D70100A41F022044D701007CD60100B9
:1007E00010B50446006803F0DFF9A06818B1BDE851
:1007F000104002F0E3BC10BD0E289ABF024B53F824
:1008000020002D20704700BF54D7010070B500258F
:1008100082B002AC44F8045D06460D4620461946F7
:10082000144603F08FF960B9019B08225872987240
:10083000D872184644EA0644DC601D611A7202B0A0
:1008400070BD019B184602B070BD00BF70B50C466C
:100850000546114620461E4603F088F900B970BDD2
:10086000206808B103F0A0F9204603F095F92E6046
:10087000232070BD38B5054601F08CFA044608B156
:10088000204638BD284601F0F5FA0028F8D0446823
:10089000002CF5D000234360204638BD38B5002336
:1008A000074D084C1946202207482B6023600BF0A7
:1008B00016FD03F041F9003018BF0120404238BD59
:1008C000D4190220D0190220DC19022000232DE9BE
:1008D000F04120F0080682B0022E009340F088809C
:1008E0004B1E012B0C4656D80746002A4FD1012932
:1008F00008BF0126414A2146684601F0B5F9009B30
:100900008046002B50D0002102A840F8041DC3E906
:1009100002741E6103F016F9002842D147F2010269
:100920004FF0FF330821019D42EA0842EA606872F5
:10093000A872E87229722B746B74AB74EB740A2F73
:100940000CBF02220122AB68EE610C33AC616A611C
:10095000AB6047F201012846009F03F007F9064605
:1009600038B3286808B103F01FF9284603F014F9DA
:10097000012323253B60404601F0CAF928460BF0CD
:10098000F2FE4FF0FF38404602B0BDE8F081012989
:100990000CD0022AAED016200BF0E5FE4FF0FF3847
:1009A000F1E7019D002DCAD10C25E4E7012AA1D071
:1009B000F1E74FF0FF334FF6FF720221404601F09E
:1009C000E9F905460028D6D1404601F053FA18B19E
:1009D00045680DB14660CEE7022CD4D1009B1A6861
:1009E00042F400321A601A6842F400221A60CAE720
:1009F0002F200BF0B8FE4FF0FF38C4E7E1070100ED
:100A00002DE9F04182B0064601F034FA002863D0A7
:100A10000446002102A8276840F8041DD4F8148079
:100A200003F090F800283AD147F209030822019D0B
:100A300043EA0643EB60C5F810806872A872E8725A
:100A40002A72236847F209011B0C1B0443F00D03B3
:100A500023602368284623F400332360236823F4AB
:100A60000023236003F082F840BB4FF0FF334FF6C2
:100A7000FF720E21304601F08DF90446A0B1174CEB
:100A800054F8260020B103F087F8002344F82630FC
:100A9000304601F03DF9002002B0BDE8F081019D33
:100AA0000C20002DCDD112E0304601F0E3F90028F2
:100AB000E5D04368002BE2D04460E0E7286808B145
:100AC00003F072F8284603F067F8232027600BF044
:100AD0004AFE4FF0FF30DFE70920F8E7DC1902207B
:100AE0002DE9F043002483B08846174699460194C7
:100AF00005460A9E01F0BEF9002800F0C080C368D8
:100B00000446012B5CD02268910340F1A68039464F
:100B100001A803F017F8002840F0AB800C22019BDD
:100B20001A7258729872D872EEB1A26871688A42CD
:100B300008D1022A03F11C00317845D00A2A01D1DC
:100B4000242968D0186810B103F02EF8019B1846CC
:100B500003F022F816200BF006FE4FF0FF36304669
:100B600003B0BDE8F08347F206021646C3F81490BE
:100B7000616942EA0542DA6019615F60B8F1000F0D
:100B800004D03A46414618680BF07CFB276823687E
:100B9000314623F400332360236843F48013236039
:100BA000019E304602F0E2FF8046C0B1306808B1D5
:100BB00002F0FAFF304602F0EFFF27602320CAE779
:100BC000002EA0D01620C6E71029BBD104223189FF
:100BD0005A83198306F10C010BF054FB22E04FF409
:100BE00000324FF0FF331146284601F0D3F840B1F0
:100BF000236843F400332360236823F480132360C5
:100C0000A9E7284601F036F90346B8B14068A8B113
:100C1000C3F80480ECE7102231895A831983B11894
:100C20000BF030FB47F20702019B16469968588B80
:100C300004310144C3F81490996099E7236823F4C0
:100C4000801323600F4C54F8253018469E6902F03B
:100C5000A3FF002344F8253081E72268D2000AD49C
:100C6000022B0AD023689BB2052B0CBF232039200E
:100C700071E70C206FE739206DE723206BE709202F
:100C800069E700BFDC1902202DE9F04F85B00F9D08
:100C9000002A00F0C3808A4698468146164601F035
:100CA000E9F80446002800F0BC8003681A031FD44A
:100CB00003689BB2062B00F0AE8003689BB2072B43
:100CC0000CBF4FF0090B4FF0390BA0690368DB68CC
:100CD0009847013003D0236843F48033236058469B
:100CE0000BF041FD4FF0FF35284605B0BDE8F08F11
:100CF00018F0020F09BF0768002787F00067C7F3E5
:100D0000C06718F0100F47D12368DB0324D5236890
:100D1000A06923F4803323600368DB6898470130BF
:100D20001AD005B12D680E9BCDE900A6CDE902359C
:100D3000A0694246036869469B689847431C05467C
:100D40005CD0A0690368DB6898470130CCD0236889
:100D500043F480332360C7E7002F33D14FF0230BD8
:100D6000B3E723681A01DCD44FF48032E3691146FB
:100D7000002B08BF4FF0FF33484601F00BF88346C5
:100D80000028A2D1484601F075F820B1D0F804B08F
:100D9000BBF1000F2FD101272368D8030FD523689B
:100DA000A06923F4803323600368DB689847411C03
:100DB00005D08642B5DDE368012BB2D1D1E7002F23
:100DC000CCD0D1E74FF48032E3691146002B08BF45
:100DD0004FF0FF33484600F0DDFF834600287FF4E4
:100DE00074AF484601F046F800288DD0D0F804B022
:100DF000BBF1000F88D00023436066E7A069036859
:100E0000DB68984701300FD023684FF0230B43F481
:100E10008033236063E74FF0090B56E74FF0160B62
:100E20005DE74FF0090B5AE74FF0230B57E700BF80
:100E30002DE9F04182B0002943D0002A41D0064676
:100E40000F4601F017F80546002800F0928003686D
:100E50009BB2022B04D003689BB2042B40F0898024
:100E6000296811F0805178D102A840F8041DD5F806
:100E7000148002F067FE70BB08213304019C43F428
:100E8000E04242F00202E260C4F810806072A07298
:100E9000E072217243F4E04343F00203E360A3688D
:100EA0006A6904332261A360AB687A68934208D10F
:100EB000022B04F118003A7835D00A2B01D1242AEC
:100EC0000ED0162420460BF04EFC4FF0FF34204687
:100ED00002B0BDE8F081019C002C4CD03304D9E76E
:100EE00010223B89B918E282A3820BF0CBF9A368E8
:100EF000E28A47F202011344A360D5F800802B6810
:100F0000204643F080532B6002F030FE0746A8B124
:100F1000206808B102F048FE204602F03DFE23247E
:100F2000C5F80080CEE7102ACBD104223B8907F117
:100F30000C01E282A3820BF0A5F9D8E74FF0FF3352
:100F40004FF6FF720521304600F024FF044630B111
:100F5000732CB7D0C5F80080B4E77224B2E73046EE
:100F600000F088FF0028B2D04468002CAFD0476062
:100F7000EEE70924A6E70C24A4E700BF2DE9F04121
:100F800082B089B382B307460E4600F073FF054670
:100F900000287BD003689BB2022B77D1002102A8E6
:100FA00040F8041DD5F8148002F0CCFD30BB47F2A8
:100FB00005030822019C43EA0743E360C4F810805C
:100FC0006072A072E0722272A3680433A360AB68FF
:100FD0007268934208D1022B04F1180032783CD099
:100FE0000A2B01D1242A0ED0162420460BF0BBFB7D
:100FF0004FF0FF34204602B0BDE8F081019C002C88
:10100000E2D10C24F1E710223389B118E282A382E5
:101010000BF038F9A368E28A47F205011344A36094
:101020002B6820461B0C1B0443F003032B602E6827
:1010300002F09CFD8046D8B94FF0FF334FF6FF72A7
:101040000421384600F0A6FE044608B32B681B0CAA
:101050001B0443F002032B60C7E7102AC4D104220B
:10106000338906F10C01E282A3820BF00BF9D1E780
:10107000206808B102F098FD360C3604204646F090
:10108000020602F089FD23242E60AEE70924ACE7B6
:10109000384600F0EFFE0028ACD04468002CA9D000
:1010A000C0F80480D2E700BF2DE9F04182B00646C7
:1010B00000F0E0FE002867D0036805469BB2042BD1
:1010C00062D10021324A304600F036FE0146002847
:1010D0005CD102A840F8041D6F6902F033FDA8BB83
:1010E00047F208030822019C43EA0643E3602761B4
:1010F0006072A072E0722272A36847F208010433A2
:10110000A3602B6820461B0C1B0443F006032B60D6
:101110002F6802F02BFD8046E8B94FF0FF334FF601
:10112000FF720721304600F035FE044608B32B68F5
:101130001B0C1B0443F004032B6020460BF013FB35
:101140004FF0FF34204602B0BDE8F081019C002C36
:10115000D2D10C24F1E7206808B102F025FD3F0C44
:101160003F04204647F0040702F016FD23242F60B9
:10117000E3E7304600F07EFE0028E3D04468002C10
:10118000E0D0C0F80480D2E70924D6E72324D4E7CE
:10119000E10701002DE9F04F002585B00F4690468C
:1011A0000295064600F066FE0446002800F01C8109
:1011B00003689BB2072B0AD1036805681B0116D48C
:1011C00015F4803519D0056815F4803524D14FF019
:1011D0000909029B13B1284600F09AFD48464FF0DA
:1011E000FF390BF0C0FA484605B0BDE8F08F15F4A2
:1011F00080356DD14FF02309EBE74FF480324FF08B
:10120000FF331146304600F0C5FD814600287ED0F0
:10121000256815F48035DCD04FF0FF300023CDE990
:101220000003754AE16802A800F01EFD029B054616
:10123000002B00F0DD800021226904A81A61A26859
:1012400040F8041D9A60E268DA60D4F8149002F065
:1012500079FC002843D147F20C030821DDF80CB0DB
:1012600043EA0643CBF80C30CBF810908BF809001A
:101270008BF80A008BF80B008BF80810236847F2F4
:101280000C011B0C1B0443F0080323605846D4F8E0
:10129000009002F06BFC824648BB226800994FF038
:1012A000FF330A40226009214FF6FF72304600F0FA
:1012B00071FD8146002800F085802368019A1A4359
:1012C000226023681B0C1B0443F00703236080E7A4
:1012D0006FF000624FF00063CDE90023A1E7DDF875
:1012E0000CB04FF00C09BBF1000FC7D171E7DBF870
:1012F000000008B102F058FC4FEA194958464FEA7D
:10130000094902F049FC49F00703236072E73046BF
:1013100000F0B0FD30B1D0F80490B9F1000F01D069
:10132000456075E72368D9033FF576AF334D0299E1
:1013300055F826309B694B6147B18B680A2B24D046
:10134000022B03D1D8F80020102A32D00A682C488A
:10135000024042F005020A60029A116841F400312D
:101360001160116841F4002111602368034043F0CB
:101370000703236055F8260002F00EFC00234846C0
:1013800045F8263005B0BDE8F08FD8F80020242AB3
:10139000DCD13A7010227B6055F8263007F110003E
:1013A0009B8B3B8155F8261020310AF06BFF029988
:1013B000CCE73A707B6055F8263007F10C009B8B28
:1013C0000422EEE7304600F055FD38B1D0F8049025
:1013D000B9F1000F02D0C0F804A06EE72368019AAB
:1013E000A94613432360A1E705464FF00909F0E63B
:1013F0004FF00C09F2E600BFE1070100DC19022002
:101400000000FFFF2DE9F041012982B040F09880F3
:1014100015461E46074600F02DFD0446002800F044
:101420009580142D6ED0192D62D1002E00F0908081
:1014300030460AF0ECFE089B984240F08980236811
:101440009BB2022B40F082803146A068FEF7A4FDDB
:10145000009001307ED023689A025ED423685B023C
:101460005BD400222668236802A843F4001323609B
:10147000042140F8042DD4F8148002F063FB002806
:1014800058D147F203030822019D43EA0743EB606A
:10149000C5F810806872A872E8722A724FF0080CC2
:1014A000002310203021AA686B756244AA60AB75D6
:1014B000EB75AB76EB7685F814C028766976042256
:1014C000694628680AF0DEFE47F20301284602F06A
:1014D0004DFB804618BB4FF480024FF0FF3311469E
:1014E000384600F057FC0546002835D0266000E05D
:1014F0002A2528460BF037F94FF0FF35284602B071
:10150000BDE8F08126B3089B042B23D10025336866
:10151000C361284602B0BDE8F0812325E9E72868C9
:1015200008B102F041FB284602F036FB2325266075
:101530002660DEE7019D002DB0D126600C25D8E79E
:101540002A200BF010F94FF0FF35D7E70925D0E737
:101550000E25CEE71625CCE7384600F08BFC20B1EF
:10156000456815B1C0F80480C0E72660C6E700BF33
:1015700000F0A0BC2DE9F04F4FF0000C01246C4EA0
:10158000DFF8B8A1DFF8B89185B00746154601939A
:10159000A6F800C0CAF80040C9F8004071B108467A
:1015A0000A2261460AF092FD4FF6FE73421E9A42ED
:1015B00000F28680030243EA20203080DFF8848135
:1015C000D8F80030002B77D15A4A13605A4A13607A
:1015D000002F65D038460AF01AFE834625B1EA6925
:1015E00012B1516866296FD04FF0FF32002104AE6E
:1015F00046F8041D30465946009202F0A3FA009ABC
:1016000000284FD147F20D014FF0080C039C41EA2E
:101610000241E16022616072A072E07284F808C049
:10162000002D6AD06A6822F0080102296ED1A968EB
:10163000022908BFCAF800100A2A14BF0122022298
:10164000A261EA68C9F800102262AA68E2612A6809
:101650006261A2681032A2602FB1206818B15A46A8
:1016600039460AF00FFE012347F20D012046C8F863
:10167000003002F07BFA002846D14FF0FF3303938D
:1016800031462046FAF7A6F8D8F80030012BF7D0FB
:10169000294B186860BB274B019A1B6813600CE04C
:1016A000BB469BE7039C002CBAD10C200023C8F852
:1016B000003005B0BDE8F08F732005B0BDE8F08FB5
:1016C000162005B0BDE8F08F9168B1F5007F8BD191
:1016D00040F20221D068884286D19169002983D0E6
:1016E0006868FEF759FC431C3FF47EAF02467DE775
:1016F000114B18680028E0D0D8E72946102204F1E1
:1017000014000AF0ECFDA4E72320CFE72F200BF014
:101710002AF8A2681032A26017B94FF0FF30C5E76F
:1017200020680028F9D05A4639460AF0ABFDF4E7A4
:10173000741E0220D4190220CC190220C4190220E0
:10174000C8190220D019022038B50B4C2368022B8F
:1017500000D038BD30B10546406901F02FFD284664
:1017600001F02CFD0023054A054923601360086839
:10177000BDE8384002F018BAD0190220CC19022076
:10178000D81902202DE9F04F01F41043B3F5104FA2
:10179000054689B00E46C0684ED0040C204600F0C5
:1017A00069FB48F20D039E420746A04631D0002F48
:1017B0003ED0404633462A46394602F0B7FD98B33C
:1017C00048F207039E4252D848F206039E4280F038
:1017D000528148F202039E4200F0248178D948F2F7
:1017E00003039E4200F05F8148F205039E421FD131
:1017F0003B689BB2032B17D16B69002B00F0E4818F
:101800000E2B00F29381B84A52F823307B600020FF
:101810000BE0DFF8EC922F68D9F80030012B15D0DF
:1018200017B1384602F0C0F9002009B0BDE8F08FCA
:1018300028680028F6D1F7E700F0D4FA804600F0D7
:1018400019FB07464446002FB3D1F1E76B69002B23
:101850004DD00E2B96BFA44A2D2152F823100223FF
:10186000A24A1160C9F80030002FDAD1DCE748F253
:101870000C039E4200F0248117D848F208039E42D0
:1018800000F0E98048F209039E42D1D13B689BB247
:101890000D2BC9D16869002800F09E810E2800F246
:1018A0004581914B53F82030B0E749F201039E4245
:1018B00000F09B8049F202039E42B9D13B689BB283
:1018C000072BB1D13B68002043F480333B60ACE789
:1018D00048F201039E42ABD13B68012BA4D1686959
:1018E0000028DBD102233B60AB697B619DE7804B25
:1018F0001F60AC6963011846039301F041FC02903C
:10190000002800F00381E5002819800001F038FC70
:10191000002800F00D81002C5FD005F11002831823
:101920000193029B0424DFF8DCA1DFF8DCB100F1B5
:10193000100803F120061DE00A2248F80C2C4FF095
:101940002402404608F8102C28F8083C56F8102CC1
:101950000AF098FC56F8103C08F108081C443B19A2
:1019600046F8083C019B46F8046C43452C4406F1BC
:1019700020062CD03B593A1946F8203C5368DAF837
:101980000010022B14BF02200A20DBF8003046E9C9
:10199000070146F8143C108AA8F1100346F8100C11
:1019A000558A46F80C3C534B1434042807EB0401C9
:1019B0001B88C1D11022022028F8083C48F80C0CE2
:1019C00008F8102C56F8102CA8F10400C0E70022EB
:1019D000DDE902130B4443F8042C0222464BC9F8FC
:1019E0000020029A00201A601FE73C6814F40024CB
:1019F00000F0A280AB68042B00F2FC800023296871
:101A00006A68CDE90633CDE90412B86904A9036810
:101A10005B689847013000F0D3803B6843F4803323
:101A20003B6001E73B68D8007FF5FEAE3B6823F0E2
:101A300080533B606869002800F097800E288EBFB5
:101A40002D23294B53F8203000207B603B6843F462
:101A500080233B60E9E63B689BB2062B7FF4E4AE53
:101A6000686900287FF41AAF3B681B0C1B0443F025
:101A700007033B60D9E63B68D9027FF5D5AE6B69B9
:101A8000002B5ED13B6843F400333B603B6823F09E
:101A900080633B603B681A013FF5C6AE174B0120DF
:101AA00043F82450C1E63B689B027FF5BDAE6869F0
:101AB00000287FF4F3AE3B6843F480033B60B4E658
:101AC0003B689BB2082B7FF4AFAE6B69002B7FF4B1
:101AD00097AE0A4B012043F824503B681B0C1B04B3
:101AE00043F009033B60A0E654D70100CC19022063
:101AF000D8190220741E0220D4190220DC190220F9
:101B0000D0190220C8190220C419022001F056FB86
:101B10000C2002234B494C4A08602F68029911603F
:101B2000C9F80030002F7FF47CAE7DE62D236DE6F2
:101B30000C22444B1A6050E7286802F035F8204622
:101B400073E60E2B8EBF2D23404A52F823307B6064
:101B50003B6843F480233B606B696B2B3B6842D04E
:101B600023F0806300203B605FE63B6843F4003372
:101B70003B603B6843F400233B603B681B0C1B0449
:101B800043F005033B6050E60223102643600670D5
:101B90002B8A05F1140103810C300AF073FB6B688A
:101BA0002A68CDE90646CDE90423B86904A903688B
:101BB0005B68984701307FF430AF204601F0FEFAB1
:101BC000286801F0F1FF2FE63B6800201B0C1B0486
:101BD00043F004033B6028E63B681B0C1B0443F006
:101BE0000E033B6021E613F0806319D00C23002024
:101BF0007B601AE66B8A002B3FF400AF242001F0D3
:101C0000BFFA04460028DBD06A8A102A0ED0042AC4
:101C1000BAD0286801F0C8FF204601F0CFFA03E6E9
:101C20003A68184642F080623A60FEE50A232426AC
:101C3000436006702B8A05F11401038110300AF00D
:101C400021FBACE7CC190220D419022054D70100A3
:101C500008B54FF48072002102480AF040FB0020D2
:101C600008BD00BFC41F0220F8B5284B06461D68FA
:101C70000846E5B11C6A002C3BD01C6C002C3AD005
:101C80001C6E002C39D0D3F8801079B1D3F8A01095
:101C9000A9B3D3F8C010A1B3D3F8E01099B34FF0B3
:101CA000FF350C200AF05FFD2846F8BD04254FF0F3
:101CB000010C4FF0FF376C0143F804C01C4411467F
:101CC0006761224601F042FC0346A06158B11B68DF
:101CD0001B68984710B934602846F8BDA06901F028
:101CE00053FC0023A3612046202200210AF0F7FACA
:101CF000D5E70125DBE70225D9E70325D7E7052549
:101D0000D5E70625D3E70725D1E700BFC41F02208A
:101D1000072800D9704710B5064C04EB4014A069A1
:101D200008B101F031FC2046BDE81040202200211E
:101D30000AF0D5BAC41F022007282DE9F04118D8AF
:101D4000134D44012B592F199BB1084611463A46B1
:101D5000D7F8188001F0FAFBB861B8B103681B68C6
:101D60009847064648B9404601F00EFC3046BDE8AB
:101D7000F08105263046BDE8F081B86901F004FC29
:101D80002819C0F818803046BDE8F0810426F7E72E
:101D9000C41F0220F0B5124E4001345883B01440E5
:101DA0008C42019306EB000713D07B688BB9335844
:101DB0001B0111D40D4614463E4606E0736843B934
:101DC00001A93846F9F706FD20B933682340AB4234
:101DD000F4D1002003B0F0BD732003B0F0BD00BF0C
:101DE000C41F0220224B1A6812B15A69824231D0B4
:101DF0001A6A12B15A6B82422ED01A6C12B15A6D05
:101E000082422BD01A6E12B15A6F824228D0D3F878
:101E100080201AB1D3F89420824223D0D3F8A02096
:101E20001AB1D3F8B42082421ED0D3F8C0201AB120
:101E3000D3F8D420824219D0D3F8E0203AB1D3F8B5
:101E4000F430834214BF4FF0FF30072070474FF04B
:101E5000FF30704700207047012070470220704714
:101E60000320704704207047052070470620704704
:101E7000C41F0220072807D8044B40011A581844F1
:101E8000002A08BF0020704700207047C41F0220AE
:101E900019B1072802D908230B607047044B400191
:101EA0001A58002AF7D01B58C3F302430B6070473F
:101EB000C41F022070B50728049D1FD8124C400192
:101EC00026580444D6B1012912D1042A10D14BB1AD
:101ED00045B12A68042A05D10022616810461960BC
:101EE000626070BD16200AF03EFC4FF0FF3070BDFE
:101EF0002A200AF038FC4FF0FF3070BD09200AF0AC
:101F000032FC4FF0FF3070BDC41F0220072810B50F
:101F100016D8114C4301E05890B1012905D002298F
:101F200014D1E058C0F3C06010BD12F00100E258B7
:101F30001ABF002042F0006222F00062E25010BDA1
:101F400009200AF010FC4FF0FF3010BD16200AF0F7
:101F50000AFC4FF0FF3010BDC41F02202DE9F041F4
:101F60002E4CF9F7D1FC03272D4D2E4E04F180089D
:101F700002E0083444453BD014F8043C022BF8D16D
:101F800020682988026892B2914233D0298A91420E
:101F900032D0298C91421CD02B8E93422ED0B5F892
:101FA000403093422FD0B5F8503093422DD0B5F841
:101FB000603093422BD0B5F87030934229D0B5F8F9
:101FC0008030934227D0B5F89030934208BF092360
:101FD000CFD105EB03135A68D968904780B9012225
:101FE000206804F8042CF368083498474445C3D1AA
:101FF000BDE8F0810023ECE70123EAE70323E8E7EB
:1020000004F8047CB5E70423E3E70523E1E70623AE
:10201000DFE70723DDE70823DBE700BF381B0220EB
:10202000FC1902209C1A022008B5A02200210248B7
:102030000AF055F9002008BDFC1902200388002B86
:1020400045D042680146002A50D0304A1088834269
:102050003DD02DE9F047148AA34235D0158CAB4210
:1020600032D0168EB3422FD0B2F84070BB422BD084
:10207000B2F850C0634527D0B2F860E0734523D072
:10208000B2F8708043451FD0B2F880904B451BD00A
:10209000B2F890A0534517D0E0B15CB365B36EB30E
:1020A00077B3BCF1000F2DD0BEF1000F20D0B8F1F6
:1020B000000F29D0B9F1000F0BD00920BAF1000FA1
:1020C00008D00420BDE8F0870720BDE8F08707208E
:1020D00070470820000113524B68024453608B681C
:1020E00000209360CB68D360BDE8F0870E20704776
:1020F0000620EFE70120EDE70220EBE70320E9E708
:102100000420E7E70520E5E70720E3E7FC190220C4
:1021100038B5864A0B6810889BB2984229D0108A3D
:10212000984226D0108C984223D0108E984220D00E
:10213000B2F8400098421CD0B2F85000984218D033
:10214000B2F86000984214D0B2F87000984210D0F3
:10215000B2F8800098420CD0B2F890209A4208D091
:102160008868002800F0A980714B1B6998470020FF
:1021700038BD8868002800F091806E4A1568002DEF
:102180003BD09468002C00F09A801469002C00F079
:1021900098809469002C00F09680146A002C00F05E
:1021A0009480946A002C00F08680146B002C00F060
:1021B0009080946B002C00F09080146C002C00F048
:1021C0009080946C002C00F09080146D002C00F036
:1021D0009280946D002C00F09080146E002C00F022
:1021E0009280946E002C00F09080146F002C00F010
:1021F0008E80946F002CB7D10F2502EBC50442F8F6
:102200003500A3804C4B1A78012A60D01A7A012A33
:1022100047D01A7C012A5ED01A7E012A5FD093F83B
:102220002020012A5FD093F82820012A5FD093F85C
:102230003020012A5DD093F83820012A5FD093F82E
:102240004020012A5DD093F84820012A61D093F8FC
:102250005020012A5FD093F85820012A5DD093F8CE
:102260006020012A5BD093F86820012A59D093F8A6
:102270007020012A57D093F87820012A10D0102D11
:102280001BD000242B4B2A4A03EBC50043F83540F2
:102290008480886813699847204638BD1025B1E7C7
:1022A0000F22022403EBC200416003F83240F9F729
:1022B00023FB012038BD05259FE7002038BD0125FF
:1022C0009BE7022599E7032597E7042595E7002278
:1022D000E7E7062591E70222E3E707258DE70322DA
:1022E000DFE7082589E70422DBE7092585E70522E2
:1022F000D7E70622D5E70A257FE70B257DE70722EA
:10230000CFE70822CDE70C2577E70D2575E70E25E9
:1023100073E70922C5E70A22C3E70B22C1E70C22B3
:10232000BFE70D22BDE70E22BBE700BFFC1902206C
:102330009C1A0220B41A0220341B0220F0B4002997
:1023400052D0002850D08368002B4DD00369002B59
:102350004AD04368002B47D0C368002B44D00368A1
:10236000002B41D04369002B3ED0012600250446B6
:102370000F461F4A1F4BDFF880C01674167682F88E
:10238000206082F8286082F8306082F8386082F835
:10239000406082F8486082F8506082F8586082F8A5
:1023A000606082F8686082F8706082F878601D6111
:1023B0009D611D629D621D639D631D649D641D651D
:1023C0009D651D669D661D679D67167016721D6072
:1023D0009D600FCCACE80F0094E803008CE803008C
:1023E0003E602846F0BC70470E252846F0BC70477A
:1023F000341B0220B41A02209C1A022000283AD072
:102400002DE9F04780461D4C04F1A005A368103467
:1024100003B19847AC42F9D14FF001090026184C9E
:10242000184DDFF864A004F1800714F8043C012B78
:1024300005D0DAF80C302068984704F8049C55F869
:10244000040C083428B1DAF8103098472E8045F88B
:10245000046CBC4205F10805E7D1D8F80000182249
:10246000013800EB40000AEBC000002109F037FF03
:102470000020BDE8F0870E20704700BFFC19022045
:10248000381B0220B81A02209C1A022068B171B1D0
:10249000094A53686BB14B68088023F0FF0343F08F
:1024A000020312684B6008461047072070470E2051
:1024B00070470820704700BF9C1A02205AB3E8B149
:1024C00000232DE9F041DFF858801360D8F804307C
:1024D0001BB316460C46054698470746C8B1C4606C
:1024E00074B12046D8F808309847B86060B93846CB
:1024F000D8F80C3098470420BDE8F08107207047D9
:10250000047244728472C4723D8037600020BDE85A
:10251000F0810420F0E70E2070470820ECE700BFB0
:102520009C1A022000283DD0002900F0918038B587
:10253000524C6368002B37D0514A08465368994281
:1025400034D0D36898423DD0536998423FD0D36984
:10255000984241D0536A984244D0D36A984247D0B7
:10256000536B98424AD0D36B98424DD0536C9842EB
:1025700050D0D36C984253D0536D984256D0D36DFF
:10258000984259D0536E98425CD0D36E984261D035
:10259000536F984264D0D36F834267D0E368984703
:1025A000002038BD07207047082038BD1178032966
:1025B000C7D1002101251846E46802F83150A04730
:1025C000002038BD117A0329BED10121F2E7117C28
:1025D0000329BCD10221EDE7117E0329EAD0536A19
:1025E0009842BAD192F820100329B6D10421E1E72C
:1025F00092F828100329B3D10521DBE792F83010B7
:102600000329B0D10621D5E792F838100329ADD1BE
:102610000721CFE792F840100329AAD10821C9E782
:1026200092F848100329A7D10921C3E792F8501066
:102630000329A4D10A21BDE792F858100329A1D19A
:102640000B21B7E792F8601003299ED10C21B1E766
:102650000E20704792F86810032999D10D21A9E73F
:1026600092F87010032996D10E21A3E792F87830E2
:10267000032B93D103460F219CE700BF9C1A022035
:10268000341B022000283DD0002900F08B8038B593
:102690004F4A5368002B37D04E4B1C68A14235D0AF
:1026A0009C68A1423DD01C69A1423FD09C69A142D7
:1026B00041D01C6AA14243D09C6AA14245D01C6B08
:1026C000A14247D09C6BA14249D01C6CA1424BD087
:1026D0009C6CA1424ED01C6DA14251D09C6DA14278
:1026E00054D01C6EA14257D09C6EA1425CD01C6F8E
:1026F000A1425FD09C6F8C4262D008461369984714
:10270000002038BD07207047082038BD9C888442CF
:10271000C6D10024002003EBC40543F83400A88090
:10272000EBE79C898442BED10124F3E79C8A844272
:10273000BCD10224EEE79C8B8442BAD10324E9E7A2
:102740009C8C8442B8D10424E4E79C8D8442B6D1A9
:102750000524DFE79C8E8442B4D10624DAE79C8FFF
:102760008442B2D10724D5E7B3F844408442AFD1C4
:102770000824CFE7B3F84C408442ACD10924C9E720
:10278000B3F854408442A9D10A24C3E7B3F85C40AB
:102790008442A6D10B24BDE7B3F864408442A3D1A0
:1027A0000C24B7E70E207047B3F86C4084429ED1EA
:1027B0000D24AFE7B3F8744084429BD10E24A9E7FF
:1027C000B3F87C40844208BF0F2496D1A2E700BF33
:1027D0009C1A0220B41A022070B504460D46164613
:1027E000FBF7C4FE30B10368324629462046BDE8F7
:1027F000704018474FF0FF3070BD00BF10B5044661
:10280000FBF7F0FE20B143682046BDE810401847B2
:102810004FF0FF3010BD00BF2DE9F0470D46DDE958
:10282000088916461F460446FBF7DCFE58B1CDE981
:102830000889D0F808E03B46324629462046F4464F
:10284000BDE8F04760474FF0FF30BDE8F08700BFBC
:102850002DE9F04182B00E46174698460546FBF733
:10286000C1FE60B104460020CDE9000043463A466F
:1028700031462846A468A04702B0BDE8F0814FF079
:10288000FF30F9E72DE9F0470D46DDE908891646E6
:102890001F460446FBF7A6FE58B1CDE90889D0F8DB
:1028A0000CE03B46324629462046F446BDE8F04758
:1028B00060474FF0FF30BDE8F08700BF2DE9F041E1
:1028C00082B00E46174698460546FBF78BFE60B170
:1028D00004460020CDE9000043463A4631462846EA
:1028E000E468A04702B0BDE8F0814FF0FF30F9E79F
:1028F00070B50D4616460446FBF774FE30B14369C9
:10290000324629462046BDE8704018474FF0FF3058
:1029100070BD00BF70B50D460446FBF763FE28B1DD
:10292000836929462046BDE8704018474FF0FF30C4
:1029300070BD00BF2DE9F0410D4616460446FBF779
:1029400051FE40B1C769324629462046BC46BDE823
:10295000F041002360474FF0FF30BDE8F08100BF39
:1029600070B50D4616460446FBF73CFE30B10369D0
:10297000324629462046BDE8704018474FF0FF30E8
:1029800070BD00BF2DE9F041DDF818800D461646F8
:102990001F460446FBF726FE58B1CDF81880D0F844
:1029A00020E03B46324629462046F446BDE8F04149
:1029B00060474FF0FF30BDE8F08100BF2DE9F041E6
:1029C000DDF818800D4616461F460446FBF70AFE42
:1029D00058B1CDF81880D0F824E03B46324629465D
:1029E0002046F446BDE8F04160474FF0FF30BDE8B7
:1029F000F08100BF02F010B902F010B902F010B976
:102A000002F066B92DE9F04FDFF8CCC083B000903A
:102A10000CF13C0BDCF808302BB1DCF80020009CFA
:102A20001078A04206D00CF10C0CE345F2D103B0B3
:102A3000BDE8F08FDCF804A003EB0A08C245F2D22F
:102A40005368CDF804C0D6469C46D2F810909789BA
:102A5000AEEB0A00DFB3B9F8022090421CD3654602
:102A6000002409F1040303E05A880433824215D894
:102A700033F8046C0134A74202FB0655A0EB0200B8
:102A80001E46F1D1002081420DD00EF1010EF0451D
:102A9000DED1DDF804C0C6E765464E46338800FB4C
:102AA00003508142F1D1BEF5007FDDF804C0BAD0F9
:102AB0000123084A4FEA5E1152F821000EF01F0E62
:102AC00003FA0EFE4EEA000042F82100AFE7384656
:102AD000D9E700BFB41B0220F81B0220002850D009
:102AE0006D4BD3F8882090424BD82DE9F04FD3F8A6
:102AF0008CB083B0BBF1000F54D00BF1FF32914684
:102B000000264FF01208654F01920BF1110E06EBF3
:102B1000090253F838400132520804EB440C02F128
:102B2000120153F8315057F82CA053F83E4003EBF4
:102B3000C80CDCF804C005EB450504EB4404DAF8E6
:102B400010A057F8255057F824403AF82CA003EB72
:102B5000C10103EBCE0C49682D692469DCF804C07F
:102B6000504535F8215034F82C1015D9884211D22F
:102B7000A84208D9561CB145C0F0878002F113085D
:102B8000C5E70020704702F1FF394E457DD802F1BC
:102B9000110EBCE709F10106B34507D0102E01D094
:102BA000B34508D8002003B0BDE8F08F019A102A81
:102BB00018BF1646F6D0DFF8E8C003EBC608D8E920
:102BC000242402EB420257F8223007EB8202D2F8AB
:102BD00004E01D69002C56D02A467046A40005EB7F
:102BE00004095188043291450844FAD12919B1F8F1
:102BF00002A08244824518D941095CF8212000F0E6
:102C00001F0422FA04F919F0010F07D013E05CF851
:102C1000212022FA04F919F0010F0CD1013082456C
:102C20004FEA501100F01F04F1D101365E4508F162
:102C30000808C4D3B6E7012606FA04F49E8922EAFE
:102C40000402A0EB0E004CF821205C68002EA9D0F5
:102C50006A88824211D800212B1D03E05A88043370
:102C600082420AD833F8045C01318E4202FB0544EB
:102C7000A0EB02001D46F1D194E72B8800FB034036
:102C800003B0BDE8F08F7046B0E7BBF1100F08BF8E
:102C90000F2690D086E700BF341C0220F81B0220CC
:102CA000B41B022000284CD06B4B1A68904248D8C5
:102CB0002DE9F04F5F6883B00097002F51D07A1E46
:102CC000964600214FF0010C644C019201EB0E027C
:102CD000013253F83C50520802F1010805EB45055A
:102CE00053F8379054F825A053F8386009EB49059C
:102CF00003EBCC09D9F8049006EB4606DAF810A0ED
:102D000054F8266054F825503AF829A003EBC80B74
:102D100003EBC7093669DBF804B02D69D9F80490D4
:102D2000504536F82B6035F8295013D9A84210D2F7
:102D3000B04208D9C6454146C0F0878008F1010C71
:102D4000C4E70020704702F1FF3E71457DD8174669
:102D5000BCE73946009A8A4207D0102901D08A423E
:102D600008D8002003B0BDE8F08F019A102A18BFE0
:102D70001146F6D0DFF8E8C0DDF8009003EBC1089B
:102D8000D8E9022602EB420254F8223004EB820218
:102D9000D2F804E01F69002E55D03A467046B600BE
:102DA00007EB060A5588043292452844FAD1BD192A
:102DB000B5F802B08344834518D945095CF825204D
:102DC00000F01F0622FA06FA1AF0010F07D013E0EE
:102DD0005CF8252022FA06FA1AF0010F0CD1013016
:102DE00083454FEA501500F01F06F1D101314945E6
:102DF00008F10808C4D3B4E70121B1409E8922EA52
:102E00000102A0EB0E004CF825205C68002EA8D033
:102E10007A88824211D800213B1D03E05A8804338E
:102E200082420AD833F8045C01318E42A0EB0200E2
:102E300002FB05441F46F1D193E73B8800FB0340AA
:102E400003B0BDE8F08F7046B1E7009A102A08BFC2
:102E50000F218FD085E700BF341C0220F81B022011
:102E6000B41B022070B5002201253348510950F8E7
:102E7000214002F01F0305FA03F301322343B2F5A8
:102E8000007F40F82130F1D100242C4B21463C2218
:102E90002B481C6009F023FA10210522294B2A4EE9
:102EA000C3E90044D9605961D9615962D962596353
:102EB000D9635964D9645965D9655966D966596722
:102EC000D9679A601A619A611A629A621A639A6360
:102ED0001A649A641A659A651A669A661A679A67F6
:102EE000C3E92021C3E92244C3E92421C3E92621FF
:102EF000C3E92821C3E92A21C3E92C21C3E92E21F2
:102F0000C3E93021C3E93221C3E93421C3E93621C1
:102F1000C3E93821C3E93A21C3E93C21C3E93E2191
:102F2000C3F80411C3F80021C3F80C11C3F8082139
:102F30002046357070BD00BFB41B0220F41B022078
:102F4000F81B0220341C0220A21F02202DE9F04FA2
:102F5000874B87B01B78002B00F08C8028B321B3FF
:102F60000B78DFF8188203EB031308EBC3035B68ED
:102F7000B1F80CC06344102B11D84FF0000A8946F9
:102F80007C4B7D4F1B684FEA8C0E0093B96891B162
:102F90000AF1010ABAF1050F07F10C07F6D148F260
:102FA000071B584607B0BDE8F08F48F20E1B584685
:102FB00007B0BDE8F08FBCF1000F61D00D460C46A4
:102FC000D9F810300EEB030B5A8833F8046B154414
:102FD0009B4502FB0644F7D1D9F80830A342D7D36A
:102FE000009B2B44B3F5007FD2D2634C0AEB4A021C
:102FF0009200C0F800A0A01844F80290009A8B46F6
:10300000C0E9012599F801205A48012A0360C8D077
:10301000B9F80C30002BC4D00025CDF80490CDF8C1
:103020000CA0CDF814B0019B1F781A693B0103EB8B
:103030000709009308EBC903596832F8254002914B
:1030400039BB039ADD609A60009B3B441F4608EB46
:10305000C3014B6858F83720013394424B6012D9B2
:10306000019B48F837409B8901359D42DBD3DDF851
:1030700014B096E748F2081B584607B0BDE8F08F39
:10308000009B6546AEE7019B01359B89AB42CAD8E0
:10309000EDE7002601F1FF3A049506EB0A0009EB83
:1030A00006020132013058F832C04008324D09EBB7
:1030B000000109EB0A03013101330CEB4C0C58F809
:1030C00031E055F82CB058F833C008EBC2020EEBD3
:1030D0004E0E0CEB4C0CDBF810B0526855F82EE09D
:1030E00055F82CC008EBC10108EBC3033BF82220C4
:1030F000DEF810E04968DCF810C05B6894423EF8E6
:1031000021103CF823302DD99C422DD28C4224D959
:10311000461CB245C1D21026049D029AB24211D972
:10312000009B3B441A44334408EBC20A08EBC30932
:10313000082251460AEB0200AAF1080A09F0A2F897
:10314000D145F5D1009B03993B443344013308EB4F
:10315000C30248F83310556076E700F1FF3A564550
:103160009BD9D8E7049DD8E7049D0AF10106D4E76E
:10317000A21F0220F41B0220F81B0220341C022094
:10318000034B1B780BB1FFF78DBD1846704700BF8E
:10319000A21F022038B5084B1D7855B101FB00F481
:1031A0002046FFF77FFD054618B12246002109F0B1
:1031B00096F8284638BD00BFA21F0220044B1B789A
:1031C00023B118B101460020FFF71CBC704700BFB7
:1031D000A21F0220034B1B780BB1FFF77FBC1846E0
:1031E000704700BFA21F0220044B1B7823B118B107
:1031F00001460120FFF706BC704700BFA21F022056
:1032000038B50A4C0A4B2578072A28BF07220846FA
:1032100003EB451109F036F8237800200133DBB2C7
:10322000072B08BF0023237038BD00BFA31F022057
:1032300090D70100F0B5E5B09DF8A87158B152B132
:103240004BB11F2907D919683F2904D93FB1552926
:1032500005D80C2400E01624204665B0F0BD1D46BC
:10326000042300210446164614A84FF4A0728DF8DA
:103270000C3009F034F814A804F00AFF002329499F
:103280001A4614A8009305F005F814A82022214638
:1032900005F028F8B8B914A804F000FF21460DF194
:1032A0000D0008F0D1F80446B8B9C7B114A800F071
:1032B0003FF8022000F042F8014614A800F04CF854
:1032C000A8B10E24C8E7184A184B117820460722E7
:1032D00003EB411108F0D6FFDDE72324BCE703A987
:1032E000701C402208F0CEFF41232B60B4E703217D
:1032F000159806F0FBFE0028E3D1159803AA00F10B
:103300008801412306F0F6FC0028DAD1314614A8E2
:103310002A6800F06FF8B22304462B6000289BD087
:10332000CFE700BF01320100A31F022090D70100A8
:1033300010B10023C0E90033704700BF022805D058
:10334000034B03280CBF1846002070470148704704
:10335000A8D8010078D8010060B159B170B50668ED
:1033600066B94B6A04460D469847606020B12560F7
:10337000304670BD02487047024870BD004870BDBD
:1033800080C1FFFF80C0FFFF10B1006800B100786E
:10339000704700BF023802288CBF00200120704710
:1033A000806D70470222034B883088600A704B6042
:1033B000704700BF70D80100023801288CBF002080
:1033C0000120704710B5044605F03AFE2046BDE8DE
:1033D0001040FFF7F3BE00BF10B5AC210120FFF78E
:1033E000D9FE044608B105F0C5FD204610BD00BF5A
:1033F00006F09EBD2DE9F04F0024D7B00DF5AB735C
:1034000088469146CDE906430746FFF7BDFF0228EF
:1034100059D1852378680BAE0193224600F18801CB
:1034200000960AAB0A9406F013FC2DAD044668B969
:103430000798A8427FD30A9A431B93427BD3831AEF
:1034400018463146079308F01DFF0A9C002C31DB1B
:10345000079B5A1B002A6EDD00215A1E04F1010A47
:10346000079207A803F8011C5246294601F058FDAF
:10347000041E1FDB0322294607A801F0CBFDB0F193
:10348000000B1BDB3846FFF77FFF08AA09A906F0EF
:103490006FFE0346C8B1002B50DBC3F1A20206A9A0
:1034A000CDE90191CDF800802A442549254806F050
:1034B00097FE0446204657B0BDE8F08F5C46204694
:1034C00057B0BDE8F08F204CF4E705903846FFF781
:1034D0005BFF0228059B1DD01846DDE908320090ED
:1034E000294607A801F0ECFD002822DB5444A34440
:1034F00083445A46294607A801F012FD041ED9DB71
:1035000007A83022294601F085FD031E16DBA344DF
:103510005B44C0E77B68324618780AA906F044FE8F
:1035200028B933680A9A294607A801F081FD0028C6
:10353000D3DA0446BEE76FF06B04BBE71C46B9E77D
:10354000E4D8010000D9010080C6FFFF012838B58A
:103550000D46144611D002280AD11020FFF710FEA4
:10356000182220B1074B456013448460036038BDC6
:103570000C20FFF705FE0022F3E71420FFF700FE02
:103580003022EEE71CD9010010B5044603681B6920
:103590009847236820465B6998472046BDE810405D
:1035A000FFF70CBE10B504460C20FFF7E9FDE06004
:1035B00028B100232361BDE8104001F0D9BB0420ED
:1035C00010BD00BF70B5064614200D46FFF7D8FDAC
:1035D00078B12B68044643606B6801468360EB68F2
:1035E000C360AB680361F06801F0CCFB20B9686888
:1035F00070BD4FF0FF3070BD2046FFF7DFFD4FF08C
:10360000FF3070BD2DE9F04F824687B0C068894613
:10361000934601F0D7FB002872D00546D9F8080080
:1036200020B12B6913B1EA68002A5CD10023C9F8E4
:103630000C30D9F80020D9F80480DAF81010019283
:10364000B8F1000F5AD00BF008030024009310E0EB
:10365000DAF810303B44CAF81030284601F0BAFBC3
:103660003C440546002838D0A04536D90021D9F879
:103670000020AE68A8EB040B761A5E45374628BFDB
:103680005F4632B16868019B01443A46181908F058
:10369000F9FD009B002BE0D15E45D9D8DAF80C008B
:1036A00001F086FB064670B1D0E90123D0E90301A1
:1036B000CDE90223CDE90410DAE9013102A89847E7
:1036C0003046FFF77BFD00232846CAF8103001F092
:1036D00081FB3C4405460028C6D12046C9F8044079
:1036E00007B0BDE8F08FD9F80C309A4228BF1A46CF
:1036F000C9F80C20296908F0C5FD9AE74446ECE7B3
:103700004FF0FF30ECE700BF10B50446C06801F091
:1037100059FB50B12469644283681C4401F05AFB90
:103720000028F9D124EAE47010BD4FF0FF3010BD3D
:1037300030B50546C06885B0A8B91AE0E86801F060
:1037400037FB044670B1D0E90101D4E90332CDE979
:103750000001CDE90223D5E90131684698472046AA
:10376000FFF72CFDE86801F033FB0028E6D105B037
:1037700030BD082005B030BD30B50546C06885B005
:10378000A0B91CE001F014FB044670B1D0E90101BE
:10379000D4E90332CDE90001CDE90223D5E90131B5
:1037A000684698472046FFF709FDE86801F010FBDE
:1037B0000446E868002CE5D1FFF700FDEC6005B099
:1037C00030BD00BF006801F0CBBA00BF70B582B059
:1037D0000E4614460546FEF74DFB002842D003680E
:1037E0009B033FD50368214623F40033036003683D
:1037F00043F48013036001A801F088FA80BB04221F
:10380000019B1A7258729872D872DD6084B918469A
:10381000012101F08FFAD0B94FF400322846114649
:103820004FF0FF33FEF7B6FAA8B9204602B070BDDC
:1038300031461868224608F025FD0121019801F063
:1038400079FA0028E8D0019B186801F089FA0198FC
:1038500001F07EFA232008F086FF4FF0FF30E5E705
:103860000C20F8E71620F6E701F04ABA2DE9F041FE
:10387000002582B002AB43F8085D80460F4618462B
:10388000164602211D4AFEF7EFF9009B04460BB3D2
:10389000C3E902871E61294601A801F037FAE8B999
:1038A0000422019B052158729872D8721A72DC604A
:1038B000184601F03FFAD8B902224FF0FF33114603
:1038C0002046FEF767FA054648B9009A136843F4A4
:1038D00000331360204602B0BDE8F0810C2520467D
:1038E000FEF716FA284608F03EFF4FF0FF34F1E7E6
:1038F000019801F02DFA2325F1E700BFC53701003B
:10390000F0B583B00646FEF7B5FA00283DD00D238A
:1039100007680360036804469B031FD4002101A8C5
:1039200001F0F4F920BB0422019B06215872987221
:10393000D8721A72DE60184601F0FCF9D0B90E2276
:103940004FF0FF3311463046FEF724FA0546A8B97A
:103950003046FEF7DDF9284603B0F0BD03680021CC
:1039600023F40033036001A801F0D0F90028DAD075
:103970000C2503E0019801F0EBF923252760284688
:1039800008F0F1FE4FF0FF35E5E71625F7E700BF39
:103990002DE9F04184B0884615461E460746FEF7DD
:1039A00069FA002849D00023CDE9008516F0020508
:1039B0000446CDE902330ED01EE0002D33D14FF482
:1039C0008032E3691146002B08BF4FF0FF333846C1
:1039D000FEF7E0F905462368A06923F480332360ED
:1039E000036832469B6869469847B0F10008E4DBFB
:1039F000404604B0BDE8F0810368806923F4803359
:103A00002360036832469B6869469847B0F1000816
:103A1000EEDAB8F1FF3FEBD1232008F0A4FE4046D8
:103A200004B0BDE8F081B8F1FF3FE1D1284608F0CD
:103A30009AFE404604B0BDE8F081162008F093FEDF
:103A40004FF0FF38D4E700BFFEF734BA012901D0A8
:103A50002A20704738B51D461446FEF70BFA034678
:103A600068B1142C07D165B1049A042A05D12A68DB
:103A70000020DA6138BD2A2038BD162038BD092063
:103A800038BD0E2038BD00BF70B5054684B0C06893
:103A90000E46FEF7EFF940B3036804469BB2012BD4
:103AA0001FD003689BB20D2B27D003689BB2022B5B
:103AB0002ED0033E012E11D8002329686A68CDE973
:103AC0000233CDE90012A069694603685B68984734
:103AD000013017D0236843F480332360002004B002
:103AE00070BD022EE5D10660F8E728680028F5D001
:103AF00001F036F9002004B070BD022ED9D10E239A
:103B00000360EBE7286801F02BF9002004B070BDDA
:103B10000368DB02CDD5022ECBD1036823F48013DA
:103B20000360036843F400330360D7E750F8081BD1
:103B3000090CFDF727BE00BF0148FEF77FBA00BFA2
:103B400064D90100002310B582B0019358B1044636
:103B500001AA0420FEF7B2FC18B9019B0BB108338F
:103B6000236002B010BD072002B010BD01F4704305
:103B7000B3F5E04F0BD160B1034630F8082C0420B8
:103B800042EA014143F8081D1946FEF77FBC0F20A9
:103B900070470720704700BF20B1A0F10801042042
:103BA000FEF7C0BC0720704718B101460420FEF79D
:103BB00069BD0720704700BF2DE9F0410C460B6836
:103BC000496923F4003323602268002322F4002291
:103BD000226047F2810227680646FCF717FE00289C
:103BE0003BD00546284B06EBC60103EB810124229E
:103BF000143008F047FBAB68DFF890802433AB60EB
:103C00002368294603EA080343F00A03236047F2C6
:103C100081023B462046FCF719FE60B923681B0170
:103C20000BD44FF0FF334FF6FF720B213046FCF7F9
:103C300021FE28B12760BDE8F0817320BDE8F08146
:103C40004FF00072304611464FF0FF33FCF712FE82
:103C500030B17328EFD02760EDE70C20BDE8F0818C
:103C6000236823F000732360236803EA080848F000
:103C70000C032360236843F400332360236843F478
:103C800000232360BDE8F081441D02200000FFFFF7
:103C90000020704738B520F00803022B06D02F20F3
:103CA00008F061FD4FF0FF35284638BD14464A1E26
:103CB000012A28D814BB012906BF01234FF48274BE
:103CC0004FF487741A46FCF701FE051E26DB154BE0
:103CD00005EBC50003EB80002422134908F0D2FA5B
:103CE0002846FEF7C7F80368046123F40023036045
:103CF000036823F400330360284638BD012908D047
:103D0000B4F5877FDED0162008F02DFD4FF0FF358B
:103D1000CAE7B4F5827FF6D10B46D3E74FF0FF3503
:103D2000C2E700BF441D022074D9010010B504464B
:103D3000FEF7A0F820B12046BDE81040FCF760BEB9
:103D4000092008F010FD4FF0FF3010BD2DE9F047BD
:103D50000D46DDE9088916461F460446FEF78AF837
:103D600000283BD003689BB20C2B39D003689BB270
:103D70000B2B11D1204B04EBC40413F82430022B7D
:103D800038D0C368012B14BF39202A2008F0EBFC7F
:103D90004FF0FF30BDE8F087C368012B0BD0022B3A
:103DA00001D03920F2E703689BB2022B07D00368E9
:103DB0009BB2042B03D003689BB2052BF1D10E4BB1
:103DC00004EBC40213F82230022BEAD1014620464C
:103DD000FFF7F2FE002803D0D8DCD9E70920D5E7A9
:103DE000CDE908893B46324629462046BDE8F047E2
:103DF000FCF776BE2320C9E7441D02202DE9F043DD
:103E000083B00D46DDE90A8916461F460446FEF7D3
:103E100031F8002839D003689BB20C2B2AD0C36834
:103E2000012B12D0022B08D04FF0FF34232008F0D2
:103E30009AFC204603B0BDE8F08303689BB2022BD6
:103E400007D003689BB2042B03D003689BB2052BF9
:103E5000EAD1154B04EBC40213F82230022BE3D154
:103E600001462046FFF7A8FE002812D04FF0FF348D
:103E7000DDDCDEE72046CDE900893B4632462946B7
:103E8000FCF702FF04462320D1E74FF0FF3409205E
:103E9000CDE73B46324629462046CDE90A8903B0A4
:103EA000BDE8F043FCF7F0BE441D02202DE9F843C5
:103EB0000C4617460646FDF7DDFF00284CD0036888
:103EC00005469BB2022B50D121463A463046FDF7BB
:103ED00055F8044620B1002C3FDC2046BDE8F883AD
:103EE00006EBC607DFF89480BF0018F80730012BF7
:103EF000F3D1034647F2810269693046FCF786FC3C
:103F00008146B0B308EB07012422143008F0BAF957
:103F1000D9F8083049462433C9F808302A68042300
:103F2000120C120442F00A022A60284647F281026B
:103F3000FCF78CFCF8B92B681B0118D430464FF005
:103F4000FF334FF6FF720B21FCF794FC0028C4D01E
:103F5000042304462B60BEE7092420464FF0FF34BB
:103F600008F001FC2046BDE8F8832D24F5E7732412
:103F7000F3E70C24F1E70446ADE700BF441D02203F
:103F8000F8B50E4617460446FDF774FFE8B1134B2B
:103F900004EBC40213F82230022B1CD1036805463F
:103FA0009BB2022B03D003689BB2042B13D13A4679
:103FB00031462046FCF73CFF10B1002806DCF8BD76
:103FC00029462046FFF7F8FDF7E7092008F0CBFB6C
:103FD0004FF0FF30F8BD2D20F8E700BF441D022050
:103FE0002DE9F0470F460646FDF744FF00286BD049
:103FF000C3680446012B65D103689BB2042B56D0DD
:1040000023689BB20B2B5DD1F300DFF8C0909A19A7
:1040100019F82220012A55D1012233449D0009F8C4
:1040200005206169002347F281023046D4F8008000
:10403000FCF7ECFB8246002842D009EB0501242264
:10404000143008F01FF9DAF8083051462433CAF862
:10405000083022684346120C120442F00A02226021
:10406000204647F28102FCF7F1FBE0B923681B010F
:104070000ED44FF0FF334FF6FF720B213046FCF7A2
:10408000F9FB60B10028C4F8008002DCBDE8F087CD
:10409000732008F068FB4FF0FF30BDE8F087394629
:1040A0003046FDF701F80028F3DCBDE8F087F300A7
:1040B000DFF818909A1919F82220022AA0D1ABE74C
:1040C0000C20E6E72D20E4E70920E2E7441D02206A
:1040D000F8B50C4616461F460546FDF7CBFE0028F0
:1040E0003BD0006880B2062837D121463B46324695
:1040F0002846FDF74FF8044618B1002C2EDC204668
:10410000F8BD2846FDF7B6FE0368184F23F40033C8
:104110000360036805EBC50523F40023064603602E
:1041200007EB85012422384608F0ACF802233B70E7
:10413000336820461B0C1B0443F00B0333604FF61F
:10414000FF724FF0FF330C21FCF794FB044600286C
:10415000D5D00020FCF754FCCFE7092420464FF0CF
:10416000FF3408F000FB2046F8BD00BF441D0220CC
:104170002DE9F041B1F58D7F069F1DD11C46C3B1DD
:10418000BFB105461646FDF775FEC8B103689BB280
:10419000022B07D003689BB2042B03D003689BB2A9
:1041A000052B0DD1013E032E51D8DFE806F0253254
:1041B000180B0E20BDE8F081BDE8F041FDF722B9F3
:1041C0000920F7E7042F39D12368022B36D8214A7A
:1041D00005EBC50502EB8505AB700020EAE7012F72
:1041E0002CD12378012B29D81A4A05EBC50502EBFF
:1041F000850253700020DDE7042F1FD12068F8B13D
:1042000001281BD1134B05EBC50503F82500002041
:10421000D0E75FEA970C11D017F003060ED105EB3B
:10422000C505AD000B4B281D18442B443A462146CA
:1042300083F803C008F026F83046BBE71620B9E73C
:104240000222044B05EBC50503F82520B2E72A201E
:10425000B0E700BF441D02202DE9F041B1F58D7F8C
:10426000069F12D11D466BB167B106461446FDF795
:1042700001FE00284FD0013C032C52D8DFE804F0A7
:10428000392115090E20BDE8F081BDE8F041FDF7A8
:104290006FB93B68042B3CD1234B06EBC60603EBFE
:1042A0008606B37800202B60EDE73B68042B30D105
:1042B0001D4B06EBC60603EB8606737800202B60C9
:1042C000E1E706EBC60618493B68B6008A1913F009
:1042D0000304D07821D19B08834228BF03469A006B
:1042E000DBB1043631443A60284607F0CBFF204664
:1042F000C9E73B68042B0CD10B4B06EBC60613F841
:1043000026300020A3F10103B3FA83F35B092B608D
:10431000B9E71620B7E70920B5E70028F9D13860DA
:10432000B1E72A20AFE700BF441D022038B548F2AC
:104330008105AB420C4653D049F282018B422DD00D
:1043400048F202018B4201D0012038BD002CFBD085
:104350002369B3F5827F02D0B3F5877FF4D1236858
:1043600023F0805323605569002D48D123681B0C2E
:104370001B0443F00503236023681A010CD5254B69
:1043800000EBC00213F82230022B05D12146FFF7C3
:1043900013FC08B1732835D1002038BD002CFBD0A8
:1043A00023689BB20B2BF7D1106948BB236843F0FD
:1043B0000073236023681B01EED5236823F000738C
:1043C000236023681B0C1B0443F00C032360236849
:1043D00043F400332360236843F40023236038BD93
:1043E0000029D9D00B689BB20A2BD5D1506938B9B6
:1043F0000B681B0C1B0443F00B030B6038BD2846F5
:10440000FCF7FAF960602368002043F480232360FE
:1044100038BD00BF441D022008B5084AC168128893
:104420000346B2EB114F05D0006810B100F010FD4B
:10443000002008BD024A0120136008BD761E02203C
:104440006C1E0220002310B508480949094A0A4C8D
:1044500003800B601360236000F0C4FC10B90123DB
:10446000236010BD4FF0FF3010BD00BF761E02204C
:104470006C1E0220681E0220641E0220012808B55E
:104480000DD140F203239A4209D1022907D80A4BE1
:104490001A68012A09D102221A60084808BD1620AC
:1044A00008F061F94FF0FF3008BD0E2008F05BF90D
:1044B0004FF0FF3008BD00BF641E02203254764921
:1044C0002DE9F0434F4B85B0984240F095804E4C1B
:1044D0002368012B62D02368002B5FD02368072B51
:1044E0005CD0072325682360052D5DD0062D05D0FF
:1044F000042D03D0002005B0BDE8F0830627B846A0
:104500000021424E424BC6F81C161B6801A80293BC
:10451000029B00F06DFC0346002848D1019870B35F
:104520004FF0040EDFF8F0C04372BCF80020837235
:10453000013292B247EA0247C760364FC372037135
:1045400043718371C371414680F808E0ACF80020E4
:104550003B6000F061FC002832D0019803681BB179
:10456000184600F075FC019800F06AFC23202560D5
:1045700008F0F9F84FF0FF3005B0BDE8F0832320D4
:10458000256008F0F0F8234B18680028F2D00123CA
:104590002360046900F054FC002CABD00E2008F01E
:1045A000E2F84FF0FF30A6E72F46A846A8E7232001
:1045B000256008F0D8F84FF0FF3005B0BDE8F08373
:1045C0004FF0FF330DF1100848F8043DDFF8389044
:1045D00008E0D6F81C36002BCCD141464846F7F708
:1045E000F9F820B938680028F3D0C368CFE73C2039
:1045F000256008F0B8F8BDE7092008F0B4F84FF0DE
:10460000FF3078E732547649641E022000A0024051
:104610001CA602406C1E0220761E02202DE9F047E7
:10462000964B84B0984240F01C810F46002900F060
:1046300012811546002A00F00E81914C2368022B4E
:1046400003D02368042B40F000812668022E56D048
:1046500000218C4A8C4BC2F81C161B682946029319
:1046600001A8029B00F0C4FB002840F09980019B48
:1046700093B31868002800F09E8039462A4607F058
:1046800001FE04210022814F01983B8845600133DF
:104690009BB21E040E43C6607D4E0172427282724E
:1046A000C2723B80326000F0B7FB002800F08C80C3
:1046B000019803681BB1184600F0CAFB019800F08E
:1046C000BFFB04232320236008F04DF84FF0FF3593
:1046D000284604B0BDE8F08704232320236008F0B7
:1046E00042F86B4B18680028F0D0046900F0A8FB72
:1046F000002C40F0AA80284604B0BDE8F0870021D5
:10470000DFF88081604BC8F81C161B6802A8009374
:10471000009B00F06DFB034600286ED1029878B331
:104720000421DFF868C15B4EBCF800203668013216
:1047300092B20172110441F003010661544EC1604E
:1047400043728372C372037143718371C371032116
:10475000ACF80020336000F05FFB002857D00298CF
:1047600003681BB1184600F073FB029800F068FB69
:104770000223232023604FF0FF3507F0F4FFA7E763
:104780002320266007F0EFFF414B186800289DD0DA
:10479000066900F055FB002E57D10423236057E72C
:1047A00004234FF0FF352320236007F0DCFF284669
:1047B00004B0BDE8F087184600F042FB0423232034
:1047C000236007F0D0FF5CE74FF0FF3304AFDFF862
:1047D000B48047F8043DDFF8A89009E0D8F81C360B
:1047E000002B7FF473AF39464846F6F7F3FF30BB32
:1047F00030680028F2D0C36877E74FF0FF352320F8
:10480000266007F0B0FF284604B0BDE8F0874FF0FF
:10481000FF330DF1100949F8043DDFF864A009E009
:10482000D8F81C36002B7FF451AF49465046F6F7B6
:10483000D1FFE0B930680028F2D0C368A8E70423AC
:104840003C20236007F08FFF40E70E2007F08BFF2E
:104850004FF0FF354FE7162007F085FF4FF0FF358B
:1048600049E7092007F07FFF4FF0FF3543E70223B8
:104870003C20236007F077FF28E700BF32547649D9
:10488000641E022000A002401CA60240761E0220E8
:104890006C1E0220681E02204FF0FF30704700BFE0
:1048A0002DE9F0435E4C85B0A04240F0AE8040F26E
:1048B0000320814240F08680111F032900F282808C
:1048C000584C2168002900F09A802168012900F0E5
:1048D00096802168072900F09280062A66D0072A70
:1048E00007D0052A11D005230020236005B0BDE8BC
:1048F000F083002B66D00C9A042A63D100201A683A
:10490000494B1A6005B0BDE8F0830725A846002191
:10491000464E474B2768C6F81C161B6801A8029331
:10492000029B00F065FA0346002842D1019868B363
:104930004FF0040EDFF800C14372BCF80020837210
:10494000013292B245EA0245C5603A4DC372037125
:1049500043718371C371414680F808E0ACF80020D0
:104960002B6000F059FA98B3019803681BB1184600
:1049700000F06EFA019800F063FA2320276007F038
:10498000F2FE4FF0FF3005B0BDE8F0832320276032
:1049900007F0E9FE274B18680028F2D0046900F000
:1049A0004FFA64BB204605B0BDE8F0830825A84651
:1049B000ADE72320276007F0D6FE4FF0FF3005B0AB
:1049C000BDE8F083162007F0CEFE4FF0FF308DE7F4
:1049D0004FF0FF330DF1100848F8043DDFF8449024
:1049E00008E0D6F81C36002BCBD141464846F6F7F6
:1049F000F1FE80B928680028F3D0C368CEE70E2006
:104A000007F0B1FE4FF0FF3070E7092007F0ABFE72
:104A10004FF0FF306AE73C20276007F0A4FEB0E7C4
:104A200032547649641E0220681E022000A0024013
:104A30001CA602406C1E0220761E02202DE9F04FBB
:104A40006E4C85B0A0421E460E9B40F0C88040F2DE
:104A50000320814240F0B180002E00F0AE80002B98
:104A600000F0AB80511E082900F2A780644C216839
:104A7000002900F0AE802168012900F0AA80216899
:104A8000072900F0A680022A1F6878D0072A4ED096
:104A9000012A6FD00025A94600215A4A5A4BD4F862
:104AA0000080C2F81C161B6801A80293029B00F04C
:104AB0009FF9002858D1019B002B3DD04FF0040EE8
:104AC000DFF850C1B9F1030FBCF80010587201F1C2
:104AD000010189B245EA01429872D8721871587181
:104AE0009871D871DA60ACF8001083F808E002D150
:104AF000464A12681A610022454D494618462A6006
:104B000000F08AF900283FD0019803681BB11846CD
:104B100000F09EF9019800F093F92320C4F800807A
:104B200007F021FE4FF0FF3005B0BDE8F08F042FF5
:104B300043D10925A946AFE7354D2320C4F80080AD
:104B400007F011FE29680029ECD00C69002C4CD12B
:104B50003A461431304607F095FB286800F070F9AA
:104B6000204605B0BDE8F08F2320C4F8008007F090
:104B7000FAFDD7E7242F20D1154691468CE7042F64
:104B80001BD10225A94687E74FF0FF330DF110092D
:104B9000DFF870A049F8043DDFF864B008E0DAF807
:104BA0001C36002BBED149465846F6F713FE50B9C5
:104BB00029680029F3D0CB68C7E7162007F0D3FD9A
:104BC0004FF0FF30B0E73C20C4F8008007F0CBFD89
:104BD000A8E70E2007F0C7FD4FF0FF30A4E709203B
:104BE00007F0C1FD4FF0FF309EE70E2007F0BBFD40
:104BF000286800F025F94FF0FF3095E732547649E8
:104C0000641E022000A002401CA60240681E022072
:104C10006C1E0220761E0220FCF7ACBCFCF794BD93
:104C20002DE9F04342EAE27283B00092002847D0B7
:104C30004B1E072B44D880460546002400EBC107D5
:104C4000AB88286803F0030301A943F00C06FDF7C5
:104C50001FF9019B0835334025F8023C03B10134AC
:104C6000BD42EDD194BB69464046F6F7B3FD074619
:104C700008B13C281DD1C1460026B9F80430D9F846
:104C8000000003F0030301A943F00C04FDF700F951
:104C9000019B09F10809234029F8023C03B10136C0
:104CA0004D45EAD10EB9002FDDD0304603B0BDE846
:104CB000F08307F058FD4FF0FF3003B0BDE8F083FC
:104CC000162007F050FD4FF0FF30EFE72046EDE7EC
:104CD00008B5064B834303D0BDE80840FDF716B97D
:104CE0002D2007F040FD4FF0FF3008BD32547649CB
:104CF00020B150F8081B090CFEF7C6BE704700BF74
:104D00000148FDF79BB900BF98D9010080B100238D
:104D100010B582B002AA044642F8043D0320FDF714
:104D2000CDFB18B9019B0BB10833236002B010BD55
:104D30000E20704750B1034630F8082C032042EA99
:104D4000014143F8081D1946FDF7A0BB0E2070472E
:104D500020B1A0F108010320FDF7E4BB0E2070474D
:104D600018B101460320FDF78DBC0E20704700BF2F
:104D700028B100230360C0E90133184670470720BB
:104D8000704700BF0268034601320ED000220A605D
:104D900002683AB18268116081601A6800200132AD
:104DA0001A607047C0E90111F7E70420704700BF9F
:104DB0000346006828B158681A680168013A5960CA
:104DC0001A60704703680BB1406870471846704717
:104DD000006870470068704750F8081B090CFFF71F
:104DE0001BBB00BF0148FDF729B900BFA8D90100CE
:104DF000002310B582B0019358B1044601AA0620E1
:104E0000FDF75CFB18B9019B0BB10833236002B0BE
:104E100010BD072002B010BD11F4704F0BD160B16E
:104E2000034630F8082C062042EA014143F8081DE9
:104E30001946FDF72BBB0F2070470720704700BFB6
:104E400020B1A0F108010620FDF76CBB07207047D8
:104E500018B101460620FDF715BC0720704700BFBA
:104E600030B403460068B2F5803FA0EB010114D2D4
:104E7000022951DD411E196000F8012C19688224B5
:104E8000481E18600320120A01F8012C1A68511EEE
:104E9000196002F8014C30BC7047B2F1807F1AD221
:104EA000032939DD8324411E196000F8012C19689B
:104EB000100A4D1E1D6001F8010C1968120C481EE5
:104EC000186001F8012C1A680420511E196002F8BC
:104ED000014C30BC704704291EDD8424411E19603A
:104EE00000F8012C1968100A4D1E1D6001F8010C14
:104EF0001968100C4D1E1D6001F8010C1968120E86
:104F0000481E186001F8012C1A680520511E19600E
:104F100002F8014C30BC70476FF06B00BBE700BF7C
:104F200030B404687F2A0346A4EB010108D80029A5
:104F30006CDD611E0160012004F8012C30BC70475B
:104F4000FF2A0ED8012961DD8121601E186004F856
:104F5000012C1A680220541E1C6002F8011C30BC8F
:104F60007047B2F5803F1CD3B2F1807F2ED2032967
:104F70004CDD8325611E016004F8012C0168100AD4
:104F80004C1E1C6001F8010C1968120C481E1860B8
:104F900001F8012C1A680420511E196002F8015C06
:104FA000CCE7022932DD8225611E016004F8012C64
:104FB0000168120A481E186001F8012C1A680320C3
:104FC000511E196002F8015C30BC704704291DDDD8
:104FD0008425611E016004F8012C0168100A4C1E32
:104FE0001C6001F8010C1968100C4C1E1C6001F8C3
:104FF000010C1968120E481E186001F8012C1A687D
:105000000520511E196002F8015C97E76FF06B00F4
:1050100094E700BF0368591A002905DD591E016095
:10502000012003F8012C70476FF06B00704700BF40
:10503000F8B50568A9423FD80F46691A8B423BD89C
:1050400006461C46E81A114630601A4607F01AF95F
:10505000002C204615DB7F2C14D83368DA1B002A7D
:105060002ADD01205A1E326003F8014C33680134F6
:10507000DF1B002F20DD0622591E3160204403F87B
:10508000012CF8BDFF2C0FD83368DA1B012A13DD81
:105090008122591E316003F8014C33680220591EE9
:1050A000316003F8012CE1E7224639463046FFF72C
:1050B000D7FE0028DADAF8BD6FF06B00F8BD00BF4C
:1050C0002DE9F041DDF818800568B8F1000F13D123
:1050D0006C1A002C40F387806C1E046005F8018C6C
:1050E0000468651A002D7EDD05254FF00208661E56
:1050F000066004F8015C0568A94274D86C1AA342E2
:1051000071D806461C46E81A0F46306011461A460A
:1051100007F0B8F8002C20462FDB7F2C41D83368ED
:10512000DA1B002A5FDD01205A1E326003F8014CB1
:1051300033680134DA1B002A55DD06220444591E67
:10514000002C3160204603F8012C16DB44447F2CF0
:1051500015D83368DA1B002A45DD01205A1E32605B
:1051600003F8014C33680134DF1B002F3BDD302294
:10517000591E3160204403F8012CBDE8F081FF2C5A
:1051800021D83368DA1B012A2DDD8122591E3160B6
:1051900003F8014C33680220591E316003F8012CDA
:1051A000E0E7FF2C17D83368DA1B012A1BDD8122C8
:1051B000591E316003F8014C33680220591E3160DA
:1051C00003F8012CB4E7224639463046FFF748FE83
:1051D0000028D2DBC6E7224639463046FFF740FEBC
:1051E0000028A5DAC9E76FF06B00C6E72DE9F04F9C
:1051F000DDF824C0BCF1000F65D0424CA4FB0C5478
:10520000640804EB4408C44518BF0134B4F1804F6E
:1052100071D2A40001348C4269D8002867D0B8F15B
:10522000000F61D086460027374EDC1C002514F89D
:10523000031C14F8023C14F801BC4FEAA10909014F
:1052400001F0300106EB131A16F809909B001AF8CA
:1052500001A003F03C0106EB9B13595C69F30705C1
:105260000BF03F03F35C6AF30F2561F31745033737
:1052700063F31F650EF10401B845CEF800502346D4
:105280008E4604F10304D1D8BC4514D91C781E4DB8
:105290000137A61067454FEA041404F0300415F8EE
:1052A00006E015D33D262B5D81F800E04B703D23D1
:1052B0008E70CB70043100239C46081A10600B706E
:1052C0006046BDE8F08FC2F800C06046BDE8F08FD0
:1052D0005B7881F800E005EB1316345D9B0003F06A
:1052E0003C034C70EE5CE2E747460146CCE71460B5
:1052F0006FF0290CE4E74FF0FF336FF0290C1360D7
:10530000DEE700BFABAAAAAAB8D901000F282DE991
:10531000F04F864640F2E0824FF00008844601F1EB
:10532000400402F1400054F8406C50F8405CA3FB8C
:10533000066718EB06082CBF4FF001094FF0000973
:1053400015EB08054F444FF0000928BF4FF0010945
:1053500040F8405C54F83C6CB944A3FB06AB19EB35
:105360000A092CBF4FF001084FF0000850F83C6CC0
:1053700008EB0B0516EB09064FF0000828BF4FF0AD
:10538000010840F83C6C54F8386CA844A3FB06674D
:1053900018EB06082CBF4FF001094FF0000950F838
:1053A000385C4F4415EB08054FF0000928BF4FF05B
:1053B000010940F8385C54F8346CB944A3FB06ABDF
:1053C00019EB0A092CBF4FF001084FF0000850F804
:1053D000346C08EB0B0516EB09064FF0000828BFEC
:1053E0004FF0010840F8346C54F8306CA844A3FB2B
:1053F000066718EB06082CBF4FF001094FF00009B3
:1054000050F8305C4F4415EB08054FF0000928BFF9
:105410004FF0010940F8305C54F82C6CB944A3FB00
:1054200006AB19EB0A092CBF4FF001084FF000083A
:1054300050F82C6C08EB0B0516EB09064FF0000832
:1054400028BF4FF0010840F82C6C54F8286CA84491
:10545000A3FB066718EB06082CBF4FF001094FF0BD
:10546000000950F8285C4F4415EB08054FF000097F
:1054700028BF4FF0010940F8285C54F8246CB94467
:10548000A3FB06AB19EB0A092CBF4FF001084FF044
:10549000000850F8246C08EB0B0516EB09064FF0DA
:1054A000000828BF4FF0010840F8246C54F8206C25
:1054B000A844A3FB066718EB06082CBF4FF00109B0
:1054C0004FF0000950F8205C4F4415EB08054FF0F1
:1054D000000928BF4FF0010940F8205C54F81C6C0B
:1054E000B944A3FB06AB19EB0A092CBF4FF0010826
:1054F0004FF0000850F81C6C08EB0B0516EB090682
:105500004FF0000828BF4FF0010840F81C6C54F819
:10551000186CA844A3FB066718EB06082CBF4FF0D5
:1055200001094FF0000950F8185C4F4415EB0805CD
:105530004FF0000928BF4FF0010940F8185C54F8FB
:10554000146CB944A3FB06AB19EB0A092CBF4FF04E
:1055500001084FF0000850F8146C08EB0B0516EB2F
:1055600009064FF0000828BF4FF0010840F8146CFE
:1055700054F8106CA844A3FB066718EB06082CBF70
:105580004FF001094FF0000950F8105C4F4415EB43
:1055900008054FF0000928BF4FF0010940F8105CE2
:1055A00054F80C6CB944A3FB06AB19EB0A092CBFE9
:1055B0004FF001084FF0000850F80C6C08EB0B0599
:1055C00016EB09064FF0000828BF4FF0010840F81D
:1055D0000C6C54F8086CA844A3FB066718EB06088B
:1055E0002CBF4FF001094FF0000950F8085C4F4400
:1055F00015EB08054FF0000928BF4FF0010940F8EE
:10560000085C54F8046CB944A3FB06AB19EB0A0917
:105610002CBF4FF001084FF0000850F8046C08EB65
:105620000B0516EB09064FF0000828BF4FF00108E4
:10563000ACF1100CBCF10F0F40F8046CA84404F15D
:10564000400400F140003FF66EAEAEF110000009DC
:1056500001308001014402440EF00F000728176852
:1056600040F292800C685668A3FB049A18EB090874
:105670002CBF4FF0010C4FF0000C17EB08072CBFAC
:105680000124002417604F680AEB0C05A3FB07896F
:105690002C4414EB08042CBF01250025A61905EBAA
:1056A00009074FF0000528BF012556608E683D446C
:1056B000A3FB0678ED192CBF01240024966808EBA3
:1056C0000407AD194FF0000428BF01249560CE688F
:1056D0003C44A3FB0678E4192CBF01250025D668BD
:1056E00008EB0507A4194FF0000528BF0125D46079
:1056F0000E693D44A3FB0678ED192CBF012400245C
:10570000166908EB0407AD194FF0000428BF012407
:1057100015614E693C44A3FB0678E4192CBF0125B2
:105720000025566908EB0507A4194FF0000528BFAE
:10573000012554618E693D44A3FB0678ED192CBF09
:1057400001240024966908EB0407AD194FF000040A
:1057500028BF01249561CE693C44A3FB069A14EB53
:1057600009042CBF4FF001084FF00008D66908EB80
:105770000A05A4194FF0000828BF4FF00108D461B2
:105780002031A84408382032002800F097800C68A7
:105790001668A3FB049A19EB08082CBF0124002407
:1057A00016EB08064FF0000528BF012554440128D8
:1057B00005EB040816607FD04C685668A3FB049A7A
:1057C00019EB08082CBF0124002416EB08064FF043
:1057D000000528BF01255444022805EB0408566043
:1057E0006AD08C689668A3FB049A19EB08082CBF52
:1057F0000124002416EB08064FF0000528BF012500
:105800005444032805EB0408966055D0CC68D6684C
:10581000A3FB049A19EB08082CBF0124002416EB03
:1058200008064FF0000528BF01255444042805EB65
:105830000408D66040D00C691669A3FB049A19EBE2
:1058400008042CBF4FF001084FF00008A6190AEB1E
:1058500008054FF0000828BF4FF001080528A844AC
:10586000166129D04C695669A3FB049A18EB090408
:105870002CBF4FF001084FF00008A6190AEB0805ED
:105880004FF0000828BF4FF001080628A8445661D1
:1058900012D08C699169A3FB044514EB08082CBF56
:1058A0000123002311EB08014FF0000428BF01245D
:1058B0002B4404EB0308916102EB8002156800237E
:1058C00015EB080528BF012342F8045B4FF00108DF
:1058D000002BF3D1BDE8F08F4FF00008BEE600BF0B
:1058E0004368002B33D030B403F180428568013A1D
:1058F00055F8224005EB82021CB109E052F8044D34
:1059000034B9013BFAD18B681868D0B930BC704704
:105910008A68126892B1012B10D800680B680028C1
:1059200001DD002B11DB002B01DD002816DB2B68CD
:105930009342EBD806D330BC00207047006830BCDF
:1059400070470868404230BC70470120DEE78B6832
:10595000186800B9704708684042FBE74FF0FF3015
:10596000D4E700BF20B100230122C0E900238360F7
:10597000704700BFB0B110B50446806860B162687E
:10598000531E3AB10022013B591C026000F1040091
:10599000F9D1A068FDF712FC00230122C4E900231D
:1059A000A36010BD704700BF70B5426805468A42CB
:1059B0000C4607D842F21073994251D88A4235D327
:1059C000002070BD511E10D0836853F821000028BC
:1059D00049D102F18042013A03EB820303E053F81C
:1059E000040D18B911464A1EF9D101218C4238BF65
:1059F0000C4604212046FDF7CDFB064680B3A9687E
:105A000081B1A20006F03EFCD5E90120531E3AB157
:105A10000022013B591C026000F10400F9D1A86882
:105A2000FDF7CCFBC5E90146002070BD04212046EE
:105A3000FDF7B0FB064698B1A9680029F2D06A6864
:105A4000920006F01FFCD5E90120531E002AE7D082
:105A50000022013B591C026000F10400F9D1DEE78D
:105A60006FF00F0070BD1146C0E700BF884252D0F2
:105A7000F8B58A680E460546002A4ED049684B1E86
:105A80000ED052F8230000283BD101F180410139AA
:105A900002EB810202E052F8040D90BB013BFAD107
:105AA000012433682B606A68A2420CD3AF6892006D
:105AB0000021384606F013FCA200B168A86806F081
:105AC000E1FB0020F8BD04212046FDF763FB0746FB
:105AD000F0B1A96889B16A68920006F0D3FBD5E9F4
:105AE0000120531E3AB10022013B591C026000F113
:105AF0000400F9D1A868FDF761FB2246C5E901471A
:105B0000D5E742F2107231685C1C94422960CAD910
:105B10006FF00F00F8BD002070470028D1D08068DA
:105B200058B169684B1E31B1013B5C1C026000F149
:105B30000400F9D1A868FDF741FB00200123C5E965
:105B40000030A860F8BD00BFF0B54B680D4685B0C9
:105B50001446064651687BB1A86803F18042013AB9
:105B600050F8227000EB820027B14FE050F8042D6E
:105B7000002A4BD1013BF9D189B101F18040A768DE
:105B8000013857F82020002A40F0998007EB800068
:105B900003E050F8042D002A42D10139F9D1002345
:105BA0000122B442CDE9012303937FD0B54205D051
:105BB00029463046FFF75AFF0746A8B9012333604C
:105BC000606880B1D4F808C000F18043013B5CF804
:105BD00023200CEB830322B142E053F8042D002A6A
:105BE0003ED10138F9D10027039860B1029A531EC3
:105BF0003AB10022013B591C026000F10400F9D1C6
:105C00000398FDF7DBFA384605B0F0BD0029C6D091
:105C100001F18040A768013857F82020002AB5D04C
:105C20008B42BCD84BD3002BB9D0A86803F180417C
:105C3000013950F821C057F821E08900E6450844B1
:105C400007EB0102ABD33AD8014606E051F8047DD8
:105C500052F8040D8742A2D831D3013BF6D19EE71A
:105C600000252B46B16851F8046B0135F21A41F852
:105C7000042C5CF8047B0C46BA422CBF4FF0000E9B
:105C80004FF0010ED21B9E422CBF73460EF1010352
:105C9000854241F8042CE6D30BB9A4E7012322681E
:105CA000D11A9A4244F8041BF8D39CE7214601A874
